:020000041000EA
:1000000000B5324B212058609868022188439860DF
:10001000D860186158612E4B002199600221596106
:100020000121F02299502B49196001219960352056
:1000300000F044F80222904214D00621196600F024
:1000400034F8196E01211966002018661A6600F04E
:100050002CF8196E196E196E052000F02FF8012189
:100060000842F9D1002199601B49196000215960AB
:100070001A491B48016001219960EB211966A021F2
:10008000196600F012F800219960164914480160C1
:100090000121996001BC002800D000471248134993
:1000A000086003C880F30888084703B5996A0420EC
:1000B0000142FBD001200142F8D103BD02B5186610
:1000C0001866FFF7F2FF186E186E02BD00000240BE
:1000D000000000180000070000035F00212200005C
:1000E000F4000018222000A00001001008ED00E03C
:1000F00000000000000000000000000074B24E7A12
:1001000000200420E3010010C3010010C50100100D
:10011000C1010010C1010010C1010010C101001097
:10012000C1010010C1010010C1010010C701001081
:10013000C1010010C1010010C9010010CB01001065
:10014000CD010010CD010010CD010010CD01001037
:10015000CD010010CD010010CD010010CD01001027
:10016000CD010010CD010010CD010010CD01001017
:10017000CD010010CD010010CD010010CD01001007
:10018000CD010010CD010010CD010010CD010010F7
:10019000CD010010CD010010CD010010CD010010E7
:1001A000CD010010CD010010CD010010CD010010D7
:1001B000CD010010CD010010CD010010CD010010C7
:1001C00000BE00BE00BE00BE00BE00BEEFF3058054
:1001D000103800BE21482249086006C881F308880B
:1001E000104720480068002801D01C48F3E70DA400
:1001F0000ECC002902D000F012F8F9E71A491B4A88
:10020000002000E001C19142FCD1194988471949F9
:1002100088471949884700BEFDE701C901C29A42D3
:10022000FBD370477C020010C00000204024002057
:10023000FC2500104024002038270020F42800105E
:100240000000042000000420F42800100010042006
:1002500000100420000000007047000000000000B3
:1002600008ED00E0000000D038270020C02B00205F
:100270008D220020A501002019030020F8B5C046FA
:100280000448054B10B5834203D0044B002B00D02B
:10029000984710BD382700203827002000000000B4
:1002A00006480749091A8B10C90FC91810B549101B
:1002B00003D0044B002B00D0984710BD38270020F6
:1002C000382700200000000010B5074C2378002BD1
:1002D00009D1FFF7D5FF054B002B02D0044800E001
:1002E00000BF0123237010BD38270020000000004C
:1002F00040240020054B10B5002B03D004490548CD
:1003000000E000BFFFF7CCFF10BDC04600000000BA
:100310003C27002040240020B0B500AF054B064A22
:100320009A60054B1D68054B1B681C002B009D4601
:10033000A047C04600ED00E000300010043000107F
:1003400080B500AF00F016F803001A0001235340F7
:10035000DBB2002B01D0FFF7DFFFC046BD4680BDFA
:1003600080B582B000AF7860396000F02FF8FFF7F9
:10037000D3FF0000104B10B51B6818680F4B1B68AB
:100380001A68904201D1002010BD8021121A490143
:1003900000F010F90028F6D0094C0A49200000F0BE
:1003A00059F90028EFD008222000074902F0C0F8D0
:1003B00043425841C0B2E7E7A4260020A02600200F
:1003C00004FA03208828002068250020012370B546
:1003D000002201263C4C86B05B42A15C08254B40C4
:1003E0003A498C46190060463140494201405B0859
:1003F000013D4B40002DF5D1A321013289008A42F5
:10040000EBD1DB43A2589A425BD1A368002B58D0B2
:100410002D4B9B689D4209D32D4B186800F0C0F806
:1004200000216422080001F027FEFEE7E368012BAB
:1004300011D12000103000F037F9002841D0206D94
:1004400000F0AAF900283CD0666DA36D0193002E40
:1004500004D100F0B4F901355034D9E78023029675
:100460005B019E4200D90293029800F06FF903905D
:10047000002826D080220199520102F059F8002864
:1004800017D0EFF3108372B6F02212069446802143
:100490000593019B490163441800049302F0CCF8D2
:1004A000802203990498520102F002F9059B83F31C
:1004B0001088802252019446029BF61A019B6344E5
:1004C000C4E706B070BDC04604FA03202083B8ED2F
:1004D00088280020FEE7FEE70020704770B5094C31
:1004E000094A236810684B43C018EFF3108572B6B1
:1004F000F0231B062168C01802F09EF885F31088CF
:10050000002070BD54270020842800200A4810B520
:1005100000680A4C4843821820688018EFF3108462
:1005200072B6F022120680181900029A02F0C0F882
:1005300084F31088002010BD542700208428002058
:1005400070B50D00074918000C68074B6C4319681B
:10055000A4180919049A01F071FF044B00201D60D2
:1005600070BDC0465427002084280020AC270020FE
:10057000802370B5074D04002A00056006495B0121
:10058000064801F007F823682D185A1C65602260A0
:10059000187870BD04E7032058270020B0270020FA
:1005A00010B5034B01001800FFF798FF10BDC046BF
:1005B00030280020F8B51C4B1C4F18601C4B0D0058
:1005C0001960160000218022380001F031FF194C1B
:1005D00054220021200001F02BFF174BE5616360DE
:1005E000164BA360164BE360164B236180235B0020
:1005F0006361A361002D04D02900300001F05EFE8C
:10060000050010236362F033A362E3620E4B3800EF
:1006100063630E4B2100A3630D4B2562E36300F07F
:10062000E3FDC043C00FF8BD84280020B0270020A0
:10063000542700203028002085030020510300208B
:10064000210300201D03002004F9032004F80320E7
:1006500004F70320F0B5104B104E99B005000C00C4
:100660000093300001230E4A03A900F0EBFE00289E
:1006700002DA002019B0F0BDA427BF003B002A0019
:10068000300003A900F086FFB842F2D1054B0120EB
:100690001B682360EEE7C046B4260020B027002088
:1006A00071250020AC270020F0B50027204B87B033
:1006B000204E1F70204D0393204B02000093310009
:1006C0000123280000F0BEFEB8422BDB05AC02235C
:1006D00022003100280000F05DFF022822D1310005
:1006E000280001F05FF823781F2B02D163788B2B51
:1006F00002D0012007B0F0BD01F080F98022104C3B
:10070000104B20001049120227606760A36001F0BF
:1007100076F9200001F0EBFA002805D0310028001E
:1007200001F040F80020E5E70123039A1370E0E7A9
:10073000BC2B002058270020B0270020A82600202E
:1007400000520320B5030020046703200D4B70B551
:100750001B7805000C4C002B09D12B0022000B4903
:100760000B4800F017FF85420AD1200070BD0948F0
:100770002D1944618461C56101F050F90128F4D953
:100780000020F3E7BC2B002004570320582700204B
:10079000B02700200052032070B5802604007601A7
:1007A000002C01D1012070BD2500B44200D93500D4
:1007B0002800FFF7CBFF0028F5D0641BF0E7704757
:1007C00010B50A68046803000020944208D05B68F2
:1007D00049688B4204D08C4202D0D01A431E984103
:1007E00010BD02008005801501304142484180184B
:1007F0008005800D043070470300826A2833002A88
:1008000004D01A688A4202D10A681A60704713003D
:100810001268F4E7F0B58BB0109E0493129B099216
:10082000F218836E0C00DB6905909A4205D8C36EFE
:10083000002B23D0049A934220D8542040427CE0DD
:100840002368049A129F9A4222D16168A5684D19C3
:10085000AE421DD28E4216D3AD1BBD4200D93D0023
:10086000E368711A59182A00119801F0E7FD119BED
:1008700076195B191193129B5B1B1293129B002B31
:10088000DED1180059E0129B8F1B9F4200D91F0038
:10089000059B30009D6E6B691900039301F00EFDFE
:1008A0006B68099A0793129B0691934220D3002903
:1008B0001ED1129B039A93421AD31100380001F003
:1008C000FDFC7B1A28000691039300933200119BD4
:1008D0000499079DA84700282FD1039A119B94469D
:1008E00063441193069BB618129ADB1BD318C4E716
:1008F000049B2360069BF31A08936360099B5F1EA9
:10090000039BFF18BF191900380001F0D7FCEB69F1
:100910007F1A9F4200D91F00069BAA6A9B1BFF18E3
:10092000974200D91700A76000972800E368089A4B
:100930000499079DA847002882D00BB0F0BDF0B500
:10094000036886688DB08905040006938F0DBE424A
:1009500000D93E0000251368079353680893636825
:100960000993AE4206D8A3680020BB4221D0BB4207
:1009700040411DE0721B0592082A01D90823059306
:10098000059B069902930AAB0193089B08005B192B
:100990000093079BFFF73EFF00280AD1099B059AA9
:1009A00059190AA801F0C4FD002804D0C043C00FA3
:1009B00001300DB0F0BD059BED18D2E7F8B5C76961
:1009C0000D68083F0E000020BD4215D339002800F5
:1009D00001F074FC013801F06BFC0230800039003A
:1009E000281A01F06BFC040001F062FC80002D1A53
:1009F00020006743ED1B3560F8BD0000F7B50C0023
:100A00001500496B002B03D0012B22D18D1826D461
:100A1000436FAB4223D32B008D4218D0876E0091D9
:100A200038006946FFF7CAFF01A9060038000195A2
:100A3000FFF7C4FF2B00864214D1626C01998A42F1
:100A400010D8A06C121891420CD26563E1631800B3
:100A5000FEBD0D00022BDBD1E56A5519D8D5162352
:100A60005B42F4E7226B510307D5D10202D4012186
:100A70004942216402490A4022636563E7E7C046B0
:100A8000FFFFFBFF10B50C00826AFF21E06801F058
:100A9000CFFC01235B42236010BD0000F0B51500C0
:100AA000C26E9FB0139307000E002B68002A08D077
:100AB0009A4203D854235B4205936DE069688A42E9
:100AC000F8D90022042416A91692179201910092D7
:100AD0003900220038000294FFF79CFE031E0590A7
:100AE00001D0543358D10294002417AB01930094E1
:100AF0000422390038006B68FFF78CFE0590A04295
:100B000047D1179B169A9B1ADC17E41AE40FA3002F
:100B10005A59326001225440A20052590D94726019
:100B200016AA9B58B3600023F36002330F93033B74
:100B30000593B74B18AA11CB11C231000120042232
:100B40000831404200F038FE0023119310930993BE
:100B5000013B08930023059D149007930898FFF725
:100B600040FE079BBA6E1B1807930423029315AB34
:100B70000193079B3900009338003368D269FFF76F
:100B800049FE041E0BD02300543300D13DE10594EF
:100B900002E0059B5433BAD005981FB0F0BD042283
:100BA000149815A900F008FE159B089A1BBA5A4024
:100BB0001490069215921ED5089B1D0DF023DB00A4
:100BC0001D40944BED186B425D41EDB2F368069306
:100BD000002B00D028E13368726873600D9B32608F
:100BE0009B0016AA9B58B3600F9B012B00D161E7B5
:100BF00001230F939DE70698FFF7F3FDBB6EDB69BA
:100C00000C93079B0C9AC318934200D9FDE0F02186
:100C1000A0223368C9001293079BD20004330B93C0
:100C2000069B1B0D0B40934237D1042302931CAB50
:100C300001930B9B390000933800129B0C9AFFF72D
:100C4000E9FD041E9FD11C9A149B9A4200D0DCE05F
:100C5000159B069A1B0DDB075A40069214A9042225
:100C6000F86A00F0A9FDF8621598FFF7BAFD079B36
:100C7000C018069BF0603361099BB382189BB36177
:100C8000199BF361109BF37501235B4214932B00B6
:100C9000069A059508921D0060E7031F0E930894BD
:100CA0000E9B089A934229D8159BE024190D080041
:100CB000E4002040214248D1099A1B039B0D9A422F
:100CC00001D8013309931599249B139A4B401A407C
:100CD0000892139A1A420ED133681CAA1C930B9BDC
:100CE00027985360269B9847041E00DA4BE7159916
:100CF000002875D10D002B00059DC9E70E9B089AB1
:100D00009B1A0A93082B01D908230A930C9B089A73
:100D10000B999A1A0A9B380002931CAB0193089B0B
:100D20005B1800933900129BFFF774FD041E00D07E
:100D300029E70A9A14981CA900F03EFD0A9A089B1C
:100D40009446634414900893AAE78024E400A042E8
:100D500019D14AB209993048891889B209912F49A5
:100D6000284001438B4203D180231B061D43AAE781
:100D7000691CA8D01B0329039B0D890D8B42A2D8A7
:100D8000920255199FE7C0243368E400A04211D1B4
:100D90000122114010910821BA6E029118A9019107
:100DA0000B9938000091D2693900FFF733FD041E1A
:100DB00089D0E8E64A051A49520D8A4283D10821B2
:100DC000BA6E02911AA901910B9938000091D2696B
:100DD0003900FFF71FFD543017D00123119372E73C
:100DE0002B00104A4B4013420CD0022883D12A0317
:100DF0000B03920D9B0D9A4200D27CE780252D06B5
:100E00000D4378E701256D4275E70025DEE6C04613
:100E10009025002000FBFFFF00FC0F000000F04FBA
:100E2000FF05000000FCFF7F0023B3759D4232D018
:100E3000BD6E0698A96901F041FA0C1E2BD1119BD9
:100E4000002B28D0EB69099333680A931A9B089307
:100E500001235B420793089BA34216D9089B1D1BE5
:100E6000082D00D90825099B39001A1B1CAB0193DA
:100E7000069B38001B19009302950A9BFFF7CAFCDA
:100E8000002825D0030054334FD1079A1B9B9B1A8F
:100E90005A425341B375E023FC6BDB00220D1A422A
:100EA00028D0380031004030FFF78AFC002821D1DB
:100EB000059B24031B03A40D9B0DA34210D180238B
:100EC000059A1B061A430592259B002B15D121E09C
:100ED0002A0007981CA900F06FFC64190790BAE774
:100EE000059A0132F0D0A34204D9114A059B9446D9
:100EF00063440593259B002B08D0059BB28A1B03F6
:100F00009B0D934200D91300259A1380059B002B5B
:100F100000DB41E60021059BB28A1B039B0D059176
:100F20009A4200D838E60223C5E5059034E6C0466B
:100F300000FCFFFFF0B58BB0C56B0793CB68069242
:100F400005932A0DE02314000E69DB000F000490C6
:100F500009961C401A4219D04030FFF731FC002896
:100F600000D078E0069B1C03A40D0FD0079B2D0337
:100F70001B03AD0D9B0D9D4204D102214942080087
:100F80000BB0F0BD9D42AD41AD0AAC023000FFF7A1
:100F900028FC059A031D9342EFD8059B04991B1A60
:100FA00005930423029309AB0193059B080000936A
:100FB00004223B68FFF72EFC011EE0D1099B069A34
:100FC0001BBA73405B005B0812030993920D1BD0A0
:100FD000E025320D80211000ED00C9002840884234
:100FE00012D10799081B01038C4665463103AD0DEC
:100FF000890D8D4208D31A4908401A4901438E428F
:10100000BBD052B292021419079A0699121B724071
:10101000114222D1B505AB150133AED0129BAD0DF7
:101020009D4200D91D00119B059A0193109B0499C4
:1010300004339B180295009308002A003B68FFF7D1
:10104000E9FB011E9BD1129B5A1B119B581901F001
:10105000EFF9311993E7002498E71E0096E7C046A0
:1010600000FC0F00000010401FB59C05A40D029469
:10107000069C019400240094FFF75CFF04B010BDAF
:10108000F0B593B00A9313680E0006930A9B08907C
:101090000B92002B02D04D4B0A9A1380089B4C4CAC
:1010A0001B6AB361089B5B6AF3614A4F069839007B
:1010B00001F086FA069B39001D18280001F05CFA41
:1010C0000590012806D12B782E2B0DD1059BEB180E
:1010D0000693EAE7059B022B06D11A0028003E4939
:1010E00001F026FA0028F1D0059BEB181F000693AB
:1010F00001230793374B0C93374B0D9338000C9912
:1011000001F05EFA3F1838000C9901F035FA0990A9
:10111000002815D002280DD1022238000D9901F0C7
:1011200007FA002806D1079B013B0793002B04D147
:10113000BB1CCDE7079B01330793099BFF18DDE735
:101140002B78002B3CD00B9B1D6063005B0D022BAA
:1011500039D11E4B2403A40D9C420CD032001F4BEE
:10116000A40218322343009231001D4A0898FFF769
:101170007BFF041E24DB2F21280001F077F9434276
:1011800058410A9B089A404218400FAB0F920393B4
:10119000059A144B119202930092F02332000190B1
:1011A00031000898DB0518321095FFF777FC041E14
:1011B00006DB002800D078E7F37D002BDBD1023C72
:1011C000200013B0F0BD14246442F9E7FF030000CF
:1011D00000FC2F0080250020822500200800002030
:1011E00000FC0F7083070020F0B504000B6A99B073
:1011F000E3664B6B0800A166E360002B03D08B6BAA
:10120000002B02D1E3610C20B2E0E3612100FFF783
:1012100039FC2100A06E1031FFF734FCA16ECB6BBE
:10122000002B01D16366EEE763660B6C002B4FD099
:1012300023674B6C002B00D1784B6367886C0028C8
:1012400000D17748A0670B6DE3675A1C42D1002399
:10125000E3670127002520007F4229000C22A562B8
:10126000E562276267623C3001F0E2F82000290065
:101270000C22303001F0DCF8200029000C2248302C
:1012800001F0D6F829001C2210A801F0D1F80123A2
:101290001D00179305970493169B5A1C03D0179AA9
:1012A000511C00D0B1E0226BD30F9B1823632200A6
:1012B000230030323C3323CA23C3E56EE06A2900A1
:1012C00000F0FCFF00206165A065E06525668FE009
:1012D000FF23ADE7002BBCD1CA6C8B6A002A07D074
:1012E000D208834200D903009342B1D91300AFE77B
:1012F000CA69F5E79F4203D10599914200D18BE07D
:1013000004998D4204D169001700002504910593CA
:1013100007AB0393434B444A0293002308920822ED
:101320000193424B10AE0992009331002000404BD4
:1013300016AA01350794FFF7B1FB002858DB4AD005
:1013400080058015013046D0109B31002362119B2F
:10135000200063620AAB0093354A364BFFF784FEE8
:10136000002845DB0A9B99B21B0C022B02D01620E9
:1013700040423DE00129FAD8236B2F4A1340012255
:101380004A405202134323630D9B002B03D0226F6C
:101390009342ECD823670E9B0AAA002B03D0616FFF
:1013A0008B42E4D863675369002B08D0A16F8B424E
:1013B000DDD8E16FA367994200D91900E167A36EF8
:1013C0009168186A002801D08842D0D15268DB6940
:1013D000E1669A42CBD10AAE2000184B184A00961B
:1013E00010A9FFF741FE002804DA831C00D153E75F
:1013F00019B0F0BD2300210030333C311A6801CE12
:10140000424004C38B42F9D146E70599994200D086
:1014100070E7974200D073E75420A9E7FFFFFF7FF2
:10142000FE03000083070020852500200800F00F40
:1014300000FCFF7F18001020FFFDFFFF0C00F07F75
:101440000000F07FF0B587B00B6300234B63CB63E4
:10145000CB640B00059208330C9A02930A650B1DAE
:101460000C0005AA02990600FFF70AFE051E08DA1D
:10147000831C21D1414BA2889A4202D102256D42A0
:101480001AE00123A371B36A2360B462AB1CF5D0E8
:101490002B0D03931525012BF1D1A288384B920215
:1014A00013432200283200923000364A0299FFF797
:1014B000DBFD0027051E09DA21003000FFF79CF94B
:1014C00016E0226B03990A4215D10137236D9A6801
:1014D0009742F6D31B68E364002B27D02100B06E3F
:1014E0004031FFF7CFFA284A2B0D934220D0002538
:1014F000280007B0F0BD0C21C02079435A68A388AA
:10150000521891689B020B431178800052680918A9
:1015100009050B43009230001C4A0299FFF7A4FD15
:101520000028D2DA831CD0D00500C5E70C25A6E739
:101530008023216B5B030B4323630023022263643C
:10154000B36EAD059B6A5242AD0DA262E5622264A4
:10155000A364CCD0A2880E4992028B4200D90B0022
:101560001A4380239B051343E26C300000920299DA
:10157000044AFFF779FD051EB9DA9DE7FF03000075
:101580000800002000FC0F700102000000FCFF7F3B
:10159000FE030000F0B597B00C000A924A6BC96ACE
:1015A000070000208A4200D3E2E08A1A08929A4299
:1015B00000D90893089B0693069B002B01D108983D
:1015C000D6E08022236BD202134204D0BA6EE66BBF
:1015D000D269964213D180214903626B0B4277D1C5
:1015E000A36AE66A13931492002E39D101235B4259
:1015F000A363E6638022236BD20213432363BA6E94
:101600000699D2690992921B05928A4200D90591E6
:1016100080225203134200D1ACE023000833109320
:10162000A3885E4A9B021A43059B1192099A9B1953
:101630009A4200D2AEE00A9B0B93059B0793079B4F
:10164000002B4BD1059A636B94469B186363E36B45
:101650009B18E3630A9B63440A93069B9B1AAAE7C1
:101660002300BD6E4033013E15A92800099315964D
:10167000FFF7A4F914A906002800FFF79FF90590C9
:10168000139B0793059BB34203D3079B149EA3634D
:10169000AFE7059BF01A00F0FFFD0500300000F0F9
:1016A00001FE1F235D1B854200D905000423029320
:1016B00013AB0193AB00009304223800079B0999F8
:1016C000FFF7A8F8002853D10123AB40F61AD7E75B
:1016D00002235B421600A363E2638BE7E36C0F9384
:1016E000236C023319D1616CA56C4D19AE4214D232
:1016F0008E4212D3079BAD1B9D4200D91D000F9B4C
:10170000711A59182A000B9800F098FE0B9B761955
:101710005B190B93079B5B1B90E702235B422364DF
:10172000BB6E30000D935B6919000C9300F0C6FD91
:10173000731A0C9A0E936364099B11009D18013D66
:10174000AD19280000F0BAFD0D9B6D1A9B6A9D42F1
:1017500000D91D000F9BA56401930E9B38000093D8
:101760000F4A119B10990295FFF7E4FB0028B5DAA8
:1017700017B0F0BD2100059B009602930A9B38002C
:101780000193A36B099A4031FFF744F8002800D178
:1017900058E7EDE754204042EAE7C0460000102039
:1017A00000FCF7FF002310B51A00FFF727F9002807
:1017B00000DD002010BD000070B50F250A4C8A180E
:1017C000914200D170BD0B78060958402840800036
:1017D00000591B09464073402B409B001B593009A0
:1017E00058400131ECE7C04698250020F0B50D00C7
:1017F00016000021202289B0040000F019FE2B0001
:10180000701998420ED1002369461A002380E05ACD
:101810005A5202331218202BF9D10022B24208D1B9
:1018200009B0F0BD1A7801335200A15A0131A1521A
:10183000E7E7A85C002806D040000B5A5F1C103375
:101840005B000F521A530132E8E70368426810B593
:10185000934203D25A1C0260187810BD8368841D1D
:10186000002B07D0E27F002A04D19847002801DB33
:10187000C0B2F2E701230020E377EEE7036910B579
:101880005A1E04000261002B04D1FFF7DEFF07237C
:10189000E0602361E0684308E3600123184010BD65
:1018A000F7B5002615000190B14204D001242700AD
:1018B0008F40BC4201D3A819FEBD0198FFF7DEFF9F
:1018C000604364003618F4E7F7B500250B000E00FE
:1018D0002C00203301908F1C00930198FFF7CEFF5E
:1018E000009B6D0028189F420BD03D8802372B19B2
:1018F000451B04D5241810346400A05BFEBD1C00F9
:10190000EBE703204042F9E7F0B5D5B0039202229D
:101910000091FF3205210500FFF7C2FF01220521DA
:1019200006002800FFF7BCFF0422019011002800E8
:10193000FFF7B6FF13220700002104A800F078FD8E
:101940000024BC4218D100241322009804A9FFF7F8
:101950004DFF019BF3180293029B9C4217D3320068
:10196000009804A9FFF742FF04AB0398019AF1180D
:10197000FFF73CFF002012E0002203212800FFF7C0
:101980008FFF1D4B04AA1B5D0134D054D9E72800FA
:101990000099FFF799FF002803DA0320404255B071
:1019A000F0BD112820D0122822D0102818D1002CE8
:1019B000F3D02300413304AAFF339B1802210322F2
:1019C000423BFF3B1F782800FFF76AFF029B20186D
:1019D0009842E2D804ABA042BED0E7540134FAE703
:1019E00004AB18550134B7E7032211000027EAE7DA
:1019F0000B220721FAE7C046D825002070470023B4
:101A000010B5841DE377012464420361C3628462DC
:101A1000C26381630364036310BD0000F8B5040072
:101A2000A36A013375D12000A56AFFF727FF0022C2
:101A3000E06202212000FFF733FFA062012800D0FE
:101A400081E0012D6BD0210000230831A21DD38736
:101A500002318B87CB870231CB870231CB87403174
:101A60000B804B802300182152331980803159801C
:101A70002839998021008023183064315B00FF30C1
:101A80000B8001339BB202318342F9D12000002345
:101A90009430590043520133902BFAD1D7218C2036
:101AA0004900400050521A200231FF30505202319A
:101AB000013050521C200231FF30505202310130AF
:101AC00050521E200231FF3050520231013050522C
:101AD00020200231FF3050522200C532FF32BC3983
:101AE000138001339BB202328B42F9D1A922002329
:101AF00020219200A352A218518153809380D38059
:101B00001381B1229200A1185A008B520133202B6D
:101B1000FAD1A66A002E25D0013E012E1FD8236BD4
:101B2000002B00D083E0210020004431FFF7CCFEE1
:101B3000A31DDB7F002B12D1FF284DDCA369C0B2AF
:101B40005A1CA26133E00228E3D1A92321009B00A3
:101B50002000E2184431FFF7D7FE0028D9D0032037
:101B600040429FE0206B002817D12000FFF76DFE58
:101B700005002000FFF769FE000245192000FFF76D
:101B800064FE07002000FFF760FE484B0002C0190A
:101B900043409D42E3D1681C266101382063002840
:101BA0007BD02000FFF751FEA3695A1CA261187078
:101BB000A26B002A09D0236C591C2164D054226CDA
:101BC000E36B9A4201D100232364A269E3699A423C
:101BD00000D225E7002065E080235B0098425CD0BE
:101BE0000238FF381C28BADC314B4200D25A314B44
:101BF000195C2000FFF754FEA9239B002063E11825
:101C00002000FFF761FE1D28A9DC2B4B4200D25AB1
:101C10002A4B195C2000FFF743FEA36B002B2DD04D
:101C2000E26B90423FD8236C1B1A24D46363A16BF0
:101C3000A369626B00292AD0581CA0618A5C1A70C3
:101C4000A36B002B0BD0226C616B501C2064595C81
:101C50009954226CE36B9A4201D100232364636B95
:101C6000E26B01336363934201D100236363236B0F
:101C7000013B2363A9E7D2186263D8E7A3696269CD
:101C80009B1A984200D96AE740426063CFE79A5CAA
:101C90001A70A3690133A361E9E7E36A002B00D15D
:101CA000C1E60120F8BD05205AE7C046FFFF00004D
:101CB0004626002082260020EC2500202826002031
:101CC00070B505000C00002C00D170BD2800FFF796
:101CD000BCFD013CF7E770B50400FFF7B6FD050059
:101CE0002000FFF7B2FD0002284380B270BD70B53E
:101CF0000400FFF7AAFD1F2802D00320404270BD58
:101D00002000FFF7A2FD8B28F7D12000FFF79DFDF3
:101D10000828F2D12000FFF798FD05001F28ECD815
:101D200006212000FFF7CCFF6B0706D52000FFF748
:101D3000D2FF01002000FFF7C3FF2B0704D52000CE
:101D4000FFF783FD0028FAD1EB0604D52000FFF74A
:101D50007CFD0028FAD10226354202D02000FFF790
:101D6000BAFF631DDE7701235B4200202362C6E7D2
:101D7000054B064A1360064A136053609360D360B4
:101D800013615361936170478080808000E400E0BC
:101D900004E400E0044A1078431CDBB2172B00D99E
:101DA000102313707047C046C02600200021044B4A
:101DB000044ABFF35F8F02C39342FAD17047C04613
:101DC000000100D0800100D0024BC91889000160D9
:101DD0007047C0464000003410B50400FFF7DAFF3A
:101DE00001002000FFF7F0FFFF232371BFF35F8F97
:101DF00010BD10B50400FFF7CDFF01002000FFF774
:101E0000E3FFFF23A380BFF35F8F10BD10B5084829
:101E1000084B984200D310BD040003680834002B1F
:101E200003D0FFF7E6FF2000F2E7FFF7D5FFFAE760
:101E3000F0260020F8260020142310B50100188891
:101E400004331B88984710BD162310B5010018886D
:101E500002331B88984710BDF8B50E000400002718
:101E60000125B74201D12800F8BD2068FFF7E4FF43
:101E700001C4431E984101370540F2E7F7B50C2431
:101E800044430193254B0092E4186368089A0500C7
:101E90000E00934200D26260C0232F1F9B01FFB24D
:101EA000E318012F29D8012E27D103221A60A36835
:101EB0003342FCD0009B22685B015340E022134078
:101EC00080225201A2181360012F09D80321236830
:101ED00073400B4013600123B340A2681342FCD04F
:101EE000802380229B01E31812011A60089B019A4B
:101EF00063600B4BAD00EA50F7BD802212011A60FF
:101F0000074BAA00D1580029D4D0586900F0D6F95F
:101F1000431C032058430338FDD2CBE70080004028
:101F20008C290020F7B505000E001800089917004D
:101F300000F0C4F9089A0300140231003A002800A6
:101F40000094FFF79BFFF7BD13B580246400009455
:101F5000FFF794FF13BD0000014B8000C05870478D
:101F60008C290020F8B504001F4817001E000D0042
:101F700000F0A4F90100380000F0A0F9069A33043B
:101F8000120313432268002A0FDA3F2122680A4015
:101F9000AA420AD1A2681205120D824205D1EE2191
:101FA000E268C9020A409A421CD0104A104EA11899
:101FB0004A42514101220C318A400E490A600E49C1
:101FC0000A60170031688F43391EFAD10B4A21315C
:101FD000A2182560A060116021680029FCDAE36086
:101FE00008231360F8BDC046001BB7000040FDBFCA
:101FF00008C0004000E0004000F000400430000055
:10200000024B1A68024B5A607047C046B429002040
:102010000080054003008020114AC00510B5114C16
:10202000106011480460E020104CC004002906D064
:102030002060002B05D180231B06236010BD10609B
:10204000F7E7FA20C00058438023094A5B0498420E
:1020500000D308481060FFF7D3FF8023DB05ECE7CF
:1020600000B00540FCFF01000820014000A0054031
:10207000B4290020FFFFFF0070B50400100080228B
:102080000A4BD2051A600A4B002C0CD00125094AD4
:102090002C43DA61084A62401A6259629C6200214C
:1020A000FFF7B8FF70BDDC61F9E7C04600B005403E
:1020B00000800540D3C007B02D3FF84F8023024A6F
:1020C0009B000B43D362704700800540AA22064B59
:1020D00012011A602132FF32DA600449044A1160A9
:1020E0005A68002AFCDA70470040024000B0FA004B
:1020F000006002407047000010B5044C044B9C4245
:1021000000D310BD08CC9847F8E7C046F826002059
:1021100034270020054B064A06491A60064B074A39
:10212000136018000A689043FBD1704700E000403C
:10213000BFCDFBFE08C00040FE7F3C0000F0004029
:10214000044BDB6C002B03D18022034BD2021A60BC
:102150007047C046000011504C201150044A054BF6
:102160001A60054A1368DB018033FBD17047C04613
:10217000FFFFFF0100F0004008C000404022034B79
:102180009A675A671A67DA667047C04600F00140DE
:1021900010B5FFF70BFE10BD70B5044D044CA968D7
:1021A000C022200000F04AF9AC6070BD00ED00E0F4
:1021B00000000020002373B5284DAB67FFF786FFB2
:1021C0000122274B1A606B6C012BFCD10322254B9B
:1021D0001A60AC6B012CFCD102260525210000966B
:1021E0000623214A2148FFF7BDFE2B002100009560
:1021F0001F4A2048FFF7B6FE3100002204201E4B84
:10220000FFF7A2FE2800210000221C4BFFF79CFED6
:102210000022072011001A4BFFF796FE002208202B
:102220001100174BFFF790FE80230022DB00110006
:1022300000930920124BFFF775FE00220F4B11008F
:102240000620FFF781FE0420FFF786FE0D4900F00F
:1022500035F801000020FFF731FF73BD008000401A
:102260003CB0004030B00040002F68590080024070
:10227000008C864700C00240001BB700405973071E
:10228000006CDC0240420F0001480421014B18475A
:10229000D02600209D1C0020014B5B6818470000E1
:1022A000D0260020014B9B6818470000D026002054
:1022B000014B1B6818470000D0260020114A936F7D
:1022C0009B0813D210665166002905D0FFE7FFE78F
:1022D000FFE7516F106F704704B5002801D0002050
:1022E000C04300F0C1F8002104BDC046F0B5146E33
:1022F000556E576F166FFFF7E5FF14665566576703
:102300001667F0BD000000D0132370B51C78114D86
:10231000012C0ED1002310499A000133A950202B23
:10232000FAD10D4BAB640D48FFF786FD0C4B1860DE
:1023300070BD012CF5DD0B48FFF786FD06000A484D
:10234000FFF782FD80223100280000F077F8022C90
:10235000E9D1E6E7B8290020B12100204C33000084
:10236000B82A0020534400005346000007B56046D9
:1023700001880A0A0230DF2AFAD1C9B2820804D3DE
:10238000028840880004104300E00068014A505071
:10239000039007BDB8290020132310B510481C78FE
:1023A000FFF752FD0100012C13D10E4C54222000E6
:1023B00000F044F815230C4A990001336250202B99
:1023C000FAD12262E2610948FFF736FD084B186036
:1023D00010BD012CF7DD8022024800F02FF8F2E753
:1023E00053460000BC2A0020392200204C33000054
:1023F000B82A002007B5604601880A0A0230DF2AA1
:10240000FAD1C9B2820804D302884088000410437C
:1024100000E00068014A5050039007BDBC2A00202C
:1024200001480421014B1847E02600209D1C002094
:10243000014B1B6818470000E0260020014B5B6839
:1024400018470000E026002010B5FFF755FE044CA9
:10245000044B9C4200D310BD08CC9847F8E7C04617
:1024600034270020382700207047C0460323CAB213
:10247000F0B50340002A35D00324002B2DD1FF23D3
:102480000B401D02ED182B04ED182C000168264EA0
:102490004C408B198B43A119A143244E0B4333426B
:1024A00011D14168204F0C00CB196C408B43E119CE
:1024B000A1430B4304303342F3D00378002B05D003
:1024C0009A4204D001300378002BF9D10020F0BDEE
:1024D0009342FCD001302042D1D00378002BF7D1B9
:1024E0000020F4E7002B08D0032202E00130104264
:1024F00003D00378002BF9D1E9E702680A4B0B49B6
:10250000D31893430B4206D14268074B0430D318CB
:1025100093430B42F8D00378002BD8D04378013096
:10252000002BFBD1D3E7C046FFFEFEFE80808080FB
:1025300030B5032A0CD90B0003439B0719D104685B
:102540000B689C4215D1043A04300431032AF6D8B2
:10255000551E002A0BD0002303E05A1C9D4206D0D2
:102560001300C25CCC5CA242F7D0101B00E000203C
:1025700030BD551EEFE7C04670B50478002C1CD066
:102580000E780500002E0AD00A00330003E05378CD
:102590000132002B0CD09C42F9D1281A70BD6C7806
:1025A0000135002CF9D06C780135002CF7D1F4E717
:1025B0006C780135002CE7D1EFE70020EEE7C0464C
:1025C00070B504780600002C14D00D780020002D82
:1025D00000D170BD30000A002B0003E053780132B7
:1025E000002B05D09C42F9D144780130002CF2D167
:1025F000801BEEE70020ECE7F8B5C046084A10B5AE
:102600001378002B0AD18023064807495B051C6814
:10261000C45004338B42FAD10123137010BDC0465D
:10262000BD2B00208C2800100001001010B5014BBC
:10263000984710BD8D2800208023F0B54218070070
:102640000C0085B05B049A4201D9FDF744FF1426C3
:10265000182530882B88124998472B8803901149F8
:10266000308898472B8802900F49308898472B88EC
:102670000E490190308898470500FFF7BFFF039B84
:102680009847029B984780222100D82338005202A5
:10269000019CA047A847FFF7C9FF05B0F0BDC046A1
:1026A00049460000455800005245000046430000DE
:1026B0008023F0B5170085B08218040003915B04F5
:1026C0009A4201D9FDF707FF1426182530882B8878
:1026D000104998472B8802900F49308898472B88DB
:1026E00001900E49308898472B880D49009030881A
:1026F00098470500FFF782FF029B9847019B984788
:102700003A0020000399009B9847A847FFF78EFFE7
:1027100005B0F0BD49460000455800005250000089
:10272000464300005069636F204F5441006F74614D
:10273000636F6D6D616E642E62696E002F002E2EC8
:10274000006C6974746C656673000000FFFFFFFF26
:10275000FFFFFFFF000000006410B71DC8206E3BA4
:10276000AC30D9269041DC76F4516B6B5861B24D98
:102770003C7105502083B8ED44930FF0E8A3D6D602
:102780008CB361CBB0C2649BD4D2D38678E20AA06A
:102790001CF2BDBD10111200080709060A050B0442
:1027A0000C030D020E010F000100020003000400E3
:1027B0000500070009000D0011001900210031007B
:1027C000410061008100C10001018101010201039A
:1027D000010401060108010C01100118012001305B
:1027E0000140016000000000010102020303040433
:1027F000050506060707080809090A0A0B0B0C0C51
:102800000D0D030004000500060007000800090084
:102810000A000B000D000F001100130017001B0031
:102820001F0023002B0033003B00430053006300D4
:1028300073008300A300C300E30002010000000056
:102840000000000000000101010102020202030376
:10285000030304040404050505050000F42F00101B
:10286000F02F0010005003200000000000000000C6
:1028700000510320000000000000000010000000D4
:1028800000000000000000000000000050330000C5
:102890004C33000054330000523300004D5300000D
:1028A0004D4300005334000043340000000000009A
:1028B000000000006522002085010020591F002033
:1028C000851F0020CD2000204D210020DD2100208B
:1028D000F91F0020A11F0020C11F0020D51F0020CC
:1028E000511C0020DD1F0020391F0020B51B0020D7
:0428F000390100208A
:1028F40000000000000000000000000000000000D4
:1029040000000000000000000000000000000000C3
:1029140000000000000000000000000000000000B3
:1029240000000000000000000000000000000000A3
:102FE40000000000000000000000000000F0F710E6
:0C2FF40000F0FF1000F0FF1000F0F700EC
:1030000000200420E3300010C3300010C530001051
:10301000C1300010C1300010C1300010C1300010AC
:10302000C1300010C1300010C1300010C730001096
:10303000C1300010C1300010C9300010CB3000107A
:10304000CD300010CD300010CD300010CD3000104C
:10305000CD300010CD300010CD300010CD3000103C
:10306000CD300010CD300010CD300010CD3000102C
:10307000CD300010CD300010CD300010CD3000101C
:10308000CD300010CD300010CD300010CD3000100C
:10309000CD300010CD300010CD300010CD300010FC
:1030A000CD300010CD300010CD300010CD300010EC
:1030B000CD300010CD300010CD300010CD300010DC
:1030C00000BE00BE00BE00BE00BE00BEEFF3058025
:1030D000103800BE1E481F49086006C881F30888E2
:1030E00010471D480068002801D01948F3E70DA4D7
:1030F0000ECC002902D000F012F8F9E71749184A5F
:10310000002000E001C19142FCD1164988471649D0
:1031100088471649884700BEFDE701C901C29A42A7
:10312000FBD37047C0540310C00000206866002025
:1031300068BA0310000004200000042068BA0310DD
:103140000010042000100420000000007047000060
:103150000000000008ED00E0000000D068660020DC
:103160006CC3012071EE0210CD07021039BF0210AE
:10317000F8B5C0460448054B10B5834203D0044B54
:10318000002B00D0984710BD6866002068660020BC
:103190000000000006480749091A8B10C90FC9181A
:1031A00010B5491003D0044B002B00D0984710BD38
:1031B00068660020686600200000000010B5074C1B
:1031C0002378002B09D1FFF7D5FF054B002B02D048
:1031D000044800E000BF0123237010BD388900209F
:1031E00000000000D8F00210054B10B5002B03D0F2
:1031F0000449054800E000BFFFF7CCFF10BDC04602
:10320000000000003C890020D8F002100020704728
:10321000704700207047002070477047034B10B57F
:10322000186803681B68984710BDC0466C090020E9
:10323000034B10B5186803685B68984710BDC0461B
:103240006C090020034B10B518680368DB689847C9
:1032500010BDC0466C09002000200B5C002B02D082
:1032600001308242F9D270470023C2684361137073
:103270007047000070B51F4C050020680E00002844
:1032800036D01D49002E03D01CF0DAFE1B49206801
:103290001CF0BAFEEB69002B07D0202120681CF03F
:1032A000C2FEE96920681CF0BAFE154920681CF0CE
:1032B000ABFE0A22296920681CF05BFF11492068D7
:1032C0001CF0A2FE0A22696920681CF052FF002E41
:1032D0000BD00D4920681CF097FEE96820681CF0AF
:1032E0009EFE272120681CF09EFE20681CF0A8FE90
:1032F00070BDC046B0900020E4F00210CD05031070
:10330000D8F00210DEF0021094F6021070B5057EBF
:103310000400002D1FD00269C3689B18002A1BD02F
:103320001A78002A18D001210C4A41761170002227
:103330001A70E06827F0D8FE6061002D0BD0084BB2
:103340001868002807D007491CF05EFE064B2000D5
:103350001978FFF78FFF70BD1500E8E76383012040
:10336000B0900020EAF002106809002010B50400B7
:10337000FFF7CCFF606910BD70B50400FFF7C6FF12
:1033800020006569FFF7C2FF2069401B4342584196
:10339000C0B270BD70B50400FFF7B8FF200025690A
:1033A000FFF7B4FF6069281A70BD000008B4024B33
:1033B0009C46043808BC60479533001070B50D007A
:1033C0000400FFF7A3FF2800E1681CF028FE70BD91
:1033D00010B50400FFF79AFF0123E068237610BDC3
:1033E00010B50400FFF792FFE4682078002800D1B0
:1033F00010BD22F025FC20700134F6E7F8B5050079
:10340000FFF784FF6C69002C1AD0EF683E0030781B
:1034100025F0A4F8002814D1013C3C19207825F0AF
:103420009DF800280FD10134A21B6A61BE4203D966
:103430003100380028F090FD0021EA686B69D15412
:10344000F8BD0136E3E7A642EDD8013CE6E7F7B563
:1034500005000E00FFF75AFF6B69002B01D1002019
:10346000FEBD0A22E86801A927F010FE019CEB6866
:103470000700A342F3D02078002802D13760013042
:10348000EEE725F06BF801340028E8D00194F2E76C
:1034900070B5094D04002868002808D020211CF0D0
:1034A000C2FDE1692868002902D01CF0B8FD70BD9A
:1034B00002491CF0A9FDFAE7B090002097F702102E
:1034C000F0B585B001930AAB040001CB15001A7862
:1034D0000CAB1B78AC4F039300232760AB4FE0612C
:1034E000601DA360676063762362A36223616361EA
:1034F0002276C3779D4200D13DE10198431E984159
:10350000019BEB1A5F427B4103400293002A24D0C7
:10351000039B002B21D104291DD100229C4B9D4DE2
:103520001A70E36028689C4B013221611A70627640
:10353000002800D1A9E099491CF066FD2000FFF7A2
:10354000A7FF974928681CF05FFD964B200019786B
:10355000FFF790FE99E0002D54D04B1EE560033339
:103560004AD9002A34D0039B002B31D0002913D133
:103570000122874B874D1970E3602868864B62767D
:103580001A70002800D180E087491CF03DFD200022
:10359000FFF77EFF8549D5E7280027F0A5FD060047
:1035A000029B2661002B00D12B70019B002B3DD18B
:1035B0000122784D784B28681A706276002864D012
:1035C0007B491CF021FD2000FFF762FF7949B9E734
:1035D00000226F4B6F4D1A70E36028686E4B01320A
:1035E0001A706276002850D073491CF00DFD20003F
:1035F000FFF74EFF7149A5E7714B994200D91900B9
:103600004E1ECDE70022624B624D1A70E3602868BF
:10361000614B01321A706276002836D064491CF082
:10362000F3FC2000FFF734FF66498BE7701CFF3086
:103630001DF08CF907001DF0B1F9002F28D10122EF
:10364000554B62761A702F70524D2868002818D09A
:1036500057491CF0D9FC2000FFF71AFF5A49286887
:103660001CF0D2FC0A22216928681CF082FD57490F
:1036700028681CF0C9FC4B4B200019782761FFF724
:10368000F9FD434BE36000232361200005B0F0BD4A
:10369000320020000199FFF7DFFD029B0700864200
:1036A0005BD2002B02D000236661AB550122394D5D
:1036B000394B28681A7062760028E6D0394B1E0014
:1036C000029B002B2AD13A491CF09EFC2000FFF7F8
:1036D000DFFE3F4928681CF097FC0A223900286861
:1036E0001CF047FD3B4928681CF08EFC3378002B0A
:1036F00012D028681CF0A4FC374928681CF084FC10
:10370000364928681CF080FC019928681CF087FC69
:10371000272128681CF087FC330017E7039B3049FA
:10372000002B00D124491CF06FFC2000FFF7B0FEF5
:103730002C4928681CF068FC0A22390028681CF013
:1037400018FD3378002BE7D028681CF079FC22495B
:1037500028681CF059FC2449D3E7002B04D102004F
:103760000199280028F0F8FB0022E3682169DA5566
:1037700067615A5489E7002A00D143E7039B002B75
:1037800000D03FE70293C6E60C290310242903105A
:1037900064830120B09000206383012027F1021090
:1037A00054F102106809002068F2021096F202102B
:1037B0000EF3021055F30210C6F20210ECF20210E2
:1037C000FEFFFF7F21F3021089F302109EF3021027
:1037D000DDF3021075F30210CD050310F7F30210AC
:1037E00010F402103CF402106BF4021070B50400E7
:1037F0000E00FFF78BFD6369B3422DD80122184DEF
:10380000184B28681A706276002823D016491CF0DD
:10381000FBFB2000FFF73CFE144928681CF0F4FB7A
:103820000A22310028681CF0A4FC114928681CF009
:10383000EBFB2000FFF72CFE0E4928681CF0E4FB90
:1038400061690A2228681CF094FC0B4B200019784F
:10385000FFF710FD002070BDE368985DFBE7C046F0
:10386000B09000206383012087F402108FF40210CF
:10387000A0F40210A5F402106809002070B504003D
:103880000E00FFF743FD6369B3422DD80122184DA6
:10389000184B28681A706276002823D016491CF04D
:1038A000B3FB2000FFF7F4FD144928681CF0ACFBC3
:1038B0000A22310028681CF05CFC114928681CF0C1
:1038C000A3FB2000FFF7E4FD0E4928681CF09CFBD9
:1038D00061690A2228681CF04CFC0B4B2000197807
:1038E000FFF7C8FC002070BDE368985DFBE7C046A9
:1038F000B09000206383012087F4021013F50210BA
:10390000A0F40210A5F4021068090020F0B585B0FB
:103910001E002C4C0AAB1B780190206802930BAB65
:1039200017001D780391002822D027491CF06CFB5A
:103930000198FFF7ADFD254920681CF065FB206864
:10394000002F17D1002E26D1029B002B2FD12068EB
:103950001CF076FB1E4920681CF056FB03990A22D6
:1039600020681CF006FC1B4B01981978FFF782FCBD
:1039700005B0F0BD002D02D122211CF054FB114EE8
:10398000390030681CF04BFB002DE0D1222130685B
:103990001CF049FBDBE710491CF036FB31002068C6
:1039A0001CF032FB0D4920681CF039FBCFE72721C2
:1039B0001CF039FB029920681CF035FB2721206898
:1039C000E6E7C046B090002019F80210DB070310AC
:1039D000E3F30210680900201DF5021021F5021022
:1039E00070B50D4C060020680D00002813D00B495F
:1039F0001CF00AFB3000FFF74BFD2E2120681CF065
:103A000012FB002D03D0290020681CF0FDFA0449A8
:103A100020681CF0F9FA70BDB090002019F802106F
:103A2000471B031070B50D000400FFF76FFC002D5D
:103A300017D10122164B174D1A702B686276002B96
:103A400001D1002070BD20001349FFF7C9FF1349C1
:103A500028681CF0D9FA124B20001978FFF70AFCED
:103A6000EFE7280027F040FB63698342E9D3002891
:103A700003D15A425341D8B2E4E71B1AE068290047
:103A8000C01822F0E3F943425841C0B2DAE7C04619
:103A900063830120B090002064F502102EF502101F
:103AA00068090020F8B504000D001600FFF72EFC91
:103AB00063696A1C00D178E09D422BD901223C4BFE
:103AC0003C4F1A703B686276002B21D020003A49A7
:103AD000FFF786FF394938681CF096FA0A22290058
:103AE00038681CF046FB364938681CF08DFA200017
:103AF000FFF7CEFC334938681CF086FA61690A2268
:103B000038681CF036FB304B20001978FFF7B2FB09
:103B100065692B005B1BB34234D20122244B254F35
:103B20001A703B686276002B2AD020002249FFF7EA
:103B300057FF264938681CF067FA0A2231003868B6
:103B40001CF017FB1E4938681CF05EFA2000FFF7D6
:103B50009FFC1C4938681CF057FA0A2261693868D2
:103B60001CF007FB1A4938681CF04EFA29000A229B
:103B700038681CF0FEFA144B20001978FFF77AFB26
:103B80006669761B002E0FD06269E0680132521B15
:103B9000A9194118921B401928F0DEF90021636928
:103BA000E2689B1B6361D154F8BD1D00B2E7C046BB
:103BB00063830120B09000209EF50210FAF40210F9
:103BC00060F50210A5F4021068090020A5F50210A6
:103BD000ADF5021070B504000D004B1C2ED0FFF7A0
:103BE00095FB63699D422AD901221A4B1A4E1A701D
:103BF00033686276002B21D020001849FFF7F0FED1
:103C0000174930681CF000FA0A22290030681CF0BD
:103C1000B0FA144930681CF0F7F92000FFF738FCBF
:103C2000114930681CF0F0F961690A2230681CF013
:103C3000A0FA0E4B20001978FFF71CFB70BD200086
:103C4000FFF764FB626929002000521BFFF72AFF7F
:103C5000F4E7C04663830120B09000209EF5021077
:103C6000FAF4021060F50210A5F4021068090020B1
:103C7000F7B51E0008AB170004CB3D4C1B780500C0
:103C8000019323680092002B31D0FFF7A9FE394938
:103C900020681CF0B9F90A22390020681CF069FA82
:103CA0002B7E002B0CD0344920681CF0ADF9791C18
:103CB0000A2220681CF05DFA304920681CF0A4F943
:103CC0000A9B002B0CD02E4920681CF09DF90A9904
:103CD0000A2220681CF04DFA2A4920681CF094F949
:103CE000294F3978002903D12800FFF7C3FAF7BD1F
:103CF0001F4C20681CF0A4F9244920681CF084F9AA
:103D0000002E05D1009B002B02D1019B002B21D05E
:103D10001F4920681CF078F9002E0CD0272120685C
:103D20001CF081F9310020681CF079F92721206806
:103D30001CF079F90EE0009B002B0DD0154920688E
:103D40001CF062F9009920681CF05EF912492068A5
:103D50001CF065F93978C7E7019B002BFAD02721C1
:103D600020681CF060F9019920681CF05CF9DDE71F
:103D7000B0900020E3F30210B7F50210C3F5021073
:103D8000C6F50210D6F5021068090020CD05031013
:103D9000EBF502101DF5021021F5021070B50D4C67
:103DA000060020680D00002813D00B491CF02CF9E8
:103DB0003000FFF76DFB2E2120681CF034F9002D38
:103DC00003D0290020681CF01FF9044920681CF06A
:103DD0001BF970BDB090002022F60210471B0310A3
:103DE000F7B506001700080001930C00FFF78EFAE4
:103DF0003000FFF78BFA019B75693B432B4304D1DD
:103E0000E268636113702000FEBD7B1C00D12F00AF
:103E1000019B013300D0019DAF420CD90123414ADF
:103E2000737613706376404B01931B68002B2DD182
:103E30003B002F001D007369AB4221D20123394A98
:103E4000394D7376137063762B68002B13D03000D6
:103E50003649FFF7A3FF364928681CF0D5F8300033
:103E6000FFF716FB334928681CF0CEF8324B3000C0
:103E70001978FFF7FFF97569AF4200D92F002B00C1
:103E80009F4201D0AF4218D10023B9E73000274943
:103E9000FFF784FF019B264918681CF0B5F8300035
:103EA000FFF7F6FA019B254918681CF0ADF8224B84
:103EB00030001978FFF7DEF9BAE72000FFF726FA9D
:103EC0002369ED1B9D4222D90123164A164F7376B2
:103ED000137063763B68002BD6D030001349FFF790
:103EE0007FFD174938681CF08FF82000FFF7D0FAE3
:103EF000144938681CF088F829000A2238681CF038
:103F000038F90D4B20001978FFF7B4F9BCE7F168D8
:103F10002A00E068C91928F01FF80022E3686561EB
:103F20005A5570E763830120B09000202BF60210F1
:103F300096F7021049F602106809002035F60210C3
:103F40005DF60210E3F30210F0B587B01F000CAB72
:103F50001B780C0000930DAB1B78160003930EAB7F
:103F60001B7805000293FFF7D1F90022E36800995E
:103F700062611A7005AB19705A70974200D11F0028
:103F8000731C2FD06B690093B3422BD02ED2012328
:103F90004B4A6B7663764B4C13702368002B21D011
:103FA00028004949FFF71CFD484920681CF02CF8FF
:103FB0000A22310020681CF0DCF8454920681CF01A
:103FC00023F82800FFF764FA424920681CF01CF827
:103FD00069690A2220681CF0CCF83F4B2800197848
:103FE000FFF748F90120404207B0F0BDEB68390007
:103FF00001939819029B002B54D024F027FB039BBC
:10400000002B04D0002802D00120002EECD0009B11
:104010008619B342E6D0019B39009819029B002B08
:1040200043D024F0EFFA0090009B009A9B19019373
:10403000236993423CD20123214A224F6B761370AD
:1040400063763B68002B27D028001F49FFF7C8FC88
:10405000224938681BF0D8FF2000FFF719FA2049E1
:1040600038681BF0D1FF0A22009938681CF081F8EB
:104070001C4938681BF0C8FF3868E9680368009A73
:104080005B6889199847272138681BF0CCFF124BD1
:1040900020001978FFF7EEF86B69019A9342A1D9D5
:1040A0001000A1E724F0AEFAA9E724F0CFFABAE7AE
:1040B000320021002800019BFFF792FEECE7C0468A
:1040C00063830120B090002070F6021054F50210B6
:1040D00060F50210A5F402106809002077F60210BE
:1040E000E3F302108AF60210F0B585B004000AA8C6
:1040F00005780BA806780020CF68486138708342A5
:1041000019D10123184A194D637613704B762B6829
:1041100083420CD016492000FFF762FC154928683D
:104120001BF072FF144B20001978FFF7A3F8012051
:10413000404205B0F0BD1F78002F0ED101230A4A7E
:104140000A4D637613704B762B68002BEFD008492D
:104150002000FFF745FC0949E1E7009002962000A6
:104160000195FFF7F1FEE4E763830120B0900020A2
:1041700070F60210B4F6021068090020DEF6021094
:10418000F0B585B01D000AAB1E780BAB1F7800237D
:104190000C000392CA684B61029013702800FFF76D
:1041A000B5F8019700962100EB68039A0298FFF793
:1041B0009BFF05B0F0BD000070B50C4C0D002068F1
:1041C000002812D00A4B1B78002B0ED01BF038FFB2
:1041D000084920681BF018FF074920681BF014FFEE
:1041E0000A22290020681BF0C4FF70BDB090002097
:1041F00068090020CD05031005F70210F8B5160078
:1042000004000F00FFF782F8731C43D06369B342C8
:1042100040D042D20122334B334D1A702B68627664
:10422000002B37D020003149FFF7DAFB30492868EE
:104230001BF0EAFE0A22310028681BF09AFF2D4984
:1042400028681BF0E1FE2000FFF722F92A492868C0
:104250001BF0DAFE0A22616928681BF08AFF274EEC
:104260003378002B12D028681BF0EAFE2449286816
:104270001BF0CAFE234928681BF0C6FE39002868D7
:104280001BF0D1FE272128681BF0CDFE20003178DD
:10429000FEF7F0FF01204042F8BD002F18D10122A7
:1042A000104B114D1A702B686276002B10D0200035
:1042B0000E49FFF795FB144928681BF0A5FE310055
:1042C0002000FFF779FF0D4B20001978FEF7D2FF91
:1042D000E4683900A01921F017FE0028DAD0001B8D
:1042E000DAE7C04663830120B090002014F7021083
:1042F00054F50210A0F40210A5F402106809002081
:10430000CD05031002F502101CF70210F8B50F00DE
:1043100004001500FEF7FAFF002F1BD10122444BC9
:10432000444E1A7033686276002B10D02000424948
:10433000FFF756FB414930681BF066FE290020005C
:10434000FFF73AFF3E4B19782000FEF793FF01205C
:104350004042F8BD380026F0C7FE002818D10122DF
:10436000334B344E1A7033686276002B10D0200025
:104370003149FFF735FB334930681BF045FE290012
:104380002000FFF719FF2E4B20001978FEF772FF6F
:104390006B1CDCD06369AB42D9D03DD20122244BE7
:1043A000244E1A7033686276002BD0D02000224948
:1043B000FFF716FB244930681BF026FE0A2229006D
:1043C00030681BF0D6FE214930681BF01DFE20002E
:1043D000FFF75EF81E4930681BF016FE0A2261697D
:1043E00030681BF0C6FE164D2B78002B12D03068BB
:1043F0001BF026FE174930681BF006FE1649306890
:104400001BF002FE390030681BF009FE27213068DE
:104410001BF009FE297897E7002B98D0E468390053
:10442000601923F0A1FB002800D190E7001B90E762
:1044300063830120B090002014F702102EF50210C3
:10444000680900202FF7021054F5021060F50210E1
:10445000A5F40210CD05031002F50210F7B50D000A
:1044600006001400FEF752FF002D1CD10122474B1D
:10447000474D1A702B687276002B10D045493000DA
:10448000FFF7AEFA444928681BF0BEFD210030005A
:10449000FFF792FE414B19783000FEF7EBFE012644
:1044A00076423000FEBD280026F01EFE00280DD109
:1044B0000122364B364D1A702B687276002BEED0E7
:1044C00034493000FFF78CFA3549DCE77369002B7B
:1044D000E5D0621C41D0A3423DD201222B4B2C4F90
:1044E0001A703B687276002BD9D030002949FFF74B
:1044F00077FA2C4938681BF087FD0A2221003868BA
:104500001BF037FE284938681BF07EFD3000FEF7AF
:10451000BFFF264938681BF077FD0A2271693868A9
:104520001BF027FE1D4C2378002B12D038681BF09F
:1045300087FD1F4938681BF067FD1E4938681BF06E
:1045400063FD290038681BF06AFD272138681BF0DD
:104550006AFD2178A0E7A34200D15C1E83429ED36E
:10456000F768012638003B1976420193019B984277
:1045700097D8290023F0F8FA002800D191E7C31B4F
:10458000A34200D933001E000130EFE7638301200E
:10459000B09000204FF702102EF50210680900209D
:1045A0002FF7021054F5021060F50210A5F4021066
:1045B000CD05031002F50210F0B58BB00400049194
:1045C0000592FEF7A3FE049B002B16D101227A4B25
:1045D0007A4D1A702B686276002B0CD07849200037
:1045E000FFF7FEF9774928681BF00EFD764B200097
:1045F0001978FEF73FFE0BB0F0BD059B002B0DD1E7
:1046000001226D4B6D4D1A702B686276002BF2D033
:104610006B492000FFF7E4F96C49E4E76769002F74
:10462000E9D0E568059B9D420DD10122624B634DA7
:104630001A702B686276002BDDD061492000FFF7ED
:10464000CFF96349CFE7049826F04EFD0790002884
:1046500011D10122584B594D1A702B686276002BEC
:10466000C9D020005649FFF7BBF95A4928681BF00A
:10467000CBFC5949B7E7059826F036FD079A069016
:10468000831A089390420CD0089B3E00002B3ADA24
:104690002F0024E02800069A059927F05DFC069B70
:1046A000ED182800049923F05FFA051EF2D1A2E765
:1046B000099B29005E1B32003800BF1927F04CFC13
:1046C0003800069A059927F047FC069B089AFF18C0
:1046D000079B099D9C46636965449B18636128009C
:1046E000049923F041FA09900028E1D1280026F02E
:1046F000FBFC2900421C380027F02EFC7BE7079BBF
:10470000C518089BF6182800049923F02DFA0028F4
:10471000F5D123699E4227D90122274B274F1A70D2
:104720003B686276002B00D165E7049B0290019004
:104730000090320020002249FFF79AFA224B1B78A2
:10474000002B00D157E7254938681BF05DFC244950
:1047500038681BF059FC059938681BF060FC27216C
:1047600038681BF08DFC46E77A1E04992000FFF79D
:1047700075FE62690500E168824216D9079B5B19E4
:10478000C918D21A089BC81827F0E6FBE068089BF6
:104790006769069A05994019DF1927F0DDFB0022A9
:1047A000E3686761DA55954204D10022E3686661E7
:1047B0009A5520E76A1ED8E763830120B090002055
:1047C0006DF502105BF70210680900206DF702100A
:1047D00082F70210A2F70210A9F70210CD0503100C
:1047E000B4F7021010B50249FFF7FAF810BDC04641
:1047F000FBF5021070B5084D04002868002809D0A8
:1048000006491BF001FC2000FEF742FE044928681F
:104810001BF0FAFB70BDC046B090002019F80210E2
:10482000DB070310F0B5150087B004001E000591EA
:104830002F00FEF76BFD002E01D16769EF19059B74
:10484000002B21D101224B4B4B4D1A702B68627605
:10485000002B0DD02000002E13D0FFF7CBFF4749CF
:1048600028681BF0D1FB464B19782000FEF702FDAB
:10487000002E03D00023E26863611370200007B0AC
:10488000F0BDFFF7AFFFEAE7002D05D1002EF5D010
:10489000E36865611D70F1E72A0020000599FEF7C5
:1048A000DBFCA84235D20122324B334F1A703B68F1
:1048B0006276002BDCD02000002E27D0FFF79AFF75
:1048C000304938681BF0A0FB29000A2238681BF029
:1048D00050FC2D4938681BF097FB294D2B78002B95
:1048E00012D038681BF0ACFB284938681BF08CFBF1
:1048F000274938681BF088FB059938681BF08FFB47
:10490000272138681BF08FFB2978AEE7FFF76AFF95
:10491000D6E723699F420FD90122164B62761A709F
:10492000002E17D13A0020001A49059B02950196E6
:104930000096FFF79DF9A1E7002E15D16369E068A5
:104940002A00C018059927F007FB0022E368676179
:10495000DA5593E7002539002B002000059A0195D0
:104960000095FEF7D3FF93E70023E26863611370BD
:10497000E4E7C04663830120B09000202EF50210CA
:1049800068090020C7F70210D0F70210CD05031008
:1049900002F50210FBF5021010B50023FFF742FFED
:1049A00010BD0000F0B587B0150004000591FEF7BA
:1049B000ADFC002D4DD02A0020000599FEF74CFCDF
:1049C000A84249D20122324B324E1A7033686276C5
:1049D000002B3ED020003049FFF702F82F49306805
:1049E0001BF012FB0A22290030681BF0C2FB2C4985
:1049F00030681BF009FB2B4B1B78002B24D0306850
:104A00001BF01EFB284930681BF0FEFA274930686E
:104A10001BF0FAFA264930681BF0F6FA0027059BCE
:104A20000A22D95D30681BF0A0FB6B1E2021306884
:104A3000BB4200D90C3101371BF0F5FABD42EED173
:104A40001C4930681BF0E0FA164B20001978FEF77D
:104A500011FC002007B0F0BD66692369AA199A42CB
:104A60000DD901210A4B61761970002320000193B2
:104A700000930949059B0295FFF7FAF8E9E72A0038
:104A800020000599FFF788FF6069801BE2E7C046B8
:104A900063830120B0900020E5F70210C7F70210F1
:104AA000EBF7021068090020CD050310EBF50210AA
:104AB00003F80210CC09031008B4024B9C460438DA
:104AC00008BC6047A5490010F0B585B00F00040090
:104AD0001500FEF71BFC002F21D10122214B224E95
:104AE0001A7033686276002B0DD02000002D13D091
:104AF000FFF780FE1D4930681BF086FA1C4B200032
:104B00001978FEF7B7FB002D03D00023E26863613C
:104B10001370200005B0F0BDFFF764FEEAE7002D3A
:104B200011D02669002E0ED101210E4B617619702D
:104B300032003300200001960097FEF7E7FEE3689D
:104B400066611E70E5E7002303AE300073703770B6
:104B500026F0CAFA2B00020031002000FFF762FEA7
:104B60000400D6E763830120B090002007F802100C
:104B70006809002010B50022FFF7A6FF10BD000055
:104B80007FB50E000400FEF7C1FB002E17D10122F5
:104B9000174B184D1A702B686276002B0CD0200032
:104BA0001549FEF71DFF154928681BF02DFA144B17
:104BB00020001978FEF75EFB002004B070BD62692A
:104BC0002369013201259A420BD9094B65761D7084
:104BD000002320000849029301930093FFF748F84F
:104BE000EAE731002000FFF7C5FF2800E5E7C046EF
:104BF00063830120B0900020E5F7021010F8021046
:104C00006809002008B4024B9C46043808BC604781
:104C1000814B0010F7B504000D00FEF777FB002371
:104C20000126A36201932B6828001B69984700287E
:104C300027D0626923699A4223D22B6828005B69D6
:104C40009847A36A0133A362002805D0C1B22000AF
:104C5000FFF790FF0196E6E70B4F0C4B38681E708C
:104C600066760028DFD01BF0EBF9094938681BF0A5
:104C7000CBF92000FEF70CFC064938681BF0E8F978
:104C8000D1E70198FEBDC046B090002063830120AB
:104C900016F8021020F80210F7B51E0017000400E5
:104CA0000D00FEF733FB002201AB1E705A709742D5
:104CB00000D11F00A2622B6828001B6998470028BA
:104CC00032D020006669FEF721FB23699E422BD279
:104CD0002B6828005B699847A36A06000133A3622A
:104CE00000280BD0F1B22000FFF744FF310038005C
:104CF00021F00AF90028DED001201AE001220D4E31
:104D00000D4B30681A7062760028D4D01BF098F9E9
:104D10000A4930681BF078F92000FEF7B9FB084912
:104D200030681BF095F9C6E72000FEF725FB01234C
:104D30001840FEBDB09000206383012016F80210D9
:104D400020F8021070B513000400002A17D10122C8
:104D50000D4B0E4D1A702B684276002B0BD00C4970
:104D6000FEF73EFE0B4928681BF04EF90A4B200067
:104D70001978FEF77FFA60690130C0B270BD002279
:104D8000FFF78AFFFAE7C04663830120B090002056
:104D90003BF8021097F602106809002070B5040075
:104DA000002A15D1144B154D01321A702B6842762A
:104DB000002B0BD01249FEF713FE124928681BF096
:104DC00023F9114B20001978FEF754FA002070BD2A
:104DD0001378002B0CD10122074B084D1A702B6859
:104DE0004276002BF2D00649FEF7FAFD0749E5E7C7
:104DF0000023FFF751FFEAE763830120B090002012
:104E00003BF80210B4F6021068090020DEF602102A
:104E100070B505000E0014001000FEF777FA31009F
:104E20002800E268FFF7BAFF70BD0000012270B5EC
:104E3000104B114E1A70336804000D004276002B9F
:104E40000CD0002912D0FFF7D5FC0C4930681BF0BC
:104E5000DBF80B4B20001978FEF70CFA002D03D07D
:104E60000023E26863611370200070BDFFF7BAFC95
:104E7000EBE7C04663830120B09000202EF50210BE
:104E80006809002070B50D0004001600FEF73EFA18
:104E9000002D04D131002000FFF7C8FF70BD2800AD
:104EA00026F022F93300020029002000FFF7BAFCA7
:104EB000F4E710B50022FFF7E5FF10BD10B5024979
:104EC000FEF78EFD10BDC04645F80210F0B585B066
:104ED0000F0004001500FEF719FA002F16D1012269
:104EE000394B3A4D1A702B686276002B0BD020009C
:104EF000FFF7E4FF364928681BF086F8354B197830
:104F00002000FEF7B7F9200005B0F0BD002DFAD063
:104F10002A0039002000FEF79FF9A84230D2012272
:104F2000294B2A4E1A7033686276002BEBD0200092
:104F3000FFF7C4FF284930681BF066F829000A22F1
:104F400030681BF016F9254930681BF05DF8214DDB
:104F50002B78002B12D030681BF072F82049306893
:104F60001BF052F81F4930681BF04EF839003068CA
:104F70001BF055F8272130681BF055F82978BFE75A
:104F80006269236956199E420ED901220E4B627640
:104F90001A70002332000193009320003B00124955
:104FA0000295FEF765FEAEE7E168481926F0D4FFEA
:104FB000E068B84203D02A00390026F0CDFF002275
:104FC000E36866619A559EE763830120B0900020F4
:104FD0002EF5021068090020C7F70210D0F7021062
:104FE000CD05031002F5021045F8021070B50D0052
:104FF0000400FEF78BF9002D15D101220F4B104D47
:105000001A702B686276002B0BD02000FFF756FF3A
:105010000C4928681AF0F8FF0B4B20001978FEF7AE
:1050200029F9200070BD280026F05EF82900020052
:105030002000FFF74BFF0400F3E7C0466383012025
:10504000B09000202EF50210680900200022044BC9
:1050500004495A601960044B5A60044A1A60704748
:10506000A0900020DC280310A8900020F428031052
:105070000023094910B504008360C36003614361E4
:105080008361C3610362436281622C3000F025F8C2
:105090000123237110BDC04688130000074B70B573
:1050A000040083622C300D0000F012F80023200071
:1050B00025602371FFF7DCFF200070BD881300001E
:1050C00010B500210148FFF7E9FF10BD64900020F2
:1050D0000023036043600381704710B50160040042
:1050E0001BF089FA01236060238110BD704770476F
:1050F00070B505000C008E18B44200D170BD2B684D
:10510000217828009B68984720700134F4E710B597
:10511000837D0400002B04D00023837540681DF0BC
:1051200005FD0521207C1CF0E7F8237D002B03D032
:105130000521E07C1CF0E0F8A07C05211CF0DCF8E7
:105140000521607C1CF0D8F8002323726372A372DF
:10515000E3722373637310BDF8B5160001220400D7
:1051600017008B680D1D002B08D1002A1BD0CA68C0
:1051700095420ED1236065602000F8BD1A69B242E5
:1051800004DD3A0098681D000300ECE70022D868AF
:10519000F9E7280020F08CF902690023B242E9DB2C
:1051A00020606360E8E72800F6E7F0B50E00010034
:1051B00085B002AD0400320028003031FFF7CCFF8B
:1051C000039F002F1CD02200029B34320125019244
:1051D000002B06D1974204D03A69964200DB1D1C91
:1051E000EDB2182020F01EF9002301004361066192
:1051F000019B3A00280020F077F9636C0133636467
:1052000005B0F0BD70B50400002C00D170BDE068A1
:10521000FFF7F8FFA5682000182120F0FBF82C000C
:10522000F2E7000010B50400034B0360806BFFF74A
:10523000E9FF200010BDC0463C29031010B5040052
:10524000FFF7F0FF2000482120F0E4F8200010BD17
:10525000F7B50700343705003E00836B01931C1E31
:1052600001D134000EE02269914203DDE36834008D
:105270002600F4E7A3689142FADBE268002B0FD125
:10528000002A19D1EB6BA3422DD1B7422BD1019843
:10529000FFF7B8FF0023EF63AB632F646B64F7BDC8
:1052A0001869814204DC986884461C006346E5E77F
:1052B000DB689C462300F8E71369994202DA16007E
:1052C0009268DDE7D268DBE7200020F0D9F83900EA
:1052D0000190200020F0CAF9182120F09BF86B6C97
:1052E000019C013B6B64B442EED1D8E7030033224A
:1052F0001B010009184343B29B00800893431040F0
:10530000184343B2223240085B00104093431843D5
:10531000C0B2704770B50500C0B2FFF7E7FF0400E8
:10532000280AFFF7E3FF2402204380B270BD7FB557
:105330006B46D9809D1D837D0400181E1BD0637BA6
:1053400088B2012B01D0FFF7E5FF0F2328806068AA
:105350000E2602686E449343802252018218136025
:1053600029000123320029F023FE637B3088012BC2
:1053700001D0FFF7CFFF04B070BDF8B51400827DF7
:1053800006000F00002A13D007224068E5180168C4
:105390004A400F210A408021490141180A60727B6E
:1053A000012A1FD1002C04D11A00390029F0E0FD98
:1053B000F8BD2200002F03D1FF2129F079FDF7E786
:1053C000390029F0EDFDF3E7336830009B68397848
:1053D00098472070737B012B01D0FFF787FF207067
:1053E00001370134A542EFD1E2E77FB56B46D971B1
:1053F000DD1D837D0400181E1DD0637BC8B2012B08
:1054000001D0FFF773FF0723287060680F2602683A
:105410006E4453400F2213408022520182181360C1
:1054200029000123320029F0BBFD637B3078012B7A
:1054300001D0FFF75BFF04B070BD70B505001BF035
:1054400033FD3435AC68A54202D11BF00BFD70BDB5
:105450006169206901221BF0C3FF20001FF0F8FFE3
:105460000400F0E7F0B589B005001BF01DFDD02366
:105470001B061B685A4253412F225B429343534AF7
:10548000944663440493EB6801932B1D0093009BA7
:10549000019A934203D11BF0E5FC09B0F0BD07224D
:1054A000019B1C69E31713401B19049ADB109B0036
:1054B000D718474B3A68234004D50821013B49429D
:1054C0000B4301339B0005931300059A009ED340C4
:1054D0000F2213400393AB68002B1FD1009BB342F4
:1054E00002D033699C426EDA18201FF09BFF039AAA
:1054F000009B029004614261B34219D16B69002B99
:1055000003D02A6913699C423ADC06AE22002900C6
:105510003000FFF721FE069B079A2CE01A6994429F
:1055200003DC9A681E001300D6E7DA683300F9E757
:1055300033699C420FDAEA6896420AD030001FF0C5
:10554000B7FF036902009C42DFDDC368002B17D060
:105550003200012018E09C4230DD2A6996420FD0CB
:1055600030001FF075FF026903009442CDDAF26843
:10557000002A1BD00200002A20D00120002B03D1DA
:10558000009B0120934212D1009B02991FF0ACFFB7
:105590006B6901336B610599039B3A688B405340FB
:1055A00001983B601FF054FF019070E732001369CF
:1055B00001209C4200DB0020C0B2E5E718210298E0
:1055C0001FF028FFE7E7039B7361E4E730410140E8
:1055D00007000080F0B585B0029103920D00817D37
:1055E00002AE04008368002941D09D4209D1B288EF
:1055F00083899A420CD120003030FFF733FF05B089
:10560000F0BD40681DF092FA290060681DF0FAFABA
:105610002000022731000622083002951FF0C2FC4C
:105620006168144A237B8A18486817609A1ED2B2B0
:10563000944638400125019000226046BB43013B5F
:10564000854252415F427B419201DB0113430722B5
:105650001A43CF230E6872401A4080235B01CB1897
:105660001A60054BC918019B0B60A575C3E79D42E5
:10567000CAD1CDE70430000004200000F0B505AC2D
:10568000267806AC27780C4C0500046000243435DD
:1056900004622C70C5630564477486748463446433
:1056A000416044758475047244728472C4720473D8
:1056B00044730274C374F0BD3C290310F0B50700B5
:1056C00085B00D001022684619491FF06BFC7E7DE5
:1056D0006C46002E15D1174A7B6801209B185A4250
:1056E00053410021DB002A00E41829F001FC236863
:1056F000184063681940084303D03D74012005B089
:10570000F0BD3B7CAB42F9D078680B4A0B4B0C499F
:10571000002E05D0904200D119000A481BF0B8FDB8
:10572000904200D119002A0007481BF0B1FDC04685
:10573000782903100000FCBF00000440DA120310B7
:10574000210B03104CF802107CF80210F0B5070092
:1057500085B00D001022684619491FF023FC7E7D9C
:105760006C46002E15D1174A7B6801209B185A42BF
:1057700053410021DB002A00E41829F0B9FB23681B
:10578000184063681940084303D0FD74012005B038
:10579000F0BDFB7CAB42F9D078680B4A0B4B0C494F
:1057A000002E05D0904200D119000A481BF070FD70
:1057B000904200D119002A0007481BF069FDC0463D
:1057C000882903100000FCBF00000440DA12031017
:1057D000210B0310B0F80210E0F80210F0B507003A
:1057E00085B00D001022684619491FF0DBFB7E7D55
:1057F0006C46002E15D1174A7B6801209B185A422F
:1058000053410021DB002A00E41829F071FB2368D2
:10581000184063681940084303D0BD74012005B0E7
:10582000F0BDBB7CAB42F9D078680B4A0B4B0C49FE
:10583000002E05D0904200D119000A481BF028FD27
:10584000904200D119002A0007481BF021FDC046F4
:10585000982903100000FCBF00000440DA12031076
:10586000210B031014F9021045F90210F0B50700DE
:1058700085B00D001022684619491FF093FB7E7D0C
:105880006C46002E15D1174A7B6801209B185A429E
:1058900053410021DB002A00E41829F029FB23688A
:1058A000184063681940084303D07D74012005B097
:1058B000F0BD7B7CAB42F9D078680B4A0B4B0C49AE
:1058C000002E05D0904200D119000A481BF0E0FCE0
:1058D000904200D119002A0007481BF0D9FCC046AD
:1058E000A82903100000FCBF00000440DA120310D6
:1058F000210B03107AF90210AAF9021070B5040006
:105900000D00007C01211BF0F7FC2575002D03D054
:105910000121E07C1BF0F0FCA07C01211BF0ECFCE1
:10592000607C01211BF0E8FC23682000A168E2688C
:105930001B6A9847236820005B6A984770BD10B5C2
:105940000021FFF7DBFF10BD132307B50193013BD7
:105950001022084900930848013BFFF78FFE0F23F0
:105960000193013B00930C2204480549013BFFF7DA
:1059700085FE07BD00C00340D8890020208A002092
:1059800000000440002270B5022406200321264BAB
:1059900007251A705A70254B08261C705C70244B22
:1059A000244A19705870012310705370224A1570E0
:1059B0005370224A16705570214A2D191570547073
:1059C000204AED18157054701F4A0A341470537031
:1059D0001E4AE418147053701D4AAD1915705370A7
:1059E0001C4A0735157053701B4A073515705370E4
:1059F0001A4AED1815705370194A05351570537011
:105A0000184A113515705370174A10705370174AA1
:105A1000233014705370164A51701070154A30318B
:105A20001170537070BDC0463A8301203C83012041
:105A30003E830120408301204283012044830120D2
:105A4000468301204A8301204C8301204E8301209C
:105A5000508301205283012054830120568301206A
:105A6000588301205A830120488301205C83012050
:105A70005E8301206083012010B5034B01001800F4
:105A800000F08AFA10BDC046188B002070B50024C3
:105A9000054B1D78AC4200D170BD2000013400F0F0
:105AA000F7FBE4B2F6E7C0466283012013B56B460C
:105AB0000268D9710733546819000122A04716BD46
:105AC00010B5407D0024FF2805D000F0AFFB041E78
:105AD00001D11AF08AFD200010BD13B5407DFF28CA
:105AE00002D10120404216BD6B46DC1D210000F0B2
:105AF000C3FB0028F5D02078F5E713B5407DFF28DB
:105B000009D06B46DC1D0122210000F09BFB002820
:105B100001D0207816BD01204042FBE710B5407D42
:105B2000FF2801D000F0B4FB10BD10B5437D00206C
:105B3000FF2B02D0180000F007FC10BDF8B5437D24
:105B400006000F0015000020FF2B10D1F8BD3F18F4
:105B50001AF04BFD707D00F043FB00280AD02200B4
:105B60003900707D00F0D0FB241A02D0EFE7141E3C
:105B7000F0D10024281BE9E7F0B597B00600171E06
:105B800003931FD08021494208004C4B5D7FAA1C23
:105B90005A779A7F1043C0B20190901C0132114392
:105BA000CAB20292DA7F987700920132DA7705ACB6
:105BB0004222002120001FF0EFF9002F07D14220E0
:105BC00017B0F0BD1500009202920192EFE7039B1F
:105BD0000020412BF4D93A48317DA0803948217406
:105BE000208139480521A081DE38FF38A07437486C
:105BF000A5700A90012020763548A5720C90354892
:105C00006B1C208404A80730C5770B258C46617473
:105C100004A96D1801990426E9772B2504A94919CF
:105C2000283D0D7004A929354919243D0D70912591
:105C30002D016585302504A949190E70013504A987
:105C4000DBB206A86D18244AA376C3772B700B002D
:105C50003321228002225B1834251A700A2304A9FA
:105C600049190B7004A930331C485B180099E27085
:105C7000A273A084A086E67619703B2104AB5B1862
:105C80001A70402304AA013152181370033104AA78
:105C90005218393B1370402204AB9B1862461A70AD
:105CA000412304AA9B18029A21001A700C4B42222D
:105CB0003800E3871FF076F981E7C046178C002093
:105CC0000202000009040000010200002001052476
:105CD0002402060524060000080B0000070500004A
:105CE0000240000008B4024B9C46103808BC6047D4
:105CF000795B0010002343600375054BFA220360B3
:105D0000044B92000361FF23826043757047C046D5
:105D1000C0290310E829031010B5437DFF2B0FD1D4
:105D2000084A1378012B0BD8437510300400591C16
:105D30001170054900F0BEF92100044800F00CF98B
:105D400010BDC04662830120DEF90210188B0020CE
:105D500007B500290BD1002809D1694600F058FA8F
:105D60009623009ADB009A4201D100F0EFF907BDBB
:105D700010B50248FFF7BEFF10BDC046688A00207C
:105D8000F7B584460020020063469D189B5C002BFB
:105D90006ED01C004034E4B2012C0FD9F42B0DD886
:105DA0005CB2002C0CDB01246E1C2D190195019DA9
:105DB000AE421DD1012C27D17F2B2DD90132E3E733
:105DC0001F241E00A643C02E02D123401D3CEBE73A
:105DD0000F241E00A643E02E02D123400C3CE3E733
:105DE00007241E00A643F02EE8D12340033CDBE746
:105DF0003F27357801360095BD43802DDED1009DCB
:105E00009B013D402B43D2E7022C26D11D00F026FA
:105E1000803DF600B542D1D2202829D01219440085
:105E200063520130B0E7F826124D36025D19B542D3
:105E3000C4D28026104D36015D19B542ECD2BDE7C3
:105E40000E4E9D0A4400AD190D539B050C4D9B0D44
:105E50000C195B190230638096E7032CE3D0094CE0
:105E60001B1980246403A342A8D204321E28E7DD54
:105E7000FEBDC04600F8FFFF0028FFFF00D8FFFF6F
:105E800000DCFFFF0000FFFF018142817047FC3012
:105E900081627047FC30C1627047FC30016370471B
:105EA000A82210B552000300805C0B2808D80029F6
:105EB00008D0441C9C54020048329200D15010BDBE
:105EC0000020FCE70800FAE770B5040088B01D4E1A
:105ED00003AD3100122228001FF064F8230007CD23
:105EE00007C32A6831001A60AA8825009A801835ED
:105EF0000922684612311FF055F869460922280028
:105F00001FF050F8104B6561E435EB6180222300EF
:105F10002000FE335200DA832D300133FF3ADA7766
:105F200000212332FF301FF037F8084B04226B6248
:105F3000074BAB62074BEB62A8235B00E25408B04F
:105F400070BDC046EC2903100900000109040000DF
:105F5000EDF90210FFF90210F8B504002500080061
:105F60002600FE35698BAB8B626907685B1AFF36CA
:105F700052183F68717F9BB2B84700280AD06A8BDD
:105F80008318012062699BB26B8393701B0AD370E4
:105F9000737F1371F8BD000070B504000D00012679
:105FA000FFF792FFE121064BA671A3804902054845
:105FB000FFF7B2FE280000F0A3F8300070BDC04625
:105FC000EF020000688A0020F0B5FC30056B8BB052
:105FD0008C1C002D25D102A800F0BDF80090009A7D
:105FE000EBB2934218D2114B06AF190010223800C1
:105FF00001931EF0D7FF02AB5E5D0F233340FB5CC5
:10600000102263803800019936111EF0CBFFBB5D72
:10601000013523800434E2E7009B5800C0B20BB086
:10602000F0BD21002800FFF7ABFEF7E70AFA0210E7
:1060300010B50400002911D0032920D0A8235B004B
:10604000C35C00208B4219D948318B0021005531A7
:106050001859FF31FFF794FEC0B206E00300FC338D
:106060005A6AAA235B00C2520120C023A922013030
:1060700040009B0003435200A352A01810BD010032
:106080005331FF31FFF7A0FFEFE7000000487047F2
:10609000188B0020014B58697047C046188B0020B0
:1060A00010B5034B0A0001001800FFF7C1FF10BD37
:1060B000188B002010B504000248FFF7F1FE207194
:1060C00010BDC046188B002010B5024B18681BF09D
:1060D00009FA10BD648F002010B5084C0021200083
:1060E00028F02EFF002807D001200021404200F0B8
:1060F00075FF200028F0E4FE10BDC046C8900020C7
:1061000037B505000D481BF001FC01246B4601A9C1
:1061100028009C8000F02AFE20001BF0E3FB084DC5
:10612000084928601BF0EEF9286821001BF0BAF935
:106130000022052004491BF005FA37BDC890002055
:10614000648F0020D9600010C9600010002110B5D4
:1061500008001CF0FDF810B51EF0B4FF082010BDBB
:1061600010B5084C0021200028F0EAFE002807D0D6
:1061700001200021404200F031FF200028F0A0FE65
:1061800010BDC046C890002070B5040000F0DEFDD0
:10619000002820D000F0E2FD051E1CD1E378002B82
:1061A00019D026001036300000F002FC3F2812D92A
:1061B0002800E17800F084FE00280CD0300000F0C8
:1061C000F7FBE1783F2807D992239B00E2182800CB
:1061D000402300F099FE70BD280000F083FEFAE72E
:1061E00010B5040000F0B2FD002801D1002010BD60
:1061F00000F0B4FD0028F9D1B22080006043034BC9
:106200001B18187901231840F1E7C046D4900020EC
:1062100003000800B221890010B55943024B072240
:10622000C9181EF0BFFE10BDDC900020B2239B00F9
:10623000434310B50248181800F08CFB10BDC0464F
:10624000E490002070B5B2248023A40044435B0294
:106250009A4200D3064A2000064E103092B28019AE
:1062600000F0DBFB0500A019FFF78EFF280070BDD2
:10627000FFFF0000D4900020B2239B00434310B5E1
:106280000248181800F0ECFB10BDC046E490002056
:10629000F7B5060000F05AFD002830D000F05EFD92
:1062A000051E2CD1B224A40074432600154F2436B9
:1062B000F619300000F04EFB002820D03B192800D2
:1062C0009978019300F0FCFD002818D0A2239B00D0
:1062D000E418E41921003000402200F09EFB019BED
:1062E00006009978002808D003002200280000F05A
:1062F0000BFE002803D03000FEBD00F0F3FD0020AF
:10630000FAE7C046D490002070B5B224A4004443FC
:106310000B4B0500E41880235B029A4200D3094A24
:10632000200092B200F0E8FB0600200000F012FB13
:106330003F2802D92800FFF7ABFF300070BDC046F0
:10634000F8900020FFFF0000B2239B00434310B5EC
:106350000248181800F02CFB10BDC046F890002031
:10636000B222F0B500252E4C85B000212000D200CD
:106370001EF012FE2B4BE1211D700827FF23802207
:1063800049026371A160A77327490095FE3B520043
:10639000264800F0ADFA012680223300244952003D
:1063A0000096244800F0A4FA234802901BF0AEFAAD
:1063B000224803901BF0AAFAFF22E121204B029809
:1063C000E25449020333E1500433E55220621D4B8D
:1063D0000398E75420633300E561656392191A4915
:1063E00000951A4800F084FA8022330018495200C0
:1063F0000096184800F07CFA174F38001BF086FA18
:10640000164E30001BF082FAB9239B00E55004338E
:10641000E7501033E6500433E55005B0F0BDC046F8
:10642000D4900020698301200C910020E49000208A
:106430000C920020F89000200C9300201493002070
:10644000CD020000D6020000D4930020AC930020BF
:10645000D4940020C0930020D4950020DC95002027
:10646000114B30B51A6A196B002A02D00022DA618A
:106470001A62002902D000221A635A63BA22BE218E
:106480009200985889005C58002804D0B925002053
:10649000AD0058519850002C04D000225A50BF2112
:1064A00089005A50012030BDD490002070B50522DB
:1064B000002116481EF070FD154C2378DB0702D42E
:1064C000144800F0A1FB2378134D9B0702D4280049
:1064D00000F09AFB0121280000F0B5FB0522002105
:1064E0000E481EF059FD2378DB0702D40C4800F05B
:1064F0008BFB23780B4C9B0702D4200000F084FB1D
:106500000121200000F09FFB70BDC046D490002008
:1065100069830120E4900020F89000209C930020E3
:10652000AC930020C0930020F0B587B004904B7965
:10653000022B03D00025280007B0F0BD8B79022B79
:10654000F8D1284EB778002F04D0274BF35C002BEE
:10655000F0D10127B22309259B007842184003900F
:106560007B43301805908878F0540C780C196378C8
:10657000242B24D195421DD96378042B16D163793D
:106580000A2B13D1039B27780233F3180193039B43
:1065900004980333F6180223E1191A00009600F05C
:1065A00069FC0028C6D00E35ED19ADB20598FFF78D
:1065B000EBFDC0E723785D19ADB2E418D7E7052BF2
:1065C000DAD12100049800F03BFC0028B2D0B223BD
:1065D0009B007B43A278F3185A7023785D19ADB203
:1065E000E418C9E7D4900020CA020000F8B50400FE
:1065F00060200B001100127800260240202A2CD1C6
:106600004D790A792D0215432E4A1078A8420FD0F1
:10661000B2208000125CAA421FD101252A4A487884
:1066200000262038032818D828F0D2FC04191C3C76
:106630003500F4E7012B05D120000832063300F0C5
:10664000D7FF09E0032B07D1204B002B04D00832E1
:106650001100280000E000BF01263000F8BD012B2A
:10666000FAD1E9E7012B03D1200000F0AFFFF3E7F7
:10667000032BF1D10126CC788B78310024021C4306
:106680002700147124321000A14300F0DCFA104BF3
:106690003740002BE0D06208390028003240FFF775
:1066A00057FBD9E7012BDFD0032BD5D1094B002BAA
:1066B000D2D08B78C97828000902194300E000BFC6
:1066C000CAE7C046D49000209C9300200000000040
:1066D000515D001000000000F0B5404C85B0029004
:1066E00000911E00E3788B424ED0A3788B4249D0B4
:1066F0003B4BE35C8B4200D16DE03A4B0020E35C06
:106700008B4266D10125384C5EE062793B789A4233
:1067100008D1019800F032F9002803D128006179EE
:1067200000E000BF013746E0019800F027F900289B
:1067300047D1280000E000BF43E02C4B002B02D0E3
:10674000280000E000BF2800FFF7A2FD00283FD18D
:106750002000243000F0FEF8002839D1002E37D078
:106760003F2335001D401E4232D1A178029800F02F
:10677000A7FB00282CD02B002A00A178029800F05B
:10678000C3FB25E000251FE0002523001033019303
:1067900092239B00E71839000198B2B200F0ACF9DF
:1067A000134B002B0AD06379FF2B07D092239B0059
:1067B000F318E3180393039BBB42A6D10D4B002BA8
:1067C000B2D12000FFF7E0FCA378009A9342B4D046
:1067D000012005B0F0BD0125034CD6E7D490002080
:1067E000CB020000CA0200009C93002000000000C1
:1067F00000000000000000008A1892B240009142A0
:1068000001D8824201DB121A92B21000704770B5B3
:106810000500D41A0800A4B2A9889A4202D24E00F8
:10682000A419A4B2261E11D0A14204D291420FD8BD
:10683000521A93B26B8199420CD9EA8829685204A2
:10684000520C5343C9181EF0ADFB0126300070BD39
:106850008A18EEE75B1A9BB2EDE7F0B585B00391BD
:106860000AA90C8801901D1B8688ADB2A34202D2F2
:1068700071006D18ADB2002D21D0AE4206D29E42FD
:1068800020D89B1B35009CB2019B5C812B1C954240
:1068900000D9131C9DB2A64216D9019B019ADB8830
:1068A00011685B045B0C02936343371BBFB2C918CA
:1068B000BD420CD8029A03986A431EF073FB28006D
:1068C00005B0F0BDF318DDE7A41BA4B2E3E7029B1B
:1068D00003985F43BFB23A001EF064FB039BAE1BFC
:1068E000D819029BA2195A43019B92B21968E4E796
:1068F000F7B5019308AB1D78802304000F00160044
:1069000000201B029A4221D8E068002803D0012110
:10691000494228F025FB2069002803D00121494283
:1069200028F01EFB019BED035B045B0C1D43002361
:10693000E06863812760A680E5802381984201D0CA
:1069400028F0BEFA2069002801D10120FEBD28F000
:10695000B7FAFAE710B5048941898288A3B288B2F0
:106960008C4207D31B1A9BB2101C9A4200D9181CE8
:1069700080B210BD5100091A5B18F4E70389408901
:10698000181A43425841C0B2704710B50489428971
:106990008188A3B290B2944206D31B1A00209BB206
:1069A0008B424041C0B210BD4A00121A9B18F5E755
:1069B00010B5048941898288A3B288B28C4207D37A
:1069C0001B1A9BB200209A4201D9D21A90B210BD74
:1069D0005100091A5B18F4E770B5040000690D0056
:1069E000002803D00121494228F0BAFA228963899C
:1069F000290092B29BB22000FFF709FF05006189D0
:106A00002A00A08889B2FFF7F7FE6081206900287C
:106A100001D028F055FA280070BD73B50400006954
:106A20000D001600002803D00121494228F098FAF1
:106A30002389628929009BB2009220003200FFF76F
:106A40000CFF050061892A00A08889B2FFF7D4FEF7
:106A500060812069002801D028F032FA280076BD34
:106A600070B5040000690D00002803D001214942DF
:106A700028F076FA228963892900200092B29BB21D
:106A8000FFF7C5FE05002069002801D028F018FA9C
:106A9000280070BDF8B50400C0680E00002803D0BF
:106AA0000121494228F05CFA25892000ADB2FFF7A8
:106AB0006CFF002802D0E779FF0913D02800A388D3
:106AC000834216D9E28823685204520C50433100A5
:106AD00018181EF067FA01222900A088FFF78CFE23
:106AE00001272081E068002801D028F0E9F938006A
:106AF000F8BDC01A80B2E3E7F0B585B00600141EF9
:106B000001913FD0C068002803D00121494228F0FC
:106B100027FA3789F3797189B588BFB289B2DB0961
:106B200037D18F4231D3791A89B2A94200D369E0B3
:106B3000691A0B1C89B2A14200D9231C9CB2009790
:106B4000009BAB4245D2F28830685204520C02924C
:106B50000299009AEB1A4A439BB28018A3423DD394
:106B60000A00624301991EF01DFA22003900B08824
:106B7000FFF742FE25003081F068002801D028F0A0
:106B80009FF92C00200005B0F0BD6B00591A791850
:106B9000CAE7AC420CD3002DEED0631BF4880F0083
:106BA0006404640C5C43019B1B1901932C00C6E731
:106BB0006A007B1A8F4201D2531AFB189BB21B1931
:106BC0009342BCDB2A1B280092B2FFF715FE070098
:106BD000B5E7009B5B1B9BB20093B1E7029A01995A
:106BE00053439BB21A0003931EF0DCF9009B651B14
:106BF0005A19029B01995A43039B30689C4692B2F2
:106C00006144B0E70025B7E710B50400C06800286C
:106C100003D00121494228F0A3F92069002803D0BC
:106C20000121494228F09CF90023E0686381238117
:106C3000984201D028F044F92069002801D028F0BA
:106C40003FF9012010BD70B50400C0680D00002898
:106C500003D00121494228F083F92069002803D09C
:106C60000121494228F07CF97F23E179ED011940A7
:106C7000E0682943E171002801D028F021F920695A
:106C8000002801D028F01CF9012070BD0CC8BFF30A
:106C90005F8F0021116083F3108870470168EFF364
:106CA000108372B60A68002AFCD0BFF35F8F43607E
:106CB000704770B505000C001600486900F0CAFC6A
:106CC0003200280001216369984770BD70B5050046
:106CD0000024134B1B78A3420FD2542200211148E9
:106CE0001EF05AF91022FF210F481EF055F92022FC
:106CF000FF210E481EF050F907E0A34206D90C4BC5
:106D000062011B689B18002B04D170BD094AE31A6D
:106D10005B019B182800DB6801349847E4B2D8E790
:106D2000688301206B8301206F8301207F83012012
:106D3000D0900020082A0310704770470020704749
:106D4000002070477047704770477047024B587873
:106D5000431E9841C0B270476B830120024B1878E4
:106D60004007C00F7047C0466B830120F7B5284F1E
:106D700005003B780E00FF2B33D1002901D1002004
:106D8000FEBD0021542223481EF006F90022224CA9
:106D9000224B20001A701AF0B9FD214B21481C60CB
:106DA0001AF0EEFD204C2000FFF72EFF1F4B204A6B
:106DB0001C60204B0192002B04D0100000E000BFAB
:106DC0001D4B18600024019B1B78A3420BD231009D
:106DD00028003D7000F026FE0028D0D0280000F0EA
:106DE00065FE0120CCE7A3420CD9134B62011B685E
:106DF0009B18002BC3D05B68002BC0D00134984790
:106E0000E4B2E0E70D4AE31A5B019B18F3E7C046E2
:106E10008C0900206B830120789600207F8401205C
:106E2000C09600208409002070090020C49600202C
:106E30006883012000000000D0900020082A031081
:106E4000702370B58A780C001A4201D0002070BD02
:106E5000064B20001D78064B997801F05DF800285C
:106E6000F4D02100280000F06DFEF0E78C0900202E
:106E70006B830120F7B50C0016001F000025019060
:106E8000AE4201DC012003E06378052B01D0002035
:106E9000FEBDE3789B079B0FBB42F8D12100019810
:106EA000FFF7CEFF0028F2D0A378DA09012A05D136
:106EB000099A137023780135E418E1E7089AF8E796
:106EC0007F2010B50840C909044B054A3431400001
:106ED00040188018196800F0DBFF10BDC096002034
:106EE0006B8301207F2010B50840C909044B054A77
:106EF0003431400040188018196800F0F1FF10BDCF
:106F0000C09600206B83012070B57F240E480C4092
:106F100064000419CD09641930342079C00710D4F5
:106F20000125267909482E430078267100F02EFEAF
:106F3000002807D104222379AB432371237993439B
:106F40002371002070BDC0466B8301208C09002096
:106F500010B50B4B0C00187800F03AFE7F22094B5D
:106F60002240520099180223E409091930310A79A4
:106F700013430B7101230A7913430B7110BDC046F3
:106F80008C0900206B83012010B50B4B0C00187886
:106F900000F03AFE7F22094B22405200991802224B
:106FA000E409091930310B7993430B710B79013ADC
:106FB00093430B7110BDC0468C0900206B830120E8
:106FC0007F22054B0A405200C9099B185B183033D9
:106FD00018798007C00F70476B830120F0B5BB4B59
:106FE0008BB01B78FF2B00D17BE2B94B07AC1D683F
:106FF0002E0014363000FFF751FE28002100FFF765
:10700000EBFC05003000FFF741FE002D00D168E2E7
:10701000607801380728E8D827F07AFF08001100C7
:1070200088026E02790219003E0281022078FFF781
:107030004DFE00F005FBA74B22799A70D5E720782A
:10704000FFF744FE00F0FCFAFFF77DFECDE7A24A11
:107050001378002B00D144E21378013BDBB21370AC
:107060001378D8B2002BC0D101269A4D04212B7879
:10707000277833432B702B0034331A78B2431A70BD
:107080001A788A431A702B0035331A78B2431A7073
:107090001A788A431A7000F0DDFA602322791340CF
:1070A000602B29D0402B0CD18C48002824D000F034
:1070B000D1FA3100380008AA00E000BF002894D1BE
:1070C0001AE0D206D20E012A00D161E1022A00D1D3
:1070D00092E1002A10D1202B20D1237A0F2B0BD83C
:1070E0007F4AEB181B79127893420FD27D4A5B01DD
:1070F0001168C91800290CD107AC2078002100F0D4
:1071000067FD8021207800F063FD6EE79342F3D1A4
:10711000754908AA3800FFF7CCFDCFE7002BEBD16B
:1071200060790928E8D827F033FF24011C01E7FF24
:107130001301E7FF0A00B900E7FF16001C0008A8CA
:1071400000F08EFA3800A17900F0C6FC02232A78FC
:1071500013432B7049E706AA6B78023213700123A0
:1071600011E1A4796B789C423BD06B78002B0BD05B
:107170000021380000F0C8FC380000F003FDAE78B4
:107180003800FFF7A3FDAE706C70002C00D182E0D8
:10719000013CE0B2FEF77EFF002803D100224D4BF8
:1071A0005A70A9E743780393022BF7D10121C279E2
:1071B000931152110B400A4012015B0113432A78CC
:1071C0002F318A4313432B700500C37882781B024A
:1071D0001343C31809350493049BAB4206D8FFF749
:1071E000B1FD380008A900F0F1F9FEE601226B7844
:1071F00001920B2B03D1EB7801932B78ED186B7870
:10720000042BCBD10026049B5B1B9BB20593344B14
:107210001C78B442C2D32BD9324A73011468E418E3
:10722000002CBBD0290038002369059A98470290AA
:1072300008282DD9059B83422AD3019B012B05D118
:107240002A4B22699A4201D1039B019300222149D2
:10725000019B9A4211D1330029002548029A00F07F
:107260008BFE029BED181E4B1B78B342B4D295E700
:107270001D4B341B6401E418D4E7AB78D318DBB2A0
:10728000CB181879FF2889D101321E71D2B2DFE7FD
:107290000136F6B2BBE7FFF756FDA2E7E3881A0A0C
:1072A000501EDBB20E2800D926E727F071FE23001E
:1072B0003C00450025FF25FF4E003C0025FF25FF33
:1072C00025FF25FF25FF25FF25FF2E008C09002027
:1072D000C49600206B8301207F8401200000000001
:1072E00068830120D0900020082A0310296500102F
:1072F0007F830120FEF7CAFE1223021E00D1FBE6A7
:10730000380008A900F074F9D8E6904B002B00D1A2
:10731000F2E600E000BF021E00D1EDE6C3788178FE
:107320001B020B43ECE71800022A02D1FEF7B2FE63
:10733000F1E7FFF705FDEEE718002189FEF7B0FE43
:10734000021E00D1D8E60378DAE7FFF7F7FCF7E78B
:10735000E388012B00D0CFE62A78073313432B7044
:107360003FE7E388012B00D0C6E608222B78934341
:10737000F5E72B7806AA980699080223C00F194052
:10738000023201431180380008A900F031F92CE6DF
:10739000237A0F2B00D9AFE66D4AEB181B791278D0
:1073A000934224D26B4A5B011168C918002900D1AD
:1073B000A2E6380008AAFFF77CFC002800D014E6FB
:1073C0002279602315001D401A4200D094E66379AB
:1073D0000A3B012B00D98FE6280000F03BF96379C6
:1073E0000A2B00D0FDE606AB9A1C1570B7E6934257
:1073F00000D081E65849DCE77022217A114200D0A2
:107400007AE60F320A405200C809AA1812185048EA
:10741000127D0078824216D24E4852010668B61894
:10742000002B19D1637902201A008243012A17D058
:10743000002B00D060E63800FFF7C2FD06AB9A1CB7
:10744000108002239FE7824200D079E0424E002B59
:10745000E8D0310008AA5DE6002E00D14CE6F8E73E
:10746000E288002A04D13800012B12D1FFF78CFDED
:10747000002E00D1B9E5310008AA3800FFF719FC49
:107480003535002000F0E6F82B78DB0700D5ACE5B9
:10749000A7E6FFF75DFDEBE77F2221792F4B0A403E
:1074A0005500C8095B191B181800012630300579F2
:1074B000B543057105790336B5430571002A05D139
:1074C00062792078A36800F0D9F88EE5204A1B7D08
:1074D0001278934207D21F485A0103689B18002B69
:1074E00004D10BB0F0BD9342FBD11B4B9D69627977
:1074F0002078A368A84778E5184B1A78D20700D4FB
:1075000073E518780007C00FFFF71EFC6DE5134BFD
:107510001B78DB0700D468E5FFF717FC65E56368B7
:10752000002B00D161E5A06898475EE501220B4B76
:10753000DB78134200D158E56068FFF7FEFB54E5A5
:107540000026002B00D0D7E56CE7C0460000000005
:1075500068830120D0900020082A03106B8301204B
:1075600070B5134B06009C89D889221A151C92B25B
:10757000402A00D940251A78ADB27F2A0ED984421C
:1075800012D00C4C2A00996820001DF00BFD8021C0
:1075900022002B003000FFF7B7FC70BD00210A006D
:1075A0008442F6D0034AF4E780210022F1E7C04686
:1075B000649600208096002080238B4319000023CE
:1075C00010B51A00FFF7A0FC10BD000070B5074C05
:1075D00006000D00082220001DF0E4FC002330000E
:1075E0002978A360E360FFF7E7FF70BD6496002091
:1075F000F7B5124F15000190082238000C001E004C
:107600001DF0D0FC0023BD60FB81E379A2791B0251
:1076100013431A1CB34200D9321C91B2BA81002B19
:1076200007D0002901D0281E02D00198FFF798FF4B
:10763000FEBD21780198FFF7BFFFF9E764960020AF
:1076400010B51422002102481DF0A6FC10BDC04652
:1076500064960020014B18617047C0466496002074
:1076600010B5054C0100082220001DF09BFC0023F2
:10767000A360E36010BDC0466496002070B5234C43
:107680001E0023780500DA09C9098A420FD00020BC
:1076900086420BD12100280000F048FA2369002B14
:1076A00003D02200032128009847012070BD7F2BC2
:1076B00006D8A368181EF9D0320015491DF072FCD7
:1076C000A268E38992199B19A260E2889BB2E381C8
:1076D0009A4201D03F2E15D82369002B04D12800EF
:1076E0002178FFF769FFE1E702212200280098478F
:1076F000011EF4D1280000F06BFA8021280000F070
:1077000067FAD2E72800FFF72BFFCFE76496002047
:1077100080960020F8B57F230340C4095D00304EF9
:107720002F197F01F719B8700120A043787000204D
:10773000F87098013983FA768C46DF003018012CF6
:1077400010D128497F188762002728194001301876
:1077500080680760BB4209D1640134196360224B21
:10776000E360F8BD21497F188760EDE7581E9B0153
:10777000C000F318012C1AD11D4940185862614607
:107780003F233F3189B29943022A00D14900194869
:107790002D1903686D0175195918EB600160880691
:1077A00009D05121144B154A15481EF0F9FA154914
:1077B00040185860E3E7144843404840802149019D
:1077C000884204D95321114B0C4A0D48EDE792062B
:1077D0001A4380231B0613436A681360C1E7C0463F
:1077E0009CD70020800010500001105084001050E1
:1077F0000800105000E800201BFA0210632A031052
:107800004AFA02100C00105000001050D7FA021073
:107810000023190010B50948DA00121801339160ED
:10782000D1600F2BF7D1F0229200002104481DF007
:10783000B3FB044B044A1A6010BDC0460000105050
:10784000DCD7002000E80020800110506C4BF0B520
:107850001F6880233C009B0287B01C401F4214D04D
:10786000684A1278002A01D1674A1360C022674B28
:1078700092009B6C02A95B058A805B0D012180242C
:1078800003A8049327F07CFBA40210231F420CD012
:107890001C435E4B01269B6D019300230093019BCB
:1078A000002B02D0009B202B78D180235B021F424B
:1078B00035D00225564E1C43B37E002B1AD019F04A
:1078C000E1FC012806D9534B504A1D66536E2B40EC
:1078D000AB42FBD1C02200213000920100F046FAF9
:1078E000300000F03DFA19F0CDFC012802D94A4BD6
:1078F0005D661D660123F37020369D427BD1C02357
:1079000002AADB009380454A04AB03CA03C32900E3
:1079100003A827F035FB80223F4B92021A65802393
:107920005B011F4212D000251C43384B1D60FFF73E
:107930006FFF802302AA5B0093801572012103A8C8
:1079400027F01EFB8022344B12031A658023DB01D3
:107950001F420BD01C43802302AADB00938001212D
:1079600003A827F00DFB10222B4B1A6580231B0266
:107970001F420CD01C43A02302AADB0093800121EC
:1079800003A827F0FDFA8022234B12011A65BC429E
:1079900033D021002248794019F07AFC019B1E4225
:1079A00023D01D4B009A9E65009B5D0801236D004E
:1079B0009343ED18164B6D01ED18280000F044FAC2
:1079C00000280FD0EB8AE02105930023AA7803A8B2
:1079D000C900018002714371012127F0D1FA28000A
:1079E00000F0BEF9019BB3430193009B7600013385
:1079F000DBB2009353E701255EE707B0F0BDC04658
:107A0000980011506A8301209030115000001150ED
:107A10009CD7002000201150003011500000105061
:107A200008FB021070B5041E06D0BB21164B174A86
:107A3000174849001EF0B4F900F072F90C23154DF7
:107A4000FF22AB670520144919F07CFD210040227C
:107A500012481DF0A1FA220020004021FFF75AFE33
:107A6000220040218020FFF755FEFFF7D1FE802342
:107A700001209B0528640A4AEB640A4B1A608022A5
:107A8000094B5202DA6470BD1CFB0210762A031007
:107A90004AFA0210000011504D7800109CD70020C7
:107AA00010D00100900011500020115010B5002896
:107AB00006D0D521054B064A064849001EF070F94C
:107AC0000121052019F0EEFC10BDC0461CFB021080
:107AD000542A03104AFA0210010010B5002806D0FB
:107AE000DA21054B054A064849001EF059F90A00FB
:107AF000044800F09FF910BD1CFB0210442A03103B
:107B00004AFA0210BCD70020054B197080239B0253
:107B1000002902D0034A13607047034AFBE7C046BE
:107B20006A83012090201150903011500B785B0631
:107B300005D14B78052B02D18A78014B1A6070472A
:107B40000000115010B50C00002806D0F2210A4B9D
:107B50000A4A0B48FF311EF023F96379CA78097984
:107B60001B020B435B059207A078920F590DFFF79C
:107B7000D1FD012010BDC0461CFB0210362A0310A7
:107B80004AFA021010B5FFF743FE10BD10B50C0005
:107B900011001A00002806D0FF21094B094A0A48A3
:107BA00049001EF0FDF87F2020404000E409074B0B
:107BB00000194001C01800F03DF9012010BDC04679
:107BC0001CFB0210282A03104AFA02109CD700203E
:107BD0007F2307B508001840194204D14B424B419E
:107BE000074A013393668022C9094000054B4018BB
:107BF00040010021C018120100F0B8F807BDC046CE
:107C0000002011509CD700207F220B0010B513409C
:107C100011420AD00022C9095B005B1803485B01CE
:107C2000C0180349C27000F0A1F810BD9CD7002015
:107C3000FFF7FFFFF0B50300828A008B041C90421F
:107C400000D9141CDD78A4B22800121B9A8280226D
:107C5000461EB041D20022434003104301226A4035
:107C6000DA705A78002A0BD1DD688E01AD191E69D1
:107C700094420FD11A6912191A618022120210431C
:107C80009B8A002B02D18023DB011843002900D0FE
:107C90000004F0BDB75CAF540132E9E7826803002D
:107CA00070B51268002900D0120C802424029005BF
:107CB00022405C78800D002C10D1002A05D0E821EC
:107CC000134B144A14481EF06BF8DA8A8218DA82D1
:107CD0001A8B824201D900229A8270BD002A04D1F7
:107CE000EE210E4B0B4A0C48EDE7DA68890151187A
:107CF00000221C69904206D1DA8A8218DA821A6957
:107D000012181A61E4E78D5CA5540132F2E7C0460F
:107D100028FB02107F2A031048FB0210D5FB02103B
:107D200080230A4A5B0410B51360094A09481360AE
:107D3000190002689143FBD18022074852011DF0CF
:107D40002BF90922054B5A6710BDC04600E00040E0
:107D500000F0004008C0004000001050000011502A
:107D600000238376036143617047000010B5836888
:107D7000002901D01C682140002A15D08024E4008D
:107D80001143224210D01A68224203D08178084859
:107D900019F07EFA074A0A401A60074B1B6C9B07D2
:107DA00002D40C23033BFDD28368196010BDC0468A
:107DB000F2FB0210FFFBFFFF00001150436870B59B
:107DC0000021802504001E68FFF734FF164B6D016B
:107DD0001A6C0543A37892071BD57F2213405A1EC5
:107DE0009341DBB2A28A002A18D0002B16D10121C0
:107DF0002000FFF71FFF0D4B05433340A026F6057B
:107E00001E4363682A001E6000212000FFF7AEFFBA
:107E100070BD0122DB099A431300E3E7044B1E40C7
:107E200080239B05ECE7C04600001150FFFFFFDFF9
:107E3000FFFFFFAF002310B5C38201338282837638
:107E40000161FFF7BBFF10BD70B5857E0400002DFA
:107E500003D181780D4819F01BFA836800211B6853
:107E6000FFF71CFF63681B685B0006D5238B83420A
:107E700003D101212000FFF711FFA38A002B03D0BB
:107E80002000FFF79BFF0025280070BD10FC0210AA
:107E9000F8B503780400DB070E00DD0F002B1DD1C1
:107EA00003785B07DF0F002B14DB01213000494210
:107EB00027F056F82378DB07DD0F002B0CD1237851
:107EC0005B0704D404230125227813432370300078
:107ED00026F0F6FF2800F8BD3D00F8E70025F9E799
:107EE00070B50D00012104004942280027F038F840
:107EF00023785B07DE0F002B06DA2378DB0708D434
:107F00000422237893432370280026F0D9FF300001
:107F100070BD0026F8E70000437902791B02134385
:107F2000C2785B0592075B0D920F022A0DD00020EC
:107F3000032A16D0012A07D102394A4251410C4A7C
:107F4000891899424041C0B27047022904D1094AB8
:107F5000981843425841F6E7002040229A42404197
:107F6000F1E740220229F9D18022D200F6E7C0468B
:107F7000FF03000000FEFFFF70B57F268A189142C4
:107F800000D370BD4C78052C06D18D782C00344080
:107F90006400ED09041963550C780919EFE710B571
:107FA00003689C6B0123A04710BD10B50368012135
:107FB0001B6B984710BDF8B505000F001600002494
:107FC000B44201D12000F8BD2B682800395D1B6840
:107FD00098470028F6D00134F2E70300027F002022
:107FE000824203D0FC33986ADB6AC01A7047036888
:107FF00010B51B6904009847002808D02200FC3205
:10800000D36A591CE418D1620334E07F10BD01200B
:108010004042FBE7036810B51B690400984700283D
:1080200006D02300FC33DB6AE4180334E07F10BD84
:1080300001204042FBE77047FC3041637047FC3051
:108040000163704710B50022012119F077F910BDC6
:1080500070B5FA240600002519F0CAFF6400241840
:108060004D4119F0C5FF8D4202D806D1844204D992
:10807000300018F0E9FE0028F3D0300018F0E4FEDC
:10808000431E9841C0B270BD037F002B09D0C37F4F
:10809000002B06D10200FC3281779362D362013358
:1080A000C377704710B5037F8161002B02D0006950
:1080B0001AF0BCFA10BD70B5057F0400002D1CD16C
:1080C0008169457700691AF007FB2A0020692900B9
:1080D0001AF02CFB0321207D19F00EF9207DFFF70B
:1080E000B1FF607D032119F007F9607DFFF7AAFF5A
:1080F0000123E5772377FC34A56270BD70B5037F5B
:1081000004000D00002B2ED10126816946770069FD
:108110001AF0E2FA2A00310020691AF007FB2369FD
:1081200011491A681163114A9D1A69424D4110495B
:108130001735934200D00F49280019F0E3F90121C7
:10814000280019F0AFF90321207D19F0D5F8207D22
:10815000FFF778FF0321607D19F0CEF8607DFFF70F
:1081600071FF0123237770BD64160000F05F0020CB
:108170003983001049830010F0B5FA25AD00856001
:108180000D4D00240560050001260127FE354460E1
:10819000023D76422C87EE632E644A36FF366C64CD
:1081A000AC6487552C654375044B0275016183618E
:1081B0000477C477AC62F0BD982A0310A086010052
:1081C00090B585B000AF78607B681B691B68DB6A7F
:1081D000FB60FB68002B00D1A9E0FB680422134080
:1081E0001ED07A6892235B00D358FF2B14DC7B6887
:1081F0001B691B681B69DCB27A6892235B00D35849
:10820000581C79689222520088507A682221D3182B
:108210005B18221C1A7003E07B681B691B681B69D2
:10822000FB68202213400ED07A6896235B00D35857
:10823000002B04D07A6896235B00D35898477B685C
:108240001B691B681B6DFB684022134003D07B68D1
:108250001B691B685B6DFA688023DB00134008D044
:108260007A689A235B000121D1547B681B691B68E3
:108270005B6EFA6880235B01134029D07A689823EB
:108280005B00D358002B0FD07A6892235B00D35841
:10829000002B09D07A6898235B00D3587968922222
:1082A00052008A58100098477A6892235B00002198
:1082B000D1507A6894235B000021D1507A689A23C8
:1082C0005B000021D1547B681B691B68A8229B5866
:1082D000FA6880239B0013402AD07A6898235B00B9
:1082E000D358002B0FD07A6892235B00D358002B11
:1082F00009D07A6898235B00D3587968922252009B
:108300008A58100098477A6892235B000021D15068
:108310007A6894235B000021D1507A689A235B002D
:108320000021D1547B681B691B681B6E00E0C046AE
:10833000BD4605B090BD000010B50248FFF740FFF4
:1083400010BDC046148E002010B50248FFF738FF5C
:1083500010BDC046C48C0020F7B50F0015001C00EE
:1083600002210190380018F0EDFC0221280018F0DD
:10837000E9FC0521280018F0BFFF0521380018F09E
:10838000BBFF0121380018F03DFD21004B481AF0D9
:108390004DFDC40F24186610E4173000210019F0B9
:1083A0009DFD2800012118F02DFD2800FFF750FE4B
:1083B000002827D1002301933000210019F08EFD01
:1083C0003800002118F01EFD3000210019F086FD54
:1083D0002800012118F016FD3000210019F07EFD63
:1083E0003800012118F00EFD3000210019F076FD53
:1083F0002800032118F080FF3800032118F07CFFCB
:108400000198FEBD0021380018F0FCFC300021006E
:1084100019F064FD0021280018F0F4FC3000210060
:1084200019F05CFD08230093019B38005B00019369
:10843000D9110123194018F0E5FC3000210019F092
:108440004DFD0121280018F0DDFC3000210019F05D
:1084500045FD2800FFF7FCFD0028ABD000212800D7
:1084600018F0D0FC0520002119F038FD009B013BDD
:108470000093002BD8D10121380018F0C3FC300044
:10848000210019F02BFD2800012118F0BBFC280069
:10849000FFF7DEFD002800D18CE7380018F0D4FC8F
:1084A000434258412100C3B23000019319F016FD38
:1084B0002800009918F0A6FC7EE7C04640420F0055
:1084C0000122431C70B50400DA77002911D003683B
:1084D000427F5B6A8669002A0CD0857F98472368B3
:1084E000310020009B6A98472368290020001B6AFE
:1084F000984770BD98470221207D18F023FC022187
:10850000607D18F01FFC0521607D18F0F5FE207DD0
:10851000052118F0F1FE207D18F096FC002817D1F7
:108520000925207D18F090FC011E1BD0207D18F03D
:108530008BFC050001280BD10021207D18F062FC86
:108540000520002119F0CAFC2900207D18F05AFCF2
:108550002368200031009B6A984723682000DB696C
:108560009847C6E7607D18F04DFC0520002119F002
:10857000B5FC0121607D18F045FC013D052000217E
:1085800019F0ACFC002DCCD1D0E70000F0B58BB0D9
:1085900008911F00037F04001600181E3ED0002023
:1085A000E57F85423AD1531E2800FF2B36D8236938
:1085B0000693A368079319F01BFD2300FA222233C8
:1085C00004900591099392000023290007981CF05C
:1085D000C1FC049A059B80185941002902DA012048
:1085E0000F49404201237B400290039100932500F4
:1085F0003300099A089906981AF0CDF8FC35030063
:10860000A862821C08D3023304D1A31C2000D97FA6
:10861000FFF756FF0020A8620023EB620BB0F0BD0D
:10862000FFFFFF7FF0B58BB00891037F04000420AB
:10863000002B14D0E37F002B11D023000025FC3346
:108640009E6AA77FE577AE420BD1A3693800627DB1
:10865000217DFFF781FE012358409840C0B20BB046
:10866000F0BD23690693A368079319F0C1FC2300AA
:10867000FA222233049005910993920000232900E5
:1086800007981CF067FC049A059B80185941002943
:1086900002DA01200F4940420123089A0290039117
:1086A0005340009339003300099A06981AF05AF89B
:1086B000831C06D1A31C2000D97FFFF701FF0520F2
:1086C000CDE70023FC34301AA362431E984180009A
:1086D000C5E7C046FFFFFF7FF7B5037F04000D002D
:1086E000002B32D0437F002B31D08368019319F0E7
:1086F0007FFCFA2206000F0000230021019892005F
:108700001CF028FC80197941002902DA012018495F
:1087100040420E002369174F1B685A6F102A09D177
:108720007A6A01929642F8D8BA6A824202D2019AD3
:108730009642F2D05A6F102A02D01D61012005E046
:10874000A31C2000D97FFFF7BBFE0020FEBDC37F26
:10875000002BFAD002008021FC32936A49008B4240
:10876000F3D0C418591C03349162E577E6E7C0469C
:10877000FFFFFF7F004005400022036910B51B6822
:1087800088331A6001231900C2774932FF328354BB
:10879000FC30026C9140054A1160C16B8B40136044
:1087A000036D002B00D0984710BDC0460434005024
:1087B000F8B5A025084C094FED052E593B6833420A
:1087C00005D0074B1868002801D0FFF7D5FF3B689C
:1087D00033402B51F8BDC0460C040000A88F002088
:1087E000B08F0020F8B5A025084C094FED052E5993
:1087F0003B68334205D0074B1868002801D0FFF7CB
:10880000BBFF3B6833402B51F8BDC0460C04000051
:10881000AC8F0020B48F0020F8B53627FF37C35D3A
:108820000500002B35D01E4A01690023914231D04A
:108830001C4A1D4913601D4A13602C000B20FC3498
:1088400018F04EFFE06B002807DB19F097FDE06B96
:1088500019F08AFD01235B42E363206C002807DBEB
:1088600019F08CFD206C19F07FFD01235B4223641D
:1088700000262B69606C1B6888331E6018F08EF828
:10888000A42301225B006664A664EE77EA542665A1
:10889000EE55F8BD064A07491360074A1360CCE756
:1088A000F05F0020A88F0020B1870010B08F00205B
:1088B000AC8F0020E5870010B48F002070B5040055
:1088C000FFF7AAFF237F002B21D0637F002B10D05E
:1088D00022690F4BD51A69424D410E4917359A420C
:1088E00000D00D49280018F0FBFE0021280018F0E8
:1088F000D9FD206919F08CFE0021207D18F022FAA4
:108900000021607D18F01EFA00232377E37770BD05
:10891000F05F0020398300104983001010B5052353
:10892000042205490548FFF727FC1B231A220449A6
:108930000448FFF721FC10BDF85F0020C48C002024
:10894000F05F0020148E0020002301730261036099
:1089500083604360704710B5017B04000B00403B0F
:1089600000200F2B0AD820690368DB6A984720692A
:1089700003685B6B984743425841C0B210BD10B5C5
:10898000040000690368DB6998472000FFF7E3FFF4
:1089900010BD70B504000D000069217B0368DB6A1F
:1089A00098472069290003681B6898472069036875
:1089B0005B6B9847206902220368217BDB6B984739
:1089C000206903685B699847050020692D020368E8
:1089D0005B699847284380B270BD000010B5022142
:1089E000FFF7D7FFC3070AD4C00880B21AF034FDDE
:1089F000044A054B1AF0B9FC1AF0C6FD10BD034835
:108A0000FCE7C046FCA9F1D24D62703F0000C8C22D
:108A100010B503210400FFF7BCFF142358431CF0DA
:108A200007F921681CF0A1F810BD10B5042104005D
:108A3000FFF7AFFF00B21CF0FBF821681CF095F8BF
:108A400010BD70B504000E0015000069217B03689D
:108A5000DB6A98472069310003681B6898472069E2
:108A6000290A03681B6898472069E9B203681B68F4
:108A70009847206903685B6B984770BD70B5040028
:108A80000020202911D81025A94200D96D190021F4
:108A90002000FFF77EFF0200202D07D0064B1A4072
:108AA00000212000FFF7CDFF012070BD80239B0136
:108AB0001A4392B2F4E7C046FFDF0000F8B50400A5
:108AC000081C151C0E1C1CF013F9184B184A1AF040
:108AD00097FC00230700984226D1281C1CF008F9B7
:108AE000124B134A1AF08CFC3B0000281CD1E021E9
:108AF000301C89051CF039F8291C2060A6606560CF
:108B00001CF033F81CF0F4F80B00020009490A4885
:108B10001AF00DFC1AF0CEFF1AF0DAFC052182B231
:108B20002000FFF78EFF01231800F8BD4D62503F73
:108B3000FCA9F1D2B5F8A43FF168E388704710B5FD
:108B4000040004211CF066FC200010BD014B024A09
:108B50001A607047C8890020E82A0310064B10B538
:108B6000040003604068002804D0A368002B01D1F2
:108B700000F004FB200010BDF82A031010B504001B
:108B8000FFF7ECFF20000C211CF044FC200010BD7E
:108B9000406870B50E00041E0AD000F01BFB0500F3
:108BA0000100300017F03BFA0400280000F018FB29
:108BB000200070BD034B044A1A6000225A609A607C
:108BC0007047C046307D0120F82A031070B5041E9E
:108BD00008D00068002805D0A568401922F084FA62
:108BE0002D18A56070BD000070B504000E000028AF
:108BF0001AD00068002817D06368002B02D0A26842
:108C0000934211D9002E0FDBA2680136B618B34289
:108C100001D3801870BD2369002B05D18023DB05AB
:108C20009E4203D3002E0FDA0020F3E77600236A7A
:108C3000002B0BD031009847051E17D1E36920683F
:108C4000984765602560EFE70B4EF0E73000A369B9
:108C500098472168051E02D10800E369F0E7A26881
:108C600001321CF09FF9E36920689847A0686660AC
:108C700025602818CEE7C046FFFFFF7FF7B5050047
:108C8000081E01D10020FEBD00272C00BD4222D0CD
:108C900001239C463D492378002B26D1641BE4190F
:108CA000E11CFFF7A1FF0028ECD0631CC318009360
:108CB000A31CC3180193461C2223002F2BD1037041
:108CC0002200290030001CF06DF92223009A137055
:108CD000019B1F7007E00321FFF786FF0028D1D01A
:108CE0002B4923F021F90120CDE7222B0ED8072BA9
:108CF0000AD91A000E00083AD2B2D64032006646AF
:108D0000324205D11F2B04D8053702E05C2B00D17D
:108D100001370134BFE75C2403702B78002B05D1A9
:108D2000222200990A70019A1370DCE71F2B07D9E1
:108D3000222B05D05C2B03D0337001350136ECE7D4
:108D400034702A78731C0D2A0ED8072A10D9100007
:108D5000083805280CD826F03BF90317130B11151A
:108D6000622272701E00E8E7222AFAD05C2AF8D04C
:108D7000180008491CF042FF0536DEE76622F0E7DE
:108D80006E22EEE77222ECE77422EAE73700000475
:108D900038FC02103BFC0210F0B506000C008DB050
:108DA000002802D100200DB0F0BD0029FAD0C5681E
:108DB000EDB2102D00D1C2E008DC681E0728F1D802
:108DC00026F0FEF8363EF02BF0F0F046402D00D1B4
:108DD000E1E0802D00D19FE0202DE3D186680121C4
:108DE0002000FFF701FF0028DCD05B230370A3689D
:108DF0000133A360E3680133E360002E00D0A2E0FA
:108E000002212000FFF7F0FE0028CBD05D23467042
:108E10000370E368013BE36008E005212000FFF7F1
:108E2000E3FEA9490028BDD023F07EF80120BAE76F
:108E300006212000FFF7D8FE0028B3D0A349F3E7AE
:108E400005212000FFF7D0FEA1490028ECD1A9E7B9
:108E50001A22F769B669002105A81CF09DF80022C6
:108E60000023300002920393390032003B001AF0D5
:108E7000E2FA002815D101227B005B0801930096DD
:108E8000944B5242009801991AF0D5FA00281ED14D
:108E90000098019901228F4B52421AF0B7FA00282C
:108EA00015D1894905A823F03FF804252000691C45
:108EB000FFF79AFE002800D174E7002305AAAB4211
:108EC00026D10022C254A268D318A360AEE73200B4
:108ED00081493B0005A81CF091FE8049050002AACB
:108EE00005A81FF043FB012807D1029A039B30001D
:108EF00039001AF07DFA002806D132003B0078498B
:108F000005A81CF07BFE0500192D00D94AE7CDE726
:108F1000995CC1540133D2E70069002800D141E7D0
:108F200022F0E2F8451C29002000FFF75DFE002832
:108F300000D137E72A0031691CF034F876E7006980
:108F4000FFF79CFE2FE721003000FFF725FF0028E8
:108F500000D127E72000FFF739FE3368002B15D03A
:108F6000616920004B1E99414F1C0231FFF73CFE06
:108F7000002800D116E72C2303706369002B07D16A
:108F8000431C00221A70A368DB19A360366834E71B
:108F9000831C4570F5E7496985684B1E994120009F
:108FA0004F1C0231FFF720FE002800D1FAE67B2398
:108FB0000370E3680133E3606369002B01D00A2387
:108FC0004370A368DB190927A3606369002D1BD1D7
:108FD0000221002B01D0E16801312000FFF704FEDF
:108FE000002800D1DEE66369002B08D005000300ED
:108FF0000926E2681800013A591B914260D37D238B
:1090000003700023437004E7002B0DD02000E168BB
:10901000FFF7EAFD002800D1C4E60023E26893428E
:109020004BD3A3689B18A3602100286AFFF726FE94
:10903000002800D1B6E62000FFF7C8FD66692000D1
:10904000731E9E4101363100FFF7CEFD002800D18E
:10905000A8E63A2303706369002B00D04770A36829
:1090600021009B192800A360FFF796FE002800D17D
:1090700098E62000FFF7AAFD2E682000731E9E418F
:1090800063695A1E9341F618711CFFF7ADFD002865
:1090900000D187E62B68002B02D02C23037001300F
:1090A0006369002B02D00A23037001300023037090
:1090B000A3682D689B19A36087E7C7540133ADE708
:1090C0001E70013395E7C04641FC021046FC0210B9
:1090D0004CFC0210FFFFEF7F51FC021058FC021005
:1090E0005CFC0210F0B580278DB003AD0E00242289
:1090F0000021019028001BF04FFF1F4C7F0038001B
:1091000023689847220003906F606E6109ABC2CA62
:10911000C2C3002811D029000198FFF73DFE0028A6
:109120000BD02800FFF752FDA968A3680131002B7E
:109130000AD003989847061E1BD10398002801D037
:1091400063689847002614E008002368984703994D
:10915000061EF2D0AA686B6801329A4200D91A0042
:1091600030001BF01FFF0022AB68F25463680398C5
:10917000984730000DB0F0BD90090020F8B580266A
:1091800004007600002C00D1F8BDE3682768104D7C
:10919000334205D1A068002811D12069002814D1DC
:1091A0008022E3689200134204D1206A002801D093
:1091B0006B68984720006B6898473C00E2E7FFF730
:1091C000DDFFE3683342E8D0EAE76B689847E7E7FA
:1091D0009009002010B50021FFF784FF10BD0000AA
:1091E00010B5024B5B68984710BDC046900900203F
:1091F000F0B51D002F4B0F00C118090D063189B0C5
:109200000400C9B22800160018F076F801233900CE
:109210002A000093200019F0AFFB80235B02049327
:10922000F31CF2011B031343234AAD0213400593C1
:10923000F823DB011D4080239B052B4307931F4B25
:109240000520069318F0A2FF1BF0EDFC1C49051C3D
:109250000E981BF08AFC011C281C1BF072FCEC21F0
:1092600089051BF06BFC03901BF036FD85B20020D6
:1092700085420DD028001BF0D6FC011C03981BF082
:109280005AFC8721C9051BF070FC1BF025FDC0B2FC
:109290002D04000228433200049004AB3900200062
:1092A00019F0BAFB0123BB4022681343236009B0C5
:1092B000F0BDC0460000E0AFFFFFFF9F000006507A
:1092C0000000204110B504000623C05E002807DB23
:1092D0000121C0B217F036FD0021A07917F092FDF0
:1092E0000123637010BD70B50500C0680E0017F053
:1092F00055FB2B7CEC7CE41A631E9C4103347443C5
:10930000A4B22000AC8017F021FBE860002805D053
:10931000220000211BF040FE6E8070BD0600A88078
:10932000FAE70322F8B58B090D098F08174013409F
:1093300015400A4047748274FF2700228F42524131
:109340000270C268C47C067CC3740574002A0AD00B
:10935000A21B5B1B51424A4159424B419A4202D0E7
:109360004188FFF7C0FFF8BD73B504000D008069A8
:109370000849160019F0E6FAE1690200A069002E1A
:1093800005D0054B00932B00FFF732FF73BD034B55
:10939000F8E7C046042B0310005043490050C3486F
:1093A000F7B51E00471C08AB15001A78FB7F0400B8
:1093B000002B03D0FFF7D8FF0023FB772A00AE195C
:1093C0000125B24200D1F7BDE16913780F001B06F9
:1093D00001932B001037BB409C46A0696346476849
:1093E0003B42FBD1019B043189000B500132E8E77D
:1093F000C36837B50400002B1AD096256D0017F00E
:109400000AF96369984201D26061F8E7C01AA8427C
:10941000F5D317F049FD2278A388A17900922000A6
:10942000E268FFF7BDFF17F01DFD17F0F4F860616B
:1094300037BD70B5437805000C00002B07D006231C
:10944000C05E002803DB0021C0B217F07BFC6B7804
:10945000EC80002B08D0E4B20121200017F072FC50
:109460000021200017F0CEFC70BD0000F7B50025EC
:109470000127040000911900124B461C83614570BE
:109480000572C5604561C561F7770192FFF749FF35
:1094900020000099FFF727FF20000199FFF7C9FF7F
:1094A0002900A06919F012FAE061A84205DA06481D
:1094B0003900A06119F00AFAE06101232000F37776
:1094C000FEBDC0460000205000003050F0B505AC95
:1094D000257844888C4216D9047A002C05D0624342
:1094E00063436543120A1B0A2D0AC47C077CC668C5
:1094F000A74209D1032461437118047C0A55427CB8
:109500008B54837CCD54F0BD8900711800260E5514
:10951000F3E74388F7B58B4219D9037A150C140A7F
:10952000002B15D1E4B2EDB20194D6B2B446047C5E
:10953000C67CC768B44217D103234B43FF18037C92
:10954000019AFD54437CFA546246837CFA54F7BD79
:10955000FF26344035405C4316405D435E43240A99
:109560002D0A0194360AE1E789007F18120E002BBC
:1095700002D1D3B2BB55E2E753431B0AFAE7F7B572
:109580004288030000208A4220D9DF7C1D7CD868F5
:109590001C7A5A7C9E7CAF421DD10323594341184B
:1095A0008D5CC85D8E5D2D02002C10D02100000264
:1095B00019F064FC21000704280019F05FFC000288
:1095C00007432100300219F059FC3843FEBD000466
:1095D00028433043FAE789004118C85D8F5C4D5D30
:1095E0008E5D3F02002C18D02100000219F046FCCD
:1095F000210003062802019319F040FC019B210081
:10960000050430021D4319F039FC210005433800E0
:1096100019F034FC00022843D8E7000638433043F1
:109620002D04F8E710B500218288C0681BF0B4FC57
:1096300010BD0023036101338382837570470000EE
:1096400010B50400FF20A3610023000620600D4830
:109650002170A0600C486270FF39FF3AA370E0618E
:109660004B42594153425A41802001230A432373FC
:109670004000FE33206222712000E381FFF7D9FF12
:10968000200010BD0024F40000093D0070B5040066
:109690000800A170012117F055FB0121A07817F0F7
:1096A000B1FBA36801261A0A62771A0CA27700227E
:1096B00023771B0EE377631CDA77A31CDE7725790B
:1096C000954208D0A06903685B6B9847A06903685E
:1096D0001B6B984770BD3100207817F033FB3100C9
:1096E000607817F02FFB2900207817F08BFB2900FA
:1096F000607817F087FBEDE7C08970474A1E0300CA
:109700000020012A01D8197501307047F7B50F0004
:109710000824802503784678019329000198394070
:1097200017F070FB0121300017F06CFB013C0021A9
:10973000300017F067FB6D08002CEED12000FEBD55
:1097400070B504000D008078002117F05BFB2379D1
:109750002E0AEDB2002B18D0A069226A0368E169D5
:109760001B6A9847A069310003689B689847A06905
:10977000290003689B689847A06903685B6A98475B
:109780000121A07817F03EFB70BD31002000FFF7EB
:10979000BDFF29002000FFF7B9FFF1E770B50D000C
:1097A000017B0023914220D9C489291CA54200D9FC
:1097B000211C130008335B0089B21D52012A16D008
:1097C00080235B018025427DED0152422A401343F4
:1097D000027D012A02D18022920113430A4A944257
:1097E00008D11943FFF7ACFF0123180070BD902387
:1097F0001B02E7E7054A944203D18900194389B265
:10980000F0E70901FAE7C046FF0F0000FF03000080
:10981000C02310B59B011943FFF792FF10BDB02381
:1098200010B51B021943FFF78BFF10BD10B50400E4
:10983000FFF706FF02232373014B2000E38110BDD5
:10984000FF0F0000F0B51D0089B00EAB00241C5FB7
:109850000FAB1B886F1A0593A31A16000190009294
:10986000F817DA179B183F185340474002930397A5
:109870000398029FA4462A000B00874205DC3300B0
:1098800022000E002C0019006546A64208DC1800D4
:109890001300020028000D00010020003400060023
:1098A0009B1ADA179B185340301B079303B2DA0F49
:1098B000D3185B100093012387B2069704938D425F
:1098C00001DB023B0493B44201DD09B0F0BD019B12
:1098D000039A1B689B691F00029B934216DD2200BE
:1098E0002900059B0198B847009A079BD31A19B223
:1098F0009AB200911B0406D5049BED18069B2DB26D
:109900009A1813B20093013424B2DCE72A00210034
:10991000059BE7E7704710B504682469A04710BDB0
:1099200037B506AC258804680095A46BA04737BD01
:1099300037B506AC258804680095E46BA04737BDB1
:1099400073B506AC0025655F07AC268804680196F0
:109950000095246CA04773BDF0B5160004000D00FF
:1099600085B003930AAB1F8803685B699847039B24
:109970002268013B9B191BB2009301972B00290021
:109980002000976A3200B84723682000DB6A9847B6
:1099900005B0F0BDF0B505001C000E00170085B045
:1099A0000AAB1B88013C039303685B6998470399E2
:1099B0002A68A3190191009731002800946A1BB20C
:1099C0003A00A0472B682800DB6A984705B0F0BD35
:1099D000F0B50E0087B003930CAB029200229B5EA1
:1099E000040004930DAB1B883500059303685B6985
:1099F0009847039A2368B218954204DB2000DB6A7B
:109A0000984707B0F0BD059A290000921F6A200010
:109A1000049B029A0135B8472DB2EAE713B50191CC
:109A20000E24015F0C22835E02680091146C0022F8
:109A30001100A04713BDF0B50400150087B00493D2
:109A40000CAB00229B5E039105930DAB1E8803684F
:109A50005B699847236800962A0020005F6A039993
:109A6000049BB847059B20005A1E23685219009694
:109A70005F6A0399049B12B2B847236800962A00D4
:109A800020001F6A0399059BB8470499039B01397D
:109A9000C918236800962A0020001E6A09B2059B97
:109AA000B04723682000DB6A984707B0F0BD7047D5
:109AB000F0B585B01E000AAB0027DF5F0BAB1B883B
:109AC00014000500026802910393B14210D1BC4218
:109AD00002DC3B0027001C00039901340091E31BCA
:109AE000966B28003A0002991BB2B04705B0F0BD52
:109AF000BC4211D1029BB34202DC3300029E0293AE
:109B0000029B0399013300919B1BD76B310022000C
:109B100028001BB2B847E9E753699847039A2B68B6
:109B20000192009728009F6A220033000299B847EB
:109B30002B682800DB6A9847D8E703230B4010B551
:109B400083760822835E0A24025FC90702D41900C3
:109B500013000A008281C38110BD000010B542814C
:109B6000C281012200235242054C4261054A4360F2
:109B7000046001818181036182610377036210BD0A
:109B80001C2B031001010001F0B595B01D001AABAC
:109B90001B88039204931BAB1E881CAB1F781DAB64
:109BA0001B78026A040008910293002A00D0BAE0F0
:109BB0000C22835E8B427ADD0E22835E039A9342EF
:109BC00075DD06237B435B18002B70DD029B039A37
:109BD000DB009B18002B6ADD037F002B03D1AF2D28
:109BE00001D90135EDB2236820005B699847052350
:109BF0005D430B9300230693904B5B190E93069ADB
:109C00000E9B9B5C0A936B461B8B09936B461B8CCC
:109C10000593099B059A7B43D3181BB20D93082328
:109C20000C930023079301220A9B2068134250D013
:109C30006B469A8B9989012F3BD1029B012B38D11E
:109C4000099B5218059985695918049B12B209B2EB
:109C50002000A847079B01335BB207930A9B5B0870
:109C60000A930C9B013BDBB20C93002BDBD1069BD0
:109C700001335BB206930B9B013BDBB20B93002BD2
:109C8000BDD1049BB3420ED02068012F3CD1029B72
:109C9000012B39D1059900960531056A039A2000F8
:109CA00009B20733A84723682000DB6A984715B03C
:109CB000F0BD029D3BB26A438A18049912B2019129
:109CC00069460825495F0091C5690D992000A8479C
:109CD000C0E7049BB342BDD06B469A8B9989012F94
:109CE0000BD1029B012B08D1099B5218059985695C
:109CF000591812B2330009B2AAE7029D3BB26A4377
:109D00008A1812B20196DBE705227A43059901967B
:109D10008A1811B2029A3BB2D2000092C569039A26
:109D20002000A847BFE7137A5168ED1A1268EDB218
:109D3000ED0011924A5B4B1907929A780D92DA78EE
:109D4000129205229A569B790E925BB20F930023D2
:109D50000C930B93029B3B43012B02D90F9B0B925D
:109D60000C93236820005B69984700231E00099329
:109D70000693129B9E4200D395E76B469B89029AFD
:109D80000A930C9BF31853430A9AD31800221BB270
:109D900010930592099B32E05A1CD2B2139207220B
:109DA000134207D1079B0799119A0133525C9BB26A
:109DB000069207936B461B7E5BB2002B16DA6B464E
:109DC0002068198C012F26D1029B012B23D10A9BDD
:109DD0000F9A9A180E9BB218C918059B12B25918FF
:109DE000836909B21D002000049BA847069B059DBE
:109DF0005B00DBB201350693EBB20593139B0D9A22
:109E000005999142C8D39446099B01366344DBB25D
:109E10000993F6B2ADE7059D0B9A3BB252197A430E
:109E20008918049A09B201926A460825525F009285
:109E3000C26920001500109AA847D7E76C2B0310C1
:109E4000F0B5026A04000B0085B0002A34D10A295B
:109E500008D1437E0282DB00628A9B186382012064
:109E600005B0F0BD0D29FAD0E17E007E657E0029A7
:109E70000ED01026A15F0626464389190C27E65FFF
:109E8000B14205DD1226A15F2282EA0052186282E9
:109E90001221625E1026A15F03950290E08A019074
:109EA000A08A00902000FFF76FFE0622237E534316
:109EB000228A9B182382D2E70A2905D10023038234
:109EC000127B437E5343C7E70D29C8D0117A8B42DA
:109ED000C5D3907A9842C2D3591A5568C9B2C900FD
:109EE0006D18AF78002F28D0E978002925D0E17EC1
:109EF000207E667E002913D005216956C919414389
:109F00008C461021675EBC440C21675EBC4507DDB2
:109F10001227E15F00272782127B72435218628268
:109F20001221625E1027E15F03960290E08A0190A1
:109F3000A08A00902000FFF727FE2B79227EB6E74B
:109F4000F0B500291BDB0C25445F8C4217DD002A8D
:109F500015DB0E25445F944211DD847E022C0FD068
:109F6000032C16D0012C04D10489A41A013C0A0048
:109F700021B2012B13D0022B31D0002B1FD0F0BD0A
:109F80000489013C611A448909B2A21A013A12B249
:109F9000EFE74489013C641A110022B2E9E7072582
:109FA000D4172C401540AB400827C65FA418E41016
:109FB0007443C06A6118425C13434354DFE70724CB
:109FC000D31723409B1814400122A2400826855F26
:109FD000DB106B43C06A5918435C9343EDE70724D9
:109FE000D31723400826855F9B18DB106B435B1853
:109FF0000121224091400A00C06AC15C4A40C2541B
:10A00000BDE7000070B5002604001D0004AB9E579C
:10A01000FFF7A4FD114B2360002363629D4200D132
:10A020000F4DE3622300FF223333A5621A70220032
:10A03000012336325B42A3861370230037331E7030
:10A04000059B8022A363069B5200E363054B20001F
:10A050006364230048331A8070BDC0467430031017
:10A06000C48C002000093D00836AF7B504000D0090
:10A070000200002B14D0303211781A681800D26A0E
:10A080009047A06A002103681B689847A06A2900CE
:10A0900003681B689847A06A03685B6B9847F7BD25
:10A0A00035321078190016F0ADFE606A002804D031
:10A0B000036829009B689847F1E70827802623005A
:10A0C000310033331878294016F09CFE23003433D6
:10A0D00001931878012116F095FE019B0021187854
:10A0E000013F16F08FFE7608002FE8D1D7E770B554
:10A0F0000400806A0D00002810D00368A16B9B6AE1
:10A1000098475A3D2000E9B2FFF7AEFFA06A002849
:10A1100013D00368E16B9B6A984770BD606A0028A2
:10A1200004D00368616C1B6AA26C98472300363325
:10A130000021187816F066FEE3E72300363318781E
:10A14000012116F05FFE606A0028E6D003685B6AB2
:10A150009847E2E770B504AC2588002A21DB0A267F
:10A16000845F94421DDD002902DA5B1800211BB2D6
:10A170000826845F5E18A64201DD631A1BB2002B1D
:10A180000FDDD61074436418C16A072002400638F8
:10A1900090400919C2B2012D08D0022D1AD0002D0D
:10A1A00009D070BD0878104308700131013B1BB223
:10A1B000581CF7D1F5E7D243D2B2013B1BB2581C71
:10A1C000EFD00878104008700131F6E70878504069
:10A1D00008700131013B1BB2581CF7D1E1E70000C8
:10A1E000F0B505AC2488002950DB0826855FA9421C
:10A1F0004CDA002A02DA9B1800221BB20A27C65F3B
:10A20000D718B74201DDB61A33B2002B3EDDD2B209
:10A21000D60875436D18C16A072649191500DBB2C7
:10A220003540324215D00822551B2B4AEDB2525D03
:10A23000AB4203D2EF1AF8363E413240012C26D011
:10A24000022C2CD0002C26D0AB421FD30826825FD4
:10A2500089185B1BDBB2072B0ED9022C22D11A0006
:10A260000D78083AED430D700826855FD2B2491982
:10A27000072AF5D807221340002B07D0174AD35CD2
:10A28000012C1ED0022C24D0002C1ED0F0BD0E7844
:10A2900032430A70D8E70E7896430E70D4E70E78F2
:10A2A0007240F6E725006A1E95411A006D42EDB234
:10A2B0000D700827C65F083AD2B28919072AF7D865
:10A2C000D8E70A7813430B70E0E70A789A430A70DC
:10A2D000DCE70A785340F6E7CC300310C4300310B3
:10A2E00037B5140006AA1588827E022A0DD0032AEB
:10A2F00018D0012A11D10289121B013A14B20A00A6
:10A3000000952100FFF76CFF37BD4289C918121B69
:10A31000013A14B20289511A09B222000095FFF7DE
:10A3200019FFF1E74289C918511A09B2E7E737B5B1
:10A33000140006AA1588827E022A0DD0032A18D09E
:10A34000012A11D10289E418141B24B20A000095D5
:10A350002100FFF7FFFE37BD0289E418521A013AC7
:10A3600011B24289141B24B222000095FFF738FF76
:10A37000F1E74289521A013A11B2E7E710B5040039
:10A380004068002801D01BF049F8082120001BF08C
:10A3900041F810BDF8B5040016F086FD2378002BB7
:10A3A00019D00027606A277017F0E8FF606A1B4E1B
:10A3B00083009F5117F0D8FF194DA06A2B68013B0D
:10A3C0002B6017F0DBFFA06A83009F5117F0CCFFD2
:10A3D0002B68013B2B6016F045FD206963689842AD
:10A3E00001D0FFF7CBFF60696368984201D0FFF7A7
:10A3F000C5FFA068002807D1E068002809D160687F
:10A40000FFF7BCFF2000F8BD0568FFF7B7FFA560A8
:10A41000EFE70568FFF7B2FFE560EDE7688F002022
:10A42000A48F0020F7B5057804000E00002D02D19E
:10A4300000252800FEBD831CDB7F002BF8D1030024
:10A4400008330193019B1B68002B05D1002AEFD034
:10A45000019B1B68002BFBD0019B1B685968236C78
:10A460005A1C9B005F58A36922649A4209D1019843
:10A4700024F036FD010020000C3024F0C9FD00233B
:10A4800023643760D5E7821CD27F0300002A0CD0FA
:10A49000C2681978081E07D0101E05D09969186C7B
:10A4A0001368081A002B02D170478268F1E71B6815
:10A4B0004018F7E7030084B010330193043302938C
:10A4C0000C3B0393039B1B68002B08D0029A436844
:10A4D00012689A4203D0019A12689342F2D104B0F2
:10A4E00070470120404270470120404270470020E1
:10A4F000704700008022064B520019681142FCD0C0
:10A50000802252009968114200D07047D968F9E75B
:10A5100000C0044070B5431CDB7F0400002B0CD04E
:10A52000050028352B78002B05D103685B69984717
:10A530000123E0622B70E06A70BD01204042FBE71E
:10A5400010B5431CDB7F0400002B1AD00300283316
:10A550001A78002A03D00022C06A1A7010BD436B1B
:10A56000002B06DC01000122806B3031FFF75AFF1F
:10A570002023226B103B1005120C000D2263636335
:10A58000ECE701204042E9E710B5431CDB7F002BDC
:10A5900002D0806BFFF78EFF10BD421C030000202D
:10A5A00010B5D27F824202D0986BFFF76CFF10BDCE
:10A5B000F0B5060085B0019300230AA807780BA820
:10A5C00005780CA804780DA800789C4602900EA887
:10A5D00000780390701CC07F984243D11A39C9B2E9
:10A5E000032901D8214840561A3AD2B20021032A41
:10A5F00001D81E498956019B01431A3BDAB2002358
:10A60000032A01D8194B9B561A3FFFB21943002366
:10A61000032F01D8154BDB571A3DEDB200220B4337
:10A62000032D01D8114A52571A3CE4B213430022B9
:10A63000032C01D80D4A12571343029A00211A3AEB
:10A64000D2B2032A01D809498956039A0B431A3A10
:10A65000D2B20021032A01D8044989560B43336141
:10A6600001239C46604605B0F0BDC046D4300310BF
:10A67000F0B58BB00793FA23040013AD2E7814AD18
:10A680002F78002510A800789B00089011A8A360DF
:10A6900000780F4B09902360631C65602563656338
:10A6A000DD77099B12A800780193089B0290009324
:10A6B0002000079B04970396FFF77AFF054B2000C5
:10A6C00063610823A5636562A361E5610BB0F0BD1A
:10A6D000E030031080BB000070B5431CDA7F04003B
:10A6E000002A0DD00022856BDA77954206D028002B
:10A6F000FFF750FE442128001AF08CFE0023A363CC
:10A700000822024B1A60FFF7F5FE70BD00F004400E
:10A7100010B50400024B0360FFF7DEFF200010BD00
:10A72000E030031010B50400FFF7F2FF20003C21D9
:10A730001AF070FE200010BD002070474160704785
:10A7400041607047012070470120704741607047A9
:10A7500010B50368DB6A984710BD000010B5094AC0
:10A760000C680300002094420AD11A00F8321278D3
:10A77000824205D1DC33180005221AF013FC0120B7
:10A7800010BDC0465454494C027F0300101E00D037
:10A790005869704798225200825C0300101E01D055
:10A7A00030331800704798225200825C0300101E5C
:10A7B00000D0D86A7047982252000300805C0028BD
:10A7C00005D028331878013843425841C0B2704749
:10A7D000982252000300805C002805D028331878A6
:10A7E000023843425841C0B270470020704770475A
:10A7F000C06810B5002802D003685B68984710BD98
:10A800000020704770477047704770477047704727
:10A81000704700207047030010B5DB680C301B68E0
:10A82000984710BD030010B51B6910301B6898478E
:10A8300010BD10B5037F002B06D0C168002903D0DE
:10A840008068083004F07CFE10BD0000074B0C301F
:10A8500010B50400994206D008001BF07DF8431E95
:10A86000984140420440200010BDC0468832031089
:10A87000074B103010B50400994206D008001BF0B9
:10A880006BF8431E984140420440200010BDC04672
:10A8900088320310074B0C3010B50400994206D0E3
:10A8A00008001BF059F8431E984140420440200024
:10A8B00010BDC04688320310074B0C3010B50400A1
:10A8C000994206D008001BF047F8431E98414042C9
:10A8D0000440200010BDC0468832031010B50400AB
:10A8E00060211AF097FD200010BD10B50400102162
:10A8F0001AF090FD200010BD10B5FFF7F6FF10BD57
:10A90000A02110B5040049001AF084FD200010BDFC
:10A9100010B5040040211AF07DFD200010BD10B5D7
:10A92000040040211AF076FD200010BD10B504008F
:10A9300010211AF06FFD200010BD10B510211AF083
:10A9400069FD10BD10B560211AF064FD10BD10B591
:10A9500040211AF05FFD10BD10B540211AF05AFDDC
:10A9600010BDA02110B549001AF054FD10BD10B55E
:10A970000400F8342378002B04D0083004F07CFB6A
:10A980000023237010BD0000064B10B503600300C8
:10A99000F8331B780400002B02D0083004F06CFB65
:10A9A000200010BD0C31031010B50400FFF7ECFFC0
:10A9B0002000FC211AF02EFD200010BD982300225B
:10A9C00030B504005B00C3B0C2544069A1690830CF
:10A9D00005F06EF8050060696A46A169083005F067
:10A9E00023F860696A466B425D41A169083005F051
:10A9F0001BF8E8B243B030BDF8B504000669270083
:10AA00000023220030373B7060692832A16908308A
:10AA100005F00AF8431E5A4253419822520005009D
:10AA2000A3540120002E07D032003800A1681EF088
:10AA30008FFC43425841C0B2012D02D10028DED024
:10AA4000F8BD0020FCE70000082330B50F4D87B0AB
:10AA5000083000936322290004AB040004F0EAFCF0
:10AA6000082804D1049B0599180007B030BD0423C1
:10AA700029000093632203AB200004F0DBFC0023D9
:10AA800019000428F0D1039BEEE7C04663FC0210D6
:10AA900030B50024002585B002940395037F0100A2
:10AAA000002B0FD0C368002B0CD0082380680093C4
:10AAB00063224969083002AB04F0BCFC082801D0CD
:10AAC000029403950298039905B030BD30B5002477
:10AAD000002585B002940395037F0100002B0FD061
:10AAE000C368002B0CD00823806800937422496946
:10AAF000083002AB04F09EFC082801D002940395B4
:10AB00000298039905B030BD30B5037FC3B0002B68
:10AB100003D10023180043B030BDC268002AF9D029
:10AB2000036884681B6B9847083401006A4620005C
:10AB30006D4604F05BFC0028EBD12B78023B5A42B7
:10AB40005341DBB2E6E730B5037FC3B0002B02D13F
:10AB5000002043B030BDC368002BF9D0036884687F
:10AB60001B6B9847083401006A4620006D4604F0CC
:10AB70003DFC0028ECD12878013843425841C0B24E
:10AB8000E7E710B5037F1C1E0AD044692F2120007F
:10AB900021F044FA002803D04378002B00D0441C55
:10ABA000200010BD10B50300007F0A00002808D067
:10ABB000D968081E05D09868083004F053FDC043DA
:10ABC000C00F10BD10B5037F002B01D1002010BDB8
:10ABD000C1680029FAD08068083004F0E5FD00283B
:10ABE000F5DAF3E7F7B5077F04000D001600002F34
:10ABF00002D100273800FEBDC368002BF9D0022A1D
:10AC000000D14D42236820009B6998470190A068BD
:10AC100033002A00E168083004F004FD0028E8DB76
:10AC2000236820009B69984723680500DB692000A2
:10AC300098478542DED92368002220005B6901998C
:10AC40009847D6E770B51300027F04000D00101E70
:10AC50000CD0E16800290AD0002D08D0A0682A0095
:10AC6000083004F089FCC343DB17184070BD002096
:10AC7000FCE710B51300027F0C00002A01D1002070
:10AC800010BDC1680029FAD0002CF8D080682200DD
:10AC9000083004F0A7FC0028F2DAF0E710B50468E9
:10ACA0002000F0342468E4304C430168A4181800F4
:10ACB000029A09191AF076F9002010BD030070B548
:10ACC000F8331E7805000C00002E02D1002630005B
:10ACD00070BD0029FAD00B78002BF7D0083528007A
:10ACE00004F0D0F90028F1D120001CF0FBFC041E78
:10ACF000EDD02F21200021F091F9002803D1200070
:10AD000015F04CFEE3E7002321000370280004F057
:10AD1000B9F9EEE710B50300F8300078002811D03B
:10AD2000081E0FD00C78201E0CD0101E0AD0002058
:10AD30001478844206D00833180004F017FA43420E
:10AD40005841C0B210BD10B500201BF0C3F810BDB3
:10AD50000300F0B5F8331B78C7B006000D001400EF
:10AD60000293002B04D100230293029847B0F0BD58
:10AD70000029F8D00B78002BF5D0030004AF08337E
:10AD80003A001800039304F031FB0028EBDB33009A
:10AD9000F0331B68397863608B1E58424341059A33
:10ADA0002376022900D10022082322600093230089
:10ADB000632229000398083304F03CFB082803D0E1
:10ADC00000220023A260E360A268E368226163615D
:10ADD000CBE700B5C3B06A46083004F007FB434236
:10ADE0005841C0B243B000BD030010B5F8331B7822
:10ADF000002B08D00B1E06D000230A789A4202D0FE
:10AE0000FFF7E7FF0300180010BD0300F0B5F833AB
:10AE1000060018780D0085B000281DD0081E1BD034
:10AE200000200B78834217D037000837380004F031
:10AE3000F1FC041E0DD17368002B0AD0984708233B
:10AE400002900391009363222900380002AB04F0C2
:10AE50002BFB63425C41E0B205B0F0BDF8B50300E6
:10AE6000F8331D780C00002D1AD00700F0373B682E
:10AE700000260B610300EC331B684B610300F433C5
:10AE80001B688B61FF23CB610300E8331B6808302C
:10AE90000B604E6004F018FE3B68E6604343A3601D
:10AEA0002800F8BD10B50300027F0020824206D0C2
:10AEB000D968814203D09868083004F08DFC10BD39
:10AEC0001FB5037F0400002B29D0C168002926D0BC
:10AED0008068083004F018FB002323776368002B98
:10AEE0001DD0236A9B071AD5A36AE26A134309D0CF
:10AEF0000823A06800932300632261690830283387
:10AF000004F0D2FA63689847082302900391A0687E
:10AF1000009374226169083002AB04F0C5FA1FBDCA
:10AF2000C06810B5002801D01AF078FA10BD0000F2
:10AF3000037870B5002B05D0094B1D78002D02D089
:10AF400000E000BF70BD043024F06AF8054C0648EC
:10AF500025701AF047F82378002BFCD0F2E7C046A2
:10AF600066830120678301202ED0DEC0037810B5F0
:10AF7000002B0BD0043023F0A3FF0022044B1A70E7
:10AF8000044B1B78934201D000E000BF10BDC046C7
:10AF90006783012066830120F8B51D000368114E08
:10AFA0001C00F0331868E434484324683378801870
:10AFB0002418002B01D115F077FF0B4F3800FFF755
:10AFC000B7FFF0231B06E0182900069A23F098FF2C
:10AFD0003800FFF7CBFF3378002B01D115F042FF8B
:10AFE0000020F8BD6683012090690020F8B505684F
:10AFF000104E2A00F0352B68E4324B431468E418F5
:10B000003378002B01D115F04FFF0B4F3800FFF7BD
:10B010008FFFF0231B06E018296823F099FF380002
:10B02000FFF7A4FF3378002B01D115F01BFF0020A0
:10B03000F8BDC046668301209069002070B5050008
:10B040000600F8352B7804000836002B04D03000B9
:10B0500004F012F800232B7000218022300019F038
:10B060009BFF21003000883103F04AFF002801D106
:10B0700001232B70287870BD0300F0B5E8331B68FE
:10B08000040087B0002B45D007000500F8373E7854
:10B090000835002E04D0280003F0EEFF00233B709B
:10B0A00000218022280019F077FF21002800883134
:10B0B00003F0AEFE00282DD16368002B23D02000C2
:10B0C000FFF7BCFF00281ED0636898470827134B82
:10B0D000049005910393632228000399009704AB21
:10B0E00004F0E2F9002815D1009774222800039992
:10B0F00004AB04F0D9F9071E0CD1280003F0BCFF03
:10B100002300F8331F700120002E04D02000FFF729
:10B1100095FF00E0002007B0F0BDC04663FC0210C0
:10B12000030070B5F8331D780400002D02D001250E
:10B13000280070BD0300E8331B68002BF8D0FFF730
:10B140007DFF0028F3D12300E0331B78002BEFD0E4
:10B15000236820005B6998470028E9D02000FFF7AA
:10B160006DFF0500E4E70000F0B587B002AFBB60FB
:10B1700098233960FA605B000500C05C002837D076
:10B18000101E35D0B868002832D02C6A261E03D095
:10B1900020001FF0A9FF06002B00303318007B6051
:10B1A0001FF0A2FF6B468019C11C0A30C008C00006
:10B1B0001B1A9D4602AE002C1DD022780F4B002A90
:10B1C00000D00F4B78680F4A0190009330002300A5
:10B1D00020F076FFFB6868690093BB6831003A682D
:10B1E000083004F027F9FB68181A43425841C0B2EE
:10B1F000BD4605B0F0BD014C2300E3E7210B031071
:10B2000063FC021065FC02101FB50822632102AB2B
:10B210000400FFF7A9FF002803D00298039904B0A7
:10B2200010BD63210422200001ABFFF79DFF011E2A
:10B23000F5D00198C117F2E71FB50822742102ABBF
:10B240000400FFF791FF002803D00298039904B08F
:10B2500010BD74210422200001ABFFF785FF011E01
:10B26000F5D00198C117F2E770B504680500002C0D
:10B2700011D06368013B6360002B0CD12368200070
:10B280009B689847A368013BA360002B03D1236808
:10B290002000DB689847280070BD000010B5094BFE
:10B2A00004000360037F002B01D0FFF709FE20009C
:10B2B0001830FFF7D9FF20001030FFF7D5FF20002E
:10B2C00010BDC0466031031010B50400FFF7E6FF63
:10B2D000200030211AF09EF8200010BD0D4B10B553
:10B2E00003603223FF33C35C0400002B04D04069A9
:10B2F000A169083004F088FB20002430FFF7B4FF78
:10B3000020001C30FFF7B0FF2000083015F074F863
:10B31000200010BDB031031010B50400FFF7DEFFB0
:10B320009A21200049001AF075F8200010BD000095
:10B33000F0B589B002AF3B6098237A605B00CB5CCC
:10B3400005000E00002B05D1036043602800BD46B8
:10B3500007B0F0BD0C6ABC60002C03D020001FF0C9
:10B36000C3FEB860330030331800FB601FF0BCFE32
:10B37000BB68C0186B46C11C0A30C008C0001B1A4D
:10B380009D4602ABBB60002C23D02278124B002AD2
:10B3900000D0124BF868009301902300104AB8685F
:10B3A00020F08EFE102371693A68FC180B68009239
:10B3B0002000DE69BA687B68B0473B6962682B6031
:10B3C000002363603B6114336A60F818FFF74CFF99
:10B3D000BCE7014C2300DDE7210B031063FC0210E6
:10B3E00065FC02100B680360002B02D05A68013222
:10B3F0005A607047F0B587B08160190000250400DD
:10B40000012708C901921A4A45600260C3601030E2
:10B41000FFF7E8FF0C9B0198236265610E9A0F9B72
:10B42000A561A262E36227771FF05EFEC0191AF0E1
:10B430000BF80600102019F0F5FF0E4B4760036073
:10B44000636987600493A369C660A061666105A80B
:10B45000059303950295FFF707FF03A8FFF704FF85
:10B460000199606920F060FD200007B0F0BDC04682
:10B4700060310310E8310310F0B591B01E0016AB37
:10B480001F780B0006910592F8331B780400002BFF
:10B4900004D123606360200011B0F0BD059B002B38
:10B4A00003D01B78002B00D08AE00023F1E7451B76
:10B4B000FE2DFADC451C2B78002B0AD02F2128000A
:10B4C0001AF022FD0028F2D128001FF00DFEFE2800
:10B4D000EBD80123334009931B02B20702D5802227
:10B4E00012011343760702D58022D20013430122B2
:10B4F0003A401A43022308921F4201D01A4308928D
:10B50000602019F08FFF0123436083605B4B0500CF
:10B51000036003000C33180054220021079319F034
:10B520003BFD079B0D950C93099B002B0DD02F2104
:10B5300005981AF0E9FC002807D005981CF0D2F80D
:10B54000061E3FD1300015F029FA069B5B68002BE0
:10B5500002D0099B002B4AD1002309930A93069D30
:10B56000089B08352800059A079903F0A9FF0300F6
:10B570000700153350D1402019F054FF0123070074
:10B5800000260500436083603D4B10370360099B34
:10B59000380002930A9B059A0393089B069900932F
:10B5A0000EAB0E960F96FFF725FF27600F9665608E
:10B5B0000E960FA8FFF758FE0DA8FFF755FE6AE795
:10B5C000059D78E72F211AF09FFC2F270500002DFD
:10B5D000B8D0002306982B703100083004F01AF917
:10B5E0002F70681C2F211AF08FFC0500EFE7069DD5
:10B5F000012308352800059A079903F061FF002808
:10B6000004D12800079903F07FFFA5E7069B5B683C
:10B61000984709900A91A2E700282BD107992800A2
:10B6200003F08EFF402019F0FDFE0123436083608C
:10B63000134B05000360030010330B93079B0DA908
:10B640000FA80E93FFF7CEFE099B0EAE02930A9B46
:10B65000059A0393089B069900930B983300FFF714
:10B66000C9FE0FA8FFF700FE0B9B0F9723606560D4
:10B670000E979EE70023236063609DE7043203106A
:10B68000203203100B00F0B5744CF833A54402913E
:10B690001B7806001000002B01D0002A07D10023E0
:10B6A00033607360300095239B009D44F0BD1CF017
:10B6B00019F8002405002B78002B25D1402019F023
:10B6C000B1FE012343608360654B04000360030007
:10B6D0000C33180034220021019319F05DFC019B0A
:10B6E00006940593029C2B780834002B16D010AFDB
:10B6F0003A002900200003F079FE002820DB3B7887
:10B70000022B1DD12A000AE028001FF0EDFC0138B1
:10B710002B5C2A182F2BD1D11470CCE7514A200072
:10B72000019904F019F9504F00281FDA280015F08C
:10B7300035F900233360736006A8FFF795FDB1E784
:10B740002F21280020F06AFC071E06D12000454A60
:10B75000019904F001F92F00E6E7002303702A00A5
:10B760002000019904F0F8F80137DDE7019952AAA9
:10B77000200004F059F952AA0199200004F054F96C
:10B78000A020400019F04EFE0123040043608360B6
:10B79000364B390003600DA814F07CFE019A06A90F
:10B7A00008A800270792FFF71DFE22002000304B5B
:10B7B0000C32E3600DA927611430039214F08DFE62
:10B7C0002000029A08A92262019A28306262FFF7DB
:10B7D00009FE2200FE3213008022200052003900B0
:10B7E000E76227633430DA87083219F0D5FB280086
:10B7F0001FF07AFC013019F027FE0190102019F09B
:10B8000011FE0123436083601A4B0A970360019B7A
:10B810000997C360E36A0B93019BE362236B206388
:10B820000CA80C93FFF720FD0AA8FFF71DFD2900C7
:10B83000E06A20F079FB08A8FFF716FD0DA814F0C8
:10B84000DBFD280015F0AAF8039B746033600EA896
:10B850000E970D97FFF708FD6EE7C046ACFDFFFFA2
:10B860003C32031063FC0210210B0310583203100A
:10B87000B0310310E8310310F0B5FC2085B019F0A9
:10B88000D1FD2C4A2C4B00269B1A01932B4B466072
:10B8900003600300DC339A60019A2949DA6080254D
:10B8A000802201271960102104006D0052011F71D0
:10B8B0001D615A6199611E7731008022083019F0AC
:10B8C0006BFB200031002422B83019F065FB230007
:10B8D0001C4A88335A601C4A1C609A601B4A5D618E
:10B8E000DA601B4A9D611A6180225201DA612200EE
:10B8F000019BA8321B0B136023001021AC3319608D
:10B900005D609D600800029419F08CFD114B124D92
:10B91000476087600360C460039003A90F482C60F0
:10B92000FFF760FD0E4B03A8AB60FFF79DFC05B071
:10B93000F0BDC04600F0F71000F0FF100C3103100E
:10B940005454494C9DAC001099AF0010EDAF00105D
:10B95000EBA7001074320310CC890020D08900209E
:10B9600047AD0010026803000120013204D058687E
:10B97000013043425841C0B2704710B50A680468AC
:10B9800003000020944208D05B6849688B4204D0D1
:10B990008C4202D0D01A431E984110BD020080058F
:10B9A000801501304142484180188005800D0430E7
:10B9B0007047002310B5C258CC586240C2500433BF
:10B9C0000C2BF8D110BD030002680020824207D181
:10B9D00059681000002903D1986843425841C0B209
:10B9E000704710B5E0240268E400120D00232242E3
:10B9F00004D00430FFF7C1FF012343400120184069
:10BA000010BD82B0019001AB002801D102B0704797
:10BA10001B688B4201D01868F6E70120F6E710B5E5
:10BA200004000800E16E636D0818C01A17F026FACA
:10BA3000A36D8B4208D90723CA081940063B8B40E7
:10BA4000606E815C0B438354002010BD80235B0536
:10BA50000B405A425341184A5B421340174A30B5D3
:10BA60009B18026814004C4023420BD093059B1591
:10BA7000013307D0124D114C124B15400C402B4393
:10BA80009C4203D100230360012030BDE0248025C7
:10BA90000B0DE400ED001C40AC4205D1140309037A
:10BAA000A40D890D8C4201D20020EEE75BB29B020F
:10BAB0009B180360F8E7C046000010F000FCFF7F11
:10BAC00000FC0F000000F04F10B504000800FFF765
:10BAD00065FF23681B182360002010BD0368013335
:10BAE0000360002070470000F0B589B00F9F0793F6
:10BAF000119B1600FA18836E0290DB6903919A423B
:10BB000005D8C36E002B29D00E9A934226D8542014
:10BB10004042BFE0039B002B47D01B680E9A119C4C
:10BB2000934225D1039B59689B68CB18BB421FD910
:10BB3000B94218D8DC1B119B9C4200D91C00039B06
:10BB4000791ADB6822005918109819F02BFA109B0B
:10BB50003F191B191093119B1B1B1193119B002B59
:10BB6000D8D1180096E0119BCC1B9C4200D91C0038
:10BB700033680E9A93421ED17168B5684D19BD4263
:10BB800019D9B94213D8ED1BA54200D92500F36895
:10BB9000791A59182A00109819F004FA109B7F1985
:10BBA0005B191093119B5B1BD7E7119CE0E7C91B46
:10BBB0008C4200D90C00119B079A934228D3029B18
:10BBC00038009B6E5D690493290017F057F900292E
:10BBD0001ED1119B9D421BD82900200017F04EF961
:10BBE000631A00930593049B06915B683A001D005D
:10BBF0000E99109B0498A84700284BD1109B059ADA
:10BC00009B181093069BBF181C1B119B1B19A4E7C4
:10BC1000029BDB6E002B08D00E9A934205D86B2155
:10BC20001D4B1E4A1E481AF0BBF80E9B38003360AD
:10BC3000029B9D6E6B691900049317F01FF97B1A24
:10BC400006937360079B05915C1E049BE418E4193E
:10BC50001900200017F012F9EB69641A9C4200D910
:10BC60001C00059BDA1BAB6AA4189C4200D91C007F
:10BC7000B460009428006C68F368069A0E99A04797
:10BC8000002804DD7621074B044A0548CBE700284D
:10BC900000D13FE709B0F0BD6CFC0210073403107F
:10BCA0009AFC021004FD0210F0B50E698BB01D0065
:10BCB000CB6805903C300F00079206930996FFF77A
:10BCC00090FE041E14D0079B1C03A40D10D0059BEE
:10BCD000DC6B2B032403A40D9B0D9C4204D1022199
:10BCE000494208000BB0F0BD9C42A441A40AA40242
:10BCF0003000FFF753FE069A031D9342EFD8069BD0
:10BD0000059A1B1A06930423039309AB0293069B1F
:10BD1000002101933B68100000930423FFF7E4FE29
:10BD2000011EDED1099B079A1BBA73405B005B08BA
:10BD300012030993920D18D0E0208021320DC0002B
:10BD4000C9001040884210D1281B0103890D8C4680
:10BD50003103890D8C4508D319490840194901431D
:10BD6000B142BCD052B2920214192A1B07997240F8
:10BD7000114222D1B505AB150133B0D0129BAD0DE8
:10BD80009D4200D91D00119B069A0293109B0395BA
:10BD900004339B1801933B68059A0021009310001F
:10BDA0002B00FFF7A1FE011E9BD1129B5A1B119B7A
:10BDB000581919F0F1F8A11993E71E0098E7C04649
:10BDC00000FC0F00000010401FB59C05A40D02945C
:10BDD000069C019400240094FFF766FF04B010BD98
:10BDE00030B587B003AD1400084B094A0095FFF742
:10BDF000EBFF002804DA831C00D1002007B030BD1F
:10BE000029002000FFF7D5FDF7E7C0460C00F07FC2
:10BE10000000F07F70B508250400006886B00100BE
:10BE2000836E039504AD0295566810310196126831
:10BE30000092DB690200FFF757FE002803D12800BB
:10BE4000211DFFF79AFD06B070BD000070B5084EC9
:10BE5000040031001CF0D6FB3100050020181CF056
:10BE6000F5FB2418605D43425841C0B270BDC04626
:10BE700063FC0210F0B51C0006002000194B0F00F7
:10BE800085B008309A4207D1174920F04DF80223B7
:10BE90002370002005B0F0BD336F95020133009090
:10BEA000124A30002B43FFF78FFF0028F2DB104BC4
:10BEB000000D2B4302AD2070390030000D4A009573
:10BEC000FFF782FF0028E5DB0B4A030D934202D106
:10BED000039B6360DDE7094A9342DAD18005800D58
:10BEE0006060D6E7FF03000063FC021000FC0F78DF
:10BEF0000800002000FC0F70020200000102000098
:10BF0000C36E10B58B4206D88A21084B084A0948EF
:10BF1000490019F045FF806EC3689847002804DD8A
:10BF20008B21054B024A0348F2E710BDC302031000
:10BF3000E23303109AFC021004FD0210F0B5002752
:10BF4000B1B0069339AB1B88150007933AAB1B8839
:10BF50000C900B933BAB00229B5E099108220021C1
:10BF600010A808933E0019F017F80698FFF716FD81
:10BF700043190593099B059ADB689A4239D2042339
:10BF800003930FAB0293099B01921B680C9A0093D9
:10BF9000002104231000FFF7A7FD002800D01AE1BC
:10BFA0000F9B069A1BBA5A401300802212061A43AE
:10BFB0001400099B06921B680F921093059B043393
:10BFC000119310AB0A933300389A634013401D005D
:10BFD000824A154013424AD1389B1B039B0D00D166
:10BFE0009EE0022F16D97E4B7E4A7F487F4919F08A
:10BFF000D7FE379B002B00DCEBE0369B05951C68D9
:10C000005B680F940A93369B08333693379B013B4A
:10C010003793D8E73C227A43099B059912A813501D
:10C020008318596006999E6199603699DC62D960DF
:10C0300037992C32196138990137596107999983D9
:10C040000B99D983089919843C9959623D99996251
:10C050000A99196310A9343350C950C32E008318AC
:10C060003D933895624B08953C930B950795059D3C
:10C070007BE78122520093421FD100250A9C0F9931
:10C080008A05920D9542F2D2C022089B0903890DC0
:10C09000C918A36889021943237892009B181B05CD
:10C0A000194362683D983C9B9847002800DA92E06B
:10C0B0000C340028DBD10135E1E7089B0A9A99028C
:10C0C0003D983C9B09199847002800DA83E0CED0C0
:10C0D000002F00D17FE03C22013F7A4312ABD158C0
:10C0E0009B185A68099105929A68DC6A0692DA6888
:10C0F0009E6936921A690F9437925A6938929A8BD0
:10C100000792DA8B0B9220215A5E08925A6A3C926F
:10C110009A6A3D921A6B34330A9210AA21CB21C23B
:10C12000389B1B039B0D07D0079A23039B0D93425B
:10C130009DD30B9A93429AD263005B0D97D0022253
:10C14000FF32934295D12A4B3C9A9A428FD03C229F
:10C1500013007B430D930D9912AB5D18280000214D
:10C1600018F01AFF20210AAB5B180D9A0999AE61ED
:10C170009950059B80266B60069B0137AB60369B10
:10C18000B605EB60379B2B61389B6B61079BAB83DC
:10C190000B9BEB83089B2B843C9B6B623D9BAB62B0
:10C1A000A3059B0D079301330B932403079BA40D59
:10C1B000E41A089B1C1923B208930A9B09930D4BA0
:10C1C0003893002337933693013B0693002305935E
:10C1D0004DE700207CE731B0F0BDC0460000F07FA5
:10C1E0000DFD02108C3303109AFC0210C5030000F1
:10C1F0004DBA001000FC0F60F0B58BB0119E099392
:10C20000139B1500F218836E0700DB6908919A42B0
:10C2100021D9542040424EE0EB6805932B6802334D
:10C220001ED16968AC680C19A64219D28E4217D388
:10C23000139BA41B9C4200D91C00059B711A591822
:10C240002200129818F0AEFE129B36191B19129399
:10C25000139B1B1B1393139B002BDDD118002AE0AB
:10C2600002235B422B60BB6E300006935B691900B2
:10C27000049316F003FE731A07936B60099B5C1E10
:10C28000049BE418A4191900200016F0F7FD069B82
:10C29000641A9B6A9C4200D91C00059BAC60019308
:10C2A000079B38000093054A109B08990294FFF7FA
:10C2B000FBFC0028B0DA0BB0F0BDC04600FCF7FF75
:10C2C000F0B5160000248BB0059006910793119BE2
:10C2D000A34202D800200BB0F0BD119B1D1B082DFE
:10C2E00000D90825109A08AFA2180192079A0021D8
:10C2F00000920598069A331B03950297FFF7F4FB0B
:10C300000028E8D1129B2A001868390003F0E0FBEE
:10C31000129B64191860DAE7F0B59BB00F93C36EF7
:10C3200007000D001600002B09D01268934203D8B5
:10C3300054235B4205936CE072689342F8D9002164
:10C34000042412AB03940293019133683A000093E2
:10C350003800230012911391FFF7C6FB031E0590CE
:10C3600001D0543355D10394002413AB02930194AC
:10C3700073683A000093210004233800FFF7B4FBF0
:10C3800003000590A04247D0543342D1A3009A59EC
:10C390002A6001225440A20092590A946A6012AAAB
:10C3A0009B58AB600023EB6002330D93033B059376
:10C3B000BF4B14AA11CB11C229000120042208315D
:10C3C000404203F085FB00230C930B930893013B41
:10C3D00009930023059E109007930998FFF7DEFA52
:10C3E0000422079B00211B180793BB6E039211AA1E
:10C3F0000292079A380001922A680092DB693A009B
:10C40000FFF772FB041E0ED02300543300D12AE143
:10C41000059405981BB0F0BD139B129A9B1ADC176C
:10C42000E41AE40FB2E70422109811A903F050FBBC
:10C43000119B099A1BBA5A401090069211921DD571
:10C44000099B1E0DF023DB001E409A4BF618734229
:10C450005E41F6B2EC68002C00D006E12B686A68F9
:10C460006B600A9B2A609B0012AA9B58AB600D9BD5
:10C47000012B00D15CE701230D9399E70698FFF7A4
:10C480008DFABB6EDA69079BC318934200D9EAE0C4
:10C490002B6807990E93A023DB009C46F023043100
:10C4A00009910699DB00090D1940614539D1042332
:10C4B0000393099B18A901930E9B029100932100FD
:10C4C000130038003A00FFF70FFB041E9CD1189AA6
:10C4D000109B9A4200D0C6E0119B069A1B0DDB0709
:10C4E0005A40069210A90422F86A03F0F1FAF862A1
:10C4F0001198FFF753FA079BC018069BE8602B6161
:10C50000089BAB82149BAB61159BEB610B9BEB759E
:10C5100001235B4210933300069A059609921E0090
:10C520005BE7099B10A90438029101900093390040
:10C5300038000E9BFFF7C4FE041E00D064E7E02025
:10C54000C00084466146119B1A0D0E9210400A42AB
:10C5500021D1089A1B039B0D9A4201D801330893FD
:10C560001199209B0F9A4B401A400E920F9A1A4233
:10C570000ED12B6818AA1893099B23985360229B0D
:10C580009847041E00DA3FE71199002857D10E00A2
:10C590003300059EC0E78021C90088421DD13821A3
:10C5A0006A4652181278089952B2891889B24248DC
:10C5B00008914249304001438B4203D180231B063E
:10C5C0001E43CDE7711CCBD01B0331039B0D890D9E
:10C5D0008B42C5D892029619C2E7C0212B68C900C8
:10C5E000884214D101220E99380011400B91082184
:10C5F000BA6E039114A90291099900930191D3692C
:10C6000021003A00FFF770FA041EA9D0FCE62C497D
:10C610005205520D8A42A3D10821BA6E039116A980
:10C620000291099900930191D36921003A003800E1
:10C63000FFF75AFA543016D001230C9390E73300D9
:10C64000204A4B4013420BD00228A1D132030B03E6
:10C65000920D9B0D9A429BD3802636060E4397E798
:10C660000126764294E70026F4E60023AB759E424D
:10C6700030D0BE6E2000B16916F000FC002929D12F
:10C680000C9B002B26D001235B42189318AB02931E
:10C69000169B00940193390038002B68F269FFF76C
:10C6A0000FFE002810D0030054330DD00590B0E6E3
:10C6B0002834031000FBFFFF00FC0F000000F04FC8
:10C6C000FF05000000FCFF7F189A179B9B1A5A4237
:10C6D0005341AB75380029003C30FFF782F9002840
:10C6E0001AD0FB6B059A1B0312039B0D920D9A4205
:10C6F00008D18023059A1B061A430592219B002B23
:10C700000DD119E005990131F8D09A4204D9104AA7
:10C71000059B944663440593219B002B08D0059B01
:10C72000AA8A1B039B0D934200D91300219A138000
:10C73000059B002B00DB6CE60021059BAA8A1B03EE
:10C740009B0D05919A4200D863E60223F1E5C046AD
:10C7500000FCFFFF1FB5012300245B4203940294F9
:10C7600001940093FFF7D8FD04B010BDF0B593B06D
:10C770000C93036A15688B61436A0F00CB612B78B9
:10C7800006900A92002B00D18FE04A4C63005B0DAB
:10C790000993022B04D1280047491BF057FF2D189D
:10C7A000280045491BF02EFF0490012806D12B7864
:10C7B0002E2B0ED16B1C0793079DE7E7049B022BE2
:10C7C00007D11A0028003D491BF0E6FD002800D1E2
:10C7D0006BE0049BEB181E00079301230593364B77
:10C7E0000B93364B0D9330000B991BF02FFF36182F
:10C7F00030000B991BF006FF089000281CD0012880
:10C8000005D133782E2B13D1089BF618EBE7089B44
:10C81000022B0DD1022230000D991BF0BDFD002826
:10C8200006D1059B013B0593002BEDD1B31CC2E75C
:10C83000059B01330593E7E72B78002B32D00A9B49
:10C840001D60099B022B33D11D4B2403A40D9C4278
:10C850000CD03A001B4BA40218322343009239003B
:10C86000194A0698FFF7B0FA041E1BDB0FAB069AB5
:10C870000393164B0F920293049A0C9B119201930F
:10C880000092F0233A0039000698DB051832109523
:10C89000FFF742FD041E05DB00288DD1FB7D002B38
:10C8A000E4D1023C200013B0F0BD16246442F9E745
:10C8B0001424FBE700FC2F0063FC021014FD02109F
:10C8C000FF0300000800002000FC0F7031C90010B9
:10C8D000F0B5160000248BB0059006910793129BCB
:10C8E000A34201D800201FE0129B1D1B082D00D978
:10C8F0000825109A08AFA2180192079A0021009209
:10C900000598069A331B03950297FFF7EDF8002868
:10C910000AD1119B2A00380019191BF03DFD00288F
:10C9200004D0C043C00F01300BB0F0BD6419D6E78E
:10C9300030B505001300AA688C05006885B0A40D09
:10C94000A24200D9220002926968019159680091BF
:10C950001B680100FFF7BCFF002805D1AB68A342AC
:10C9600002D0A3424041013005B030BD036B10B589
:10C970009A05940D002A07D1002910DA0D4B0E4AB2
:10C980000E480F4919F00CFAFF225200944206D9C2
:10C99000002904DD0B4B084A08480B49F2E7C91887
:10C9A0008B055A1E934149004908DB070B4303637B
:10C9B00010BDC04617FD0210B63303109AFC0210DA
:10C9C0001C1300004DFD02101D130000836E10B5F6
:10C9D0005B6B0400002B02D1C06813F0DFFFA36E75
:10C9E0009B6B002B02D1E06913F0D8FFA36EDB6BC9
:10C9F000002B02D1606E13F0D1FF10BDF8B5C769EE
:10CA00000D68083F0E000020BD4215D339002800F4
:10CA100016F034FA013816F003FA023080003900BB
:10CA2000281A16F02BFA040016F0FAF980002D1AD5
:10CA300020006743ED1B3560F8BDF0B58BB00600F4
:10CA400006910792002B08D10122119952420A60E7
:10CA50000020129A13600BB0F0BD846E013B09A94F
:10CA600020000993FFF7CAFF10A905002000FFF777
:10CA7000C5FF0590059B079FAB4203D3119B1F6029
:10CA8000109BE5E7059BE81A16F0BEF904002800A4
:10CA900016F0C0F91F231C1B844200D90400042394
:10CAA000039307AB0293A3000193002104233000FA
:10CAB000069A0097FFF718F80028CCD10123A3406D
:10CAC000ED1AD7E7F0B589B00C0006924A6BC96A37
:10CAD000060000208A4227D28A1A05929A4200D97B
:10CAE0000593059F002F01D105981DE08023206B41
:10CAF000DB02184204D0B36EE26BDB699A421ED1AE
:10CB000080225203636B104210D1220021003C327C
:10CB10000292043A019200933000E36AA26A403123
:10CB2000FFF78BFF002805D009B0F0BD022252426A
:10CB3000A263E3638023206BDB0218432063B36EA0
:10CB4000E26BDB6994469D1ABD4200D93D0080210D
:10CB50004903014007918021220049034032039597
:10CB600008421AD00699029161460191A0881049A5
:10CB7000800201430091210030000831FFF73CFBA7
:10CB80000028D1D1636B7F1B5B196363E36B5B1977
:10CB9000E363069B5B190693A4E70699029161463D
:10CBA0000191A06B079900903000FEF79DFFE7E729
:10CBB00000001020F0B58DB0059000201D00129BE4
:10CBC00006910792834236D0013B0993059B09A940
:10CBD000986EFFF713FF0127040029001498139B98
:10CBE0009847002827D1002C25D023003B400493F0
:10CBF0000223049A0AAE9B1A9B000190079A069999
:10CC00000598039302960095FEF76EFF002812D157
:10CC10003D00A543A84205DB049BAD00023C7559CD
:10CC2000E418DAE7139B316814989847030038003A
:10CC3000002BEFD018000DB0F0BD10B50C00826ACB
:10CC4000FF21E06818F0A8F901235B42236010BDC2
:10CC5000F0B50B6A85B0C3664B6804000D008166B1
:10CC6000002B05D1A74BA84AA848A94919F098F864
:10CC70008B68002B04D1A74BA34AA448A649F5E72B
:10CC8000CB68002B04D1A54B9F4AA048A449EDE7EF
:10CC90000B69002B04D1A34B9B4A9C48A249E5E7B2
:10CCA0004B690293002B04D1A04B974A9748A049A7
:10CCB000DCE78B690393002B04D19E4B924A934887
:10CCC0009D49D3E78E6A002E04D19C4B8E4A8F4833
:10CCD0009B49CBE73000029916F0D0F8002904D028
:10CCE000984B894A89489849C0E73000039916F063
:10CCF000C5F8002904D0954B834A84489449B5E788
:10CD0000EB6931001800009316F0B8F80F1E04D03C
:10CD1000904B7D4A7D489049A8E7009B7F2B04D823
:10CD20008E4B794A79488E49A0E76B6A002B04D173
:10CD30008C4B754A75488C4998E72B6B002B13D0A8
:10CD4000009A5208934204D2884B6F4A6F48884930
:10CD50008CE75A1C08D0009A9A4205D28521854B4F
:10CD6000694A6A48490181E7EB6C0193002B20D0A6
:10CD70001800029916F082F8002904D07E4B624A0E
:10CD800062487E4972E70399019816F077F8002906
:10CD900004D07B4B5C4A5D487A4967E7019900986B
:10CDA00016F06CF8002904D0774B574A574877495A
:10CDB0005CE76B6B002B16D0E360AB6B002B1ED0D7
:10CDC000E36128002100FFF738FF2100A06E103139
:10CDD000FFF733FFA56EE86A002817D16C4B4A4A6B
:10CDE0004A486C4942E7300013F0B0FDE06000288B
:10CDF000E3D12000FFF7EAFD0C2040427FE0300045
:10CE000013F0A4FDE0610028DBD1F2E7EB6B002B0F
:10CE100008D063662B6CFF2B0AD95F4B3A4A3B481C
:10CE20005E4923E713F092FD60660028F2D1E0E747
:10CE3000002B00D1FF3323676B6C002B04DA584BB7
:10CE4000314A3248574911E7002B00D1564B6367EE
:10CE5000AA6C564B9A4204D98721554B2A4A2B4833
:10CE600080E7002A00D11A00A267EE6CEB699E42AF
:10CE700004D9504B244A25484F49F7E6286D411CF8
:10CE800022D0A96A884204D94C4B1F4A1F484C49FA
:10CE9000ECE6904204D94B4B1B4A1C484A49E5E654
:10CEA000DB08002E00D0F308984204D9474B164AFD
:10CEB00016484749DAE6071E06D1914200D911000B
:10CEC0000F00994200D91F000123002520005B427A
:10CED000236263620C222900E767A562E5623C30A9
:10CEE00018F05AF820000C222900303018F054F8BD
:10CEF00020000C222900483018F04EF8280005B018
:10CF0000F0BDC04683FD0210133403109AFC0210DA
:10CF100078100000A1FD02107A100000BFFD021081
:10CF20007B100000DEFD02107C100000FCFD0210F2
:10CF30008110000015FE0210821000002EFE02106B
:10CF40008310000048FE02108710000078FE0210D7
:10CF500088100000A8FE021089100000D9FE0210FF
:10CF60008C100000F5FE02109810000011FF021056
:10CF70009E10000065FF0210C4FF0210A510000003
:10CF800011000310A71000005E000310A91000009C
:10CF9000AC000310C8100000C9000310D41000003A
:10CFA000E3000310DA100000FFFFFF7FFE03000024
:10CFB000040103101F010310E61000004E010310CE
:10CFC000E8100000A5010310EA100000F5010310AD
:10CFD000EC100000F0B589B007930B6807000C0057
:10CFE00006920593033302D9002009B0F0BDC36E49
:10CFF000059A9A4205D3B3211E4B1F4A1F4818F0C9
:10D00000CFFE866EA568B1694D19013D280015F067
:10D0100035FF6D1A0095B36830009C46626866461D
:10D02000E3680599B047002804DDB721144B124A84
:10D030001248E4E70028D8D1079B002B04D1210037
:10D04000B86EFFF7FAFDCFE70123069A5B42136043
:10D050000295E3682A00019363683800009323680F
:10D060000699FFF735FC0028BFDBE8D0542040428A
:10D07000BBE7C04684020310C93303109AFC0210B8
:10D0800004FD0210F7B50193089B06000C00099FF0
:10D090000092023309D0C36E089A934205D8E82162
:10D0A0002D4B2E4A2E4818F07BFEB26E0B9BD26998
:10D0B000FB18934248D9E9212A4B284A2848F2E72D
:10D0C000013305D08321284B244A25484900EAE74B
:10D0D000089B38002360B36E996915F0CFFE791A6A
:10D0E0006160A5602368089A9342E9D16068B842FC
:10D0F000E8D8B36E9D6A4519BD42E3D90B9BED1B81
:10D100009D4200D91D00E368381A2A0018180A99B0
:10D1100017F048FF0A9BA2685B190A930B9B7F19C3
:10D120005B1B0B936368FB1A934200D21300B26E31
:10D13000A360926A9A4207D121003000019B009AB5
:10D14000FFF748FF002805D10B9B002B01D00025DD
:10D15000C8E70B98FEBDC046A5020310D6330310E6
:10D160009AFC0210DC020310FF020310F0B50C0061
:10D17000010085B0029203931D00636816000193BD
:10D1800023680200009310310023FFF77BFF071E86
:10D1900008D12A003100E06802F09AFC6368E06080
:10D1A0005B196360380005B0F0BDF0B50C008BB0C2
:10D1B0000490100017000693FEF7F0FB63686269A5
:10D1C000C3180590934245D87B005B080793079AE4
:10D1D000A368210053401BBA09930498042309AAA9
:10D1E000FFF7C4FF051E0DD1059B1E1F002F0CDB92
:10D1F00033002100069A0498FFF7B8FF002827D1D2
:10D20000079BA36028000BB0F0BD002EF8D00123CF
:10D210001327039304ABFF18069B02975B68059ADC
:10D22000043B9B189B1B0193069B049A1B680021DF
:10D23000009310003300FEF757FC002808D10123AB
:10D240003A0021000498FFF791FF013E0028DCD04E
:10D250000500D7E71C256D42D4E710B513000A007E
:10D2600003C8FFF7A2FF10BD01235B4210B5136096
:10D2700000230400FFF7AEFE00280AD1A06E036968
:10D280009847002805DDDD21024B034A034818F0CA
:10D2900087FD10BD04FD0210803303109AFC0210BC
:10D2A000F0B50D00826E6B689169D2691433040089
:10D2B0008DB0934200D913004F1EDF19380015F0CE
:10D2C000DDFD00237F1A069304936B68BB421AD3DB
:10D2D00001222B6904995242C91A0A920AAE049A91
:10D2E000019102960093210020002B680432FEF782
:10D2F000E7FF00284AD10A9B069A934200D1A6E094
:10D300005420404242E004225242D61A594AF619A9
:10D31000964200D9160017220433F61804ABD2182F
:10D32000FF23BE4234D31370A16E8B69C969C91A39
:10D33000B14235D301210292039101962A6800215E
:10D34000009220002200FEF7CFFB002802D003004D
:10D3500054331BD1A36E21009A6901235B420B93C6
:10D360000BAB02930192009620002B680A92FEF705
:10D37000A7FF002802D00300543307D12900200062
:10D380003D4A0AABFFF711FF002809D00DB0F0BDF0
:10D39000390014398E4200D90E001370BE42C3D238
:10D3A00004ABDB7DA022DB430421DBB2D200DB092E
:10D3B0009B186A6849428A1A92191B0513432F4A1F
:10D3C0000AA91A43AB68079253401BBA0422E868C3
:10D3D0000A9302F07DFB2300103305930823E860D5
:10D3E00003930AAB02936B680B9001932B682200A6
:10D3F0000093200000230599FFF744FE0028C5D1C3
:10D40000049B002B04D16B6804330493EB680693F0
:10D4100004ABDB7D079ADB431B06DB0FDB075340C6
:10D42000AB6001235B426E60EB60B74206D9A36E2E
:10D4300062699B6A9B18B34200D946E7220020002C
:10D440000599FFF711FF002800D13EE79EE704226F
:10D45000049B029601920093210020002B68FEF7A6
:10D460002FFF002800D091E70A9B002B00D18DE709
:10D4700046E7C046FE03000008FCFF5F00FC0F000B
:10D4800082690B6810B54C689A4210D1C369A342F7
:10D4900011D08B68CC68A34205D15B000A60C269D9
:10D4A000CB6000234A60002001338B6010BDA24294
:10D4B000EFD1C469EBE754204042F7E70023F0B511
:10D4C0008FB00AAD93610133D36114002A00194B68
:10D4D00005900E0083CB83C21B68136027001837AA
:10D4E0003800FEF73FFA002801D002201FE0290093
:10D4F0002000FFF7C5FF002818D1059A07AB079257
:10D50000326821000892726803930B4B09920293D0
:10D510000A4B3A00019000930598094BFEF7FCFE78
:10D520000222831C9343D9D00FB0F0BD5420404257
:10D53000FAE7C0463034031015BE00100800002082
:10D54000FF03F07FF0B595B0049204001C220D009B
:10D550000CA80021059317F01FFD012313934B4BDB
:10D5600008AAC1CBC1C21B68136012A80CAEFEF79B
:10D57000F9F9002806D08027A66A7F02002E51D133
:10D5800030003DE0300008A9FFF77AFF002800D006
:10D5900079E0B1690498A847002831D1F16904986D
:10D5A000A84700282CD13100200012AAFFF7D2F89A
:10D5B000002825D106000CA98B8AB342D5D9344B5B
:10D5C000B20206AF13432000324A0097FEF7FCFB7D
:10D5D000002804DA831C13D10136B6B2EBE72E4BD8
:10D5E000000D98420ED1049B019502937B682200A6
:10D5F000009300212000069BFFF7DCFA0028EBD007
:10D6000015B0F0BD059B002BE6D080239B0098420F
:10D61000E2D106990498A8470028F1D10799049807
:10D62000A847EBE7B379012B01D03668A6E788223B
:10D63000336B52031340BB4216D09022336B52031C
:10D640001340802292029342EFD13100049B019556
:10D650000293736B220000932000B36B4031FFF7FD
:10D66000A9FA0028E1D0CBE73100049B0195029391
:10D67000F36A220000932000B36A4031FFF79AFA60
:10D680000028DAD0BCE754204042B9E73034031018
:10D690000800002000FC0F700202000010B504001A
:10D6A000406DE36DE16EC01815F0E8FB0023E36503
:10D6B000A36E6165DA6A216ED3008B4200D90B003C
:10D6C0000021A365606E17F067FC01232200200093
:10D6D0000549FFF737FF002804D00023A365E36561
:10D6E000E36E236610BDC0461FBA0010F8B50400F3
:10D6F0000D000127A16DE36D8B4208D3236E002B33
:10D700002FD02000FFF7CAFF0028F3D020E0072029
:10D71000666EDA08B25C1840C2403A4219D1606DB8
:10D72000E16E181815F0AAFB012229600721A56DEA
:10D73000E36D206E01330138E3652066AB420ED203
:10D74000D808305C0B40D840030010401342EFD1A2
:10D75000F8BD0133E365236E013B2366CBE7002070
:10D76000F6E71C204042F3E77FB50C0004310600C9
:10D77000FFF7BCFF051E2FD121003000FFF7B6FFD9
:10D78000051E29D1220004230832A06001900393D2
:10D79000029222680100009230003200FEF7A4F9E4
:10D7A000002802D00300543319D1B36E5B6A002BFA
:10D7B0000ADD0121A66801331943013E76183000C5
:10D7C00015F05CFB761AA66004230022E360053B9B
:10D7D00023616261A361E361280004B070BD0500AC
:10D7E000FAE70000F0B504000D0089B0200007A999
:10D7F000FFF77CFF061E0AD1079B20001900059346
:10D80000FEF77EFB061E62D00300543361D0300069
:10D8100009B0F0BD802029002A6B4003DB1B40319A
:10D82000024229D0012202A8039212321218029257
:10D830000197A888294A80020243009220000A002A
:10D840003839FEF7D9FC002814D10123210002AA9F
:10D85000039312339B180293059B22000093200030
:10D86000012301971031FFF70DFC002812D00300AF
:10D8700054332ED00600CAE7012202A803921232C6
:10D88000121802920197AA6B200000922200FEF764
:10D890002BF9D8E70137EB6BBB42BBD8A36EE1692C
:10D8A0009A6AE86C17F07EFB21002369A06E2B6456
:10D8B000636910316B64A369AB64FFF7BEF9059B24
:10D8C0002A6BAB6380239B0213432B639FE7070004
:10D8D000E1E701235B42236188E7C0460000102096
:10D8E000F0B593B00A930B6B06000D000992DB02B2
:10D8F0001DD54A6B0A9BC96AD3188B4200D20B0014
:10D90000F16F994213D2F36EEA6329003366300057
:10D91000FFF768FF2B6B041E06D08022120313430F
:10D920002B63200013B0F0BD874A13402B630A9B82
:10D930000593059B002B01D10A9CF2E780218022F0
:10D940002B6B890292021940134204D0B26EEF6B26
:10D95000D26997424ED16F6BDB0200D5E2E000291D
:10D960001CD1002F1AD02B001191403311A9AA6AA3
:10D970000493EB6A02912900013F38310191300094
:10D9800004990097FFF759F8041E03D080232A6BEF
:10D990001B03C4E70499B06EFFF74FF9F36E3366CB
:10D9A0002B0040330B93AB6B0C936B6B07933000E6
:10D9B0000FA9FFF79BFE041EE8D10F9B3000190052
:10D9C0000493FEF79DFA041E06D023005433DDD1E4
:10D9D00001235B422B64EAE7079BB76E002B2BD138
:10D9E000049BAB63079B1F00EB6380232A6B9B02A6
:10D9F00013432B63B36EDB69DF1B059B9F4200D98A
:10DA00001F002900099B03970293EB6B32000193DF
:10DA1000AB6B3000009340310123FFF733FB041E52
:10DA200000D182E003005433B0D129003000FFF769
:10DA3000D9FE041EE5D0A9E7079B3800013B10A9D9
:10DA40001093FEF7DBFF109B01330893089A1093A5
:10DA5000FB6906929A424CD1013015F0DBF90300C4
:10DA60002700013306930C9B08901193BB000D9384
:10DA70000423039311AB0293BB000193049B320078
:10DA80000093300001230B99FFF7FCFA041E9CD190
:10DA9000089BBB4235D1069B0137BB42E6D8049BAD
:10DAA000AB63069B9F00EF639FE7012311AA0292DD
:10DAB0000C9A03930092002132003000069B0197DC
:10DAC000FEF712F8041E00D060E70123039311ABA8
:10DAD0000293049B32000093300001230B990197BD
:10DAE000FFF7D0FA069B0400013B0693002800D004
:10DAF0006BE7089B069A9F1A002AD6D1049BAB635A
:10DB0000D1E70423039311AB0293BB000193119B54
:10DB100001000093320004233000FDF7E5FF041EEE
:10DB2000B9D033E702235B42E9E76B6BDB196B6328
:10DB3000EB6BDB19EB63099BDB190993059BDB1B83
:10DB40000593F36E3366F4E6FFFFEFFFF0B50B6B62
:10DB500005000C0099B05A0307D5DA0202D401225D
:10DB600052420A64334A134023639A0302D40020CA
:10DB700019B0F0BDE26A1900019280225203676B6E
:10DB80001140134242D103AE3000542217F004FA80
:10DB9000A36A2A000D93019B10970E9301230F9304
:10DBA00013AB43CA43C30126126876421A602E6043
:10DBB000626BE36A9A4212D3210001232A002800F3
:10DBC0004031FFF707FA002826D003005433CFD1A5
:10DBD00021002800FFF706FE0028EDD0C8E702AAC2
:10DBE00001232800033203A9FEF76CFF0028BFDBE6
:10DBF00002AA0123210028000332FFF771FE00284A
:10DC0000B6DB2B680133D3D01396D0E7019A3B00E3
:10DC1000974200D213006363A36B226BA362636B12
:10DC20006763E362044B1A4080235B021343236360
:10DC30009DE7C046FFFFFBFFFFFFFDFFF0B51E00A5
:10DC40000B6B85B005000C0001929A0705D4204BA0
:10DC5000204A2148214918F0A3F85B0316D4236B0E
:10DC60001A0519D4676B6A6FB91991422DD89B03B5
:10DC700018D5330021002800019AFFF731FE002853
:10DC800008DB236B164A1340236303E0FFF75EFFB4
:10DC90000028E4D005B0F0BDE26A616B8A42E1D9A8
:10DCA0006263DFE7E36A9F42E3D96363636B9F428A
:10DCB000DFD9002302AAD3712100280001330732E3
:10DCC000FFF70EFE0028F1DAE4E71B204042E1E70F
:10DCD00022030310EC3203109AFC02104B0E0000DA
:10DCE000FFFFF7FF002307B5044901AA0193FFF7DF
:10DCF00029FC002800D101980EBDC046DDBA0010F5
:10DD00000023F0B587B002AD93610133D3611400F5
:10DD10002A00144B01900F0043CB43C21B681360D1
:10DD2000260018363000FDF71DFE002802D0022024
:10DD3000404212E029002000FFF7A2FB00280ED18C
:10DD400039003000FDF719FE002806D0320021000E
:10DD50000198FEF7FFFC0028E2D007B0F0BD542088
:10DD6000E6E7C04630340310F0B50D009DB00E93C9
:10DD700022AB0D9204CB04001B880F920B9324ABB3
:10DD80001B880C93836EA868596A0130A86000292B
:10DD90001FDC00230A9300230993012200236968F2
:10DDA00016AE52421691B260F260A26E7360336199
:10DDB000D36C002B40D0083B20007361FEF7A0F825
:10DDC00000283BD00300543300D0D1E00A9B0993D4
:10DDD00010E001260131314315F050F80029D8D167
:10DDE0001691280016A91796FDF7C7FD0A96002878
:10DDF000D1D009960123002601275B422800236128
:10DE000016A916961797FDF7B8FDB0420CD0200062
:10DE1000291DFFF76BFCB04209D003001C3300D072
:10DE2000A6E0099BB34205D11C204042A0E00A9025
:10DE30000997B2E70A96B0E7D369BCE72A00042342
:10DE4000310020000832FFF791F90028BAD111AB58
:10DE50000793484B020006930B9B20005B421BB2CA
:10DE600005930C9B0F9904930B9B11940393424BC6
:10DE7000129602930E9B01930D9B009301235B422C
:10DE8000FEF75CF800289DD12F0018373800FDF709
:10DE900069FD00280DD1C022EB7DD2009B18374AC6
:10DEA0001B051A4331003B002000FFF77EF90028D4
:10DEB00088D10C22002113A817F06EF8099B002BC3
:10DEC00009D1210013A83C31FDF773FD210013A8EF
:10DED0003031FDF76EFD210013A84831FDF769FDD3
:10DEE000139B29009B0A9B02200013AA1393FDF7A2
:10DEF00077FF00283CD113A8FDF765FD002808D165
:10DF000020001F4A13AB16A9FFF74FF9002800D0D5
:10DF100058E716AE31002000FFF7C2F9002800D004
:10DF200050E77768A36E3800996914F0A7FF0029BD
:10DF300005D0144B144A1548154917F031FF20003D
:10DF40002B686A686B602A600C9B0B9AEF609B1AC7
:10DF5000AB82B3680C222B61483017F01DF8099B87
:10DF6000002B04D1230030343C3307CC07C309987D
:10DF70001DB0F0BD5BD2001000FC0F4008FC0F008C
:10DF80000CFCFF7F4F030310703303109AFC021048
:10DF900024080000F0B593B0089318AB079204CBA7
:10DFA0000AAE1B880C00069331001AAB05001F88CF
:10DFB0000992FFF7D9FB0590002824D1E37D3100B9
:10DFC000F375A36928001093E369079A1193069BE0
:10DFD00002970193099B0093089BFFF7C5FE002859
:10DFE00014DB012329000A9F0B9E2000A761E66134
:10DFF000E3752031FDF7C1FC002804D1069B002BFE
:10E0000001D12F626E62059813B0F0BD0590FAE75A
:10E01000F0B59DB00A93229B0D920A9ADB009B18E3
:10E020000F93C023DB0007000E0000249C4601254F
:10E030000F9B9A4229D1002C53D1B37D002B00D0E5
:10E040006DE001235B423B61B38A099300230B938C
:10E050000B9A099B9B1A0C93012B00D9FBE00B9B9D
:10E06000002B00D030E1BB6E596A002900DD40E191
:10E07000099B310002930023380001930A9A229BE6
:10E080000096FFF771FE040030E11368BA48190DDD
:10E090000B0009914905490D814204D1B38A01332E
:10E0A000B3820832C4E7B54881420CD1B38A002B51
:10E0B00005D1B34BB34AB448B44917F071FE013BE4
:10E0C0002C00B382EDE7E021C9000B406345E8D1A5
:10E0D0005368099819682840B1615B68F075F3616D
:10E0E000DFE7B38A002BA8D1239B002B04D1A84BD8
:10E0F000A44AA548A749E0E731003800239AFFF772
:10E10000FFFD041E04D0831C97D020001DB0F0BD7D
:10E11000239BDB7D002B00D18FE7022480E00121CF
:10E120003368B86E16AD49421693F2683369E960F8
:10E13000C16C6A60AB602A6100291ED00839696130
:10E1400011A9079194493800069100210591049185
:10E15000039102912299119701910A9912950091C8
:10E160003100FDF7EBFE041E09D023001C3300D163
:10E1700067E723005433C8D163E7C169DEE70C22A7
:10E18000010013A816F008FF390013A83031FDF77D
:10E1900010FC390013A83C31FDF70BFC390013A823
:10E1A0004831FDF706FC139B13A89B0A9B021393AF
:10E1B000FDF709FC00280ED13100380013AAFDF745
:10E1C0000FFE041EA1D129003800744A13ABFEF7DC
:10E1D000ECFF041EC9D116AD29003800FFF760F826
:10E1E000041EC2D16B680993BB6E0998996914F03B
:10E1F00045FE002904D06A4B624A634869495CE7DE
:10E20000099B3A00F360AB68303233613B003C332A
:10E2100023CA23C338000C222100483016F0BCFE6C
:10E220000D9B1B6816930D9B5B681793BB6A099344
:10E23000099B002B00D168E7099B16A90833180039
:10E240000B93FDF79AFB002800D185E0099B1B6822
:10E25000EDE70995FAE66B4616A99B8D07915249A1
:10E26000039306915942514B00220293229B09B21B
:10E2700001930A9B059100930123099938000491A9
:10E280005B4231001692FDF759FE041E2ED1BB6E83
:10E29000DD6C002D00D1DD690C9AFE2A0FD899693A
:10E2A0006B084C1EE418200014F0E8FD283D641AA9
:10E2B000AC4200D92C00169B9C4200D3CFE60C9BAD
:10E2C0000B9A5B08D318C2E66B469D8D099B310003
:10E2D00002933800229B0A9A01950096FFF75AFE96
:10E2E000041EB6D003001C3300D1BCE6002C97DA24
:10E2F0000BE70125B06801310130294314F0BEFD60
:10E30000002900D0B4E61691300016A91795FDF744
:10E3100034FB0B90002800D0AAE63800FFF7E2FC9F
:10E32000041E00DAF1E6FB6E1C1ADB089C4200D8E2
:10E330009EE6099B310002930B9B380001930A9AD9
:10E34000229B0096FFF726FE041E03D003001C3319
:10E35000CCD18DE609958BE632000B9B23CA23C3F3
:10E3600023CA23C303CA03C30B9B0D9A934233D022
:10E37000024B0A999C462AE001040000FF040000B9
:10E38000750303109D3303109AFC0210C8080000A7
:10E3900084030310D50800005BD200100CFCFF7F43
:10E3A0004F0303101F090000C9BA001000FC0F4002
:10E3B0000D686800400D604544D12B039B0D9A42C7
:10E3C00032D10123099A5B429360D3600831099BE3
:10E3D0009A880F9B9942EBD1099B9B880C93099BD0
:10E3E0009B8B0E930E9A0C9B934200D22EE7099BB7
:10E3F000DB7F002B00D129E73900099B2031203336
:10E4000018001D00FDF7B9FA002804D00E9A0C9BE5
:10E410009B1A099A93802A0038000B99FEF79AF903
:10E420000028D9D0040070E69A42CFD9099B013A5E
:10E430009A809B79022BC9D1099B9B6A013B099A5F
:10E440009362C3E7084B9842C0D12B039B0D9A42BD
:10E45000BCD3099B01329A809B79022BB6D1099BD0
:10E460009B6A0133EBE7C04601040000F0B50700EA
:10E470000D009FB0866A03920493002E57D12A00A4
:10E480002B6806936B6807930EAB13CA13C313CAAA
:10E4900013C303CA03C30193049B2A0000933800EB
:10E4A000039B0EA9FFF7B4FD041E6CDB280006A930
:10E4B000FDF763FA002807D12B000EAA43CA43C315
:10E4C00043CA43C303CA03C3022C25D13A0029001F
:10E4D00038004832FDF784FC041E54D1C022169B3C
:10E4E000D2000693179B16A90793EB7D01909B180A
:10E4F000914A1B0513430A930123380000931835F2
:10E500000AAB06AA0B95FFF783FD041E3BDB202216
:10E5100016A90EA816F046FD00230493012C00D185
:10E520008FE00024049BA3422DD003342BE0300065
:10E530000830A84201D136689FE72900FDF71DFA8F
:10E540000028F8D1B379012BF5D18022336B520327
:10E550001342F0D0BB6EF26A9B6A9A42EBD9736B9E
:10E560003100F363FB6E38003B66FFF73BF9041E96
:10E5700009D1336B714A3100134038003363FFF720
:10E58000E5FA041ED7D020001FB0F0BD290006A870
:10E590000831FDF7F2F9002801D1AE60EC60AB79EB
:10E5A000022B08D1290006A82C31FDF7E6F9002836
:10E5B00001D1EE622C632D684FE001213800FEF797
:10E5C000D5F9380016A93030FDF70BFA5C4C0399E9
:10E5D0002300002810D03A6B5A4913030A403A63CB
:10E5E000039A039912039B0D7D63BD63920D9342C1
:10E5F00002D20A0054495118169E179D002208960F
:10E600000995A34202D0514A9B021A430A92002262
:10E610000C910EA90B920D91019202320AAB00925D
:10E62000380008AA16A9FFF7F3FC041EABDB01288B
:10E6300036D1202216A90EA80696079516F0B2FC30
:10E640000494390006A82031FDF797F90E9E0F9C1F
:10E65000002801D13E627C62BD6A002D96D138004F
:10E6600016AA06A9FEF72AFF031E0390A5DA0233B5
:10E670005FD1059516AE06AD320029003800FFF7D0
:10E680003FFB041E0FD0831C00D07CE7039B9F1C24
:10E6900000D146E72E4B2F4A2F48304917F080FB18
:10E6A00001230593E6E73B6B9B0504D0059B3800EF
:10E6B0005942FEF75BF9380031003030FDF791F92F
:10E6C0001F490B00002808D03A6B1E481303024074
:10E6D0003A6300229B0D7A63BA63169A06927268B7
:10E6E0006A6000228B4202D0184A9B021A435F21C3
:10E6F0000A92002204AB5B18C0210B921B78C90060
:10E700005B180D491B050B430C93022301920093E8
:10E7100038000EAD0AAB06AA16A90D95FFF778FCD6
:10E72000041E00DA2FE72022280016A916F03AFC72
:10E73000F4E6039C27E7C04608FC0F00FFFFEFFF4D
:10E74000FF030000FF03008000FCFFFF0000F04F0C
:10E7500089030310EF3303109AFC0210FB09000039
:10E76000F0B5036BA3B0040003919B054FD00026C6
:10E770000AAD1C220021280016F00EFC0123EB75C7
:10E78000EB610023029310A8FDF7ECF8002804D0F9
:10E79000029B002B31D00026EBE712AF390020009E
:10E7A00010AAFDF7D7FF00280BD1EB7D002B1ED15F
:10E7B00020001AAA10A9FEF781FE002829DA831C7E
:10E7C00057D023B0F0BD914237D1059A33E0226B88
:10E7D000354913030A40226300226263A263334A6D
:10E7E0009B0D934230D09A02314B13432DE02022EF
:10E7F000280012A916F0D6FBC5E7012E01D001268C
:10E80000B7E7216B2000494249B2FEF7AFF800207C
:10E81000D7E7002EEBD104AF0300264A2000009773
:10E820001AA9FDF7D1FA0028CBDB0499109B119AA5
:10E830009942C8D1059B9342D9D020000AA9303013
:10E84000FDF7CFF80028C2D10023069300230793D9
:10E85000194B09970893022306AA0AA92000FFF77B
:10E8600005FE0028ADDB033843425841029B0343B9
:10E8700088E7002EBBD0039B002BB8D022003900C4
:10E8800020004832FDF7ACFA00289AD1C022FB7D67
:10E89000D2009B18094A1B051343069318AB079334
:10E8A0002900012306AAD9E7FF030080FF03000027
:10E8B0000000F04F00FCFF7F08FC0F6008FC0F0019
:10E8C00010B50400FFF7D2FD002804DB03D00021BF
:10E8D0002000FFF745FF10BD10B5036B040090B09A
:10E8E0009B0523D5020008A92032FDF733FF00283D
:10E8F00026D1294A02AB0292A26E0193D26901236A
:10E900000392E26E20000492226F08A90592626FC2
:10E910000692A26F0792214A00926A46FFF7D0FF43
:10E9200000280DD1236B1E4A13402363E022E36BC2
:10E93000D2001B0D134205D101212000FFF710FF6B
:10E9400010B010BD174A5B055B0D934205D0164B06
:10E95000164A1748174917F023FA220020004032C0
:10E9600008A9FDF7F7FE0028EAD1E36B226B1249F4
:10E970001B030A409B0D11499B020B43226302AA11
:10E9800002936063A06350600123200008A9FFF791
:10E9900097FF0028D0D0D3E7010002001800102014
:10E9A000FFFDFFFFFF040000AE03031062330310FE
:10E9B0009AFC021065130000FF0300800000F04F76
:10E9C00073B5140002000E00483221000500FDF767
:10E9D00007FA00280FD1C022E37DD2009B18064A17
:10E9E0001B0513430093183401236A4631002800A5
:10E9F0000194FFF765FF76BD08FC0F00F0B5802796
:10EA00000B6B3F0305000C0089B03B424ED1FFF772
:10EA10009DF8266B002803D03743276309B0F0BD6B
:10EA2000F30343D52300083318000193FCF79AFF42
:10EA300000283BD180277F033E4220D0E36CE66A6A
:10EA40001B48A188000589020E4330430490206DC5
:10EA50000593836804AA194381235B050B439360E4
:10EA600043680199D36028000223FFF729FF236B35
:10EA7000002818D08022120313432363CEE7290015
:10EA80002A0028001031FEF7EFFB0028C6D1236BC7
:10EA90003B42D3D1220002AB1900283241CA41C106
:10EAA00008260448CDE7044A134023630020B5E755
:10EAB0000102000002020000FFFFFEFF70B505002A
:10EAC0000C00FFF79BFF2B000600AA6A2833002AE0
:10EAD00004D01A6894420AD122681A60236D1B6818
:10EAE000002B02D1E06C11F059FF300070BD130013
:10EAF0001268ECE770B58CB014001E000191002381
:10EB000001AA04A90500FDF731FE00281CDB0F4B0C
:10EB10000003800D984207D12A002800203204A962
:10EB2000FDF718FE00280FD1C0239B00E418109BAE
:10EB300024051C438002044302AA0123280004A9DF
:10EB400002945660FFF7BCFE0CB070BDFF030000DE
:10EB5000F0B50D0006001400496B85B0002B0DD0F8
:10EB60005418012B0AD00C00022B07D12B6BEC6A36
:10EB70009B0302D58C4200D20C001419736FA34280
:10EB80002DD38C4202D1200005B0F0BD2B6B5B036E
:10EB90001DD5B76EEA6BFB699A4218D00291380016
:10EBA00002A9FDF72BFF03A9019038000394FDF79C
:10EBB00025FF019B83420AD16B6C039A934206D8CE
:10EBC000A96C5B189A4202D26C63EA63DBE7290006
:10EBD0003000FEF7BBFF0028D6D16C63D3E71620C8
:10EBE0004042D1E7F0B51F008BB006000D00039244
:10EBF000BB0731D4109B30002B6500236B63EB63A4
:10EC0000EB642B000833029302992F632B1D03AA98
:10EC1000FDF7ACFD041E08DA831C00D075E00398F4
:10EC2000FDF714F9002800D16FE00123AB71B36A3E
:10EC30002B60B562A31C49D1FF0566D5039C6C49C6
:10EC4000200019F0DFFC215C00293DD1336F8342A5
:10EC500009D22424644258E0FFF73EFE041EC9D0C6
:10EC600020000BB0F0BDAB88624F9B021F4304979E
:10EC7000802718437F0338435F4F04AA3B43136147
:10EC8000516003239060516130000299D460FFF716
:10EC900017FE030004001C33DBD0002835D13C00F4
:10ECA00000272B6D9A68BA4239D81B68002B68D0B0
:10ECB000EB642900B06E4031FDF7BFFF4F4A230DD2
:10ECC000934267D00024CBE71424C3E7BB0500D5EB
:10ECD00087E0240D012C00D085E0AA8892027F05F0
:10ECE00007D58023444C5B0214432A6B13432B63E8
:10ECF000D6E7434B300013432A0028320092029992
:10ED0000404AFDF761F8041ECADA80232A6B1B0310
:10ED10001343290030002B63FFF7D0FEA0E7012149
:10ED20002A6B0A4204D1296B8B071CD40137B8E740
:10ED30000C21C02079435A68AB88521891689B0215
:10ED40000B43117880005268091809050B430092A3
:10ED500030002D4A0299FDF737F80028E3DA831CCA
:10ED6000E1D00400D1E70C222B6D7A435B689B183D
:10ED70009A68B36F9A4238D880235B020B432B63A7
:10ED8000D4E7B36E986A11F0E1FDE864002890D1F1
:10ED90000C245FE78023296B5B030B432B63002369
:10EDA00002226B64B36EA4059B6A5242A40DAA6250
:10EDB000EC622A64AB6485D0AA88144992028B4223
:10EDC00000D90B001A4380239B051343EA6C3000E3
:10EDD000009202990B4AFCF7F7FF041E00DB71E773
:10EDE00093E7112436E7152434E71C2432E7C046A4
:10EDF00063FC02100000104000001020010200001F
:10EE00000800002000FC0F7000FCFF7FFE030000E4
:10EE100070B596B005000E00FDF71AFF041E04D071
:10EE20000C246442200016B070BD336A002B05D15B
:10EE30002A4B2B4A2B482C4916F0B2FFAB6E21000F
:10EE4000DA6A686E16F0A8F8AB6EEA6EDB6A6C657B
:10EE5000DB00934200D91300AB6500230EAE3100F6
:10EE60002800EB652A66FEF77FFC041E31D11F4A9D
:10EE70001F490292AA6E0891D2691E490392EA6E56
:10EE800002AB04922A6F05926A6F0692AA6F0792EC
:10EE90000A91194908AAD16018495060116153615B
:10EEA000310003232800FFF70BFD041E11D10300DE
:10EEB0000200B07531002800FFF702FD041E08D1E2
:10EEC000012300906A46310028000193FDF742FCBF
:10EED00004002800FDF77AFDA4E7C046DF03031015
:10EEE0001C3403109AFC02102C11000001000200D7
:10EEF000000010400800F00FF50303101800102068
:10EF0000F0B59DB00400FDF7A3FE0590002800D0E9
:10EF1000A0E014AE01001C22300016F03DF80123E1
:10EF2000F3614E4B0AAA23CB23C21B6813601AA8B5
:10EF3000FCF718FD002814D0226BD30F9B18236315
:10EF40002200230030323C3323CA23C3E56EE06A3B
:10EF5000290013F093FF00236165A365E36525662F
:10EF600073E030000AA9FEF78BFA002800D06FE0AA
:10EF70003B4A07AB0892082203933A4B099202934B
:10EF8000394B0190009331002000384B1AAA0794A6
:10EF9000FDF7C2F9051E54DB002849D08505AD15E3
:10EFA000013545D033680EAF236273683100636268
:10EFB00020002F4B2D4A0097FCF706FF051E40DB73
:10EFC0000E9B99B21B0C022B02D016256D4238E025
:10EFD0000129FAD8236B274A134001224A405202E2
:10EFE00013432363FB68002B03D0226F9342ECD8BA
:10EFF00023673B69002B03D0626F9342E5D86367B8
:10F000007B69002B08D0A26F9342DED8E26FA36722
:10F010009A4200D91A00E267A36EBA68196A0029F9
:10F0200001D09142D1D1E266DB697A689A42CCD1B3
:10F030002200310020003032FCF7D2FE051E00D144
:10F0400075E72000FDF7C2FC059505981DB0F0BDE1
:10F050005425BBE70C235B420593F6E730340310DD
:10F06000F503031031C900100800F00F00FCFF7F0A
:10F0700018001020FFFDFFFF10B5FDF7A7FC0020D2
:10F0800010BD0000F0B59BB004000591FFF724FC13
:10F09000002846D1030005AA200008A9FDF766FB59
:10F0A00000283EDB2C4A03039B0D934250D0A26AFA
:10F0B0009B021092020D10AE0292039306AD022A3B
:10F0C0001FD1039A254B200013430095244A08A919
:10F0D000FCF77AFE002824DB2A00200012A9FDF7A5
:10F0E00039FB00281DD1179A1E4B170027201F40FF
:10F0F0001A422ED101212000FDF738FCB771B780EC
:10F10000A662039A184B20001343069300232A009B
:10F110006B6008A90133FFF7D3FB109BA3620028A3
:10F1200001D01BB0F0BD029B022BFAD101212000BF
:10F130004942FDF71BFC200008AA12A9FEF7E0FDDA
:10F140000028EED1200012AA08A9FFF739FCE8E751
:10F1500016204042E5E7C046FF03000008000020FB
:10F1600000FC0F70FFFF00FF0000F04FF0B5B3B0E0
:10F1700005000A910B92FFF7AFFB041E00D091E04F
:10F1800003000AAA28000EA9FDF7F0FA041E049055
:10F1900000DA87E003038C4F9B0D0393BB4202D13F
:10F1A000162464427EE00E2606ABF61833002800D3
:10F1B0000BAA16A9FDF7DAFA041E6CDB03039B0DFC
:10F1C000BB42EDD016A90EA8FCF7D7FBAB6A0590A1
:10F1D0001E93A31C00D06FE00B9F7C49380019F0F0
:10F1E00011FA3B5C002B04D0049B1B0D022B00D0BA
:10F1F000E2E02B6F834200D2E0E0059B002B54D06D
:10F200002B6B734A1340039A92021343714A1343C0
:10F210002B630E9B6B630F9BAB63A31C00D086E03C
:10F22000039B0693002328930E23002206A95B1854
:10F230001F88694BBF023B432A930B9B29921800FE
:10F240002B926249079319F0DDF9049B059A1B0D77
:10F250001B053B4303432C93079B28AE7361039B21
:10F260001F435E4B3B43B36100230EAFF7619A42ED
:10F2700003D1069B9A02574B13433362002332009B
:10F2800073622800053316A9FFF71AFB00285CD02B
:10F290001E9BAB6257E0831C04D10B98FCF7D6FD94
:10F2A00000288FD1200033B0F0BD002303993288AD
:10F2B00091425B41CB18B4E70499220D090D8A42B3
:10F2C00005D0023A531E9A41153A1400EAE705990F
:10F2D0003388002974D10399994201D10024E1E7D0
:10F2E000022A24D19A023E4B28AF134328003D4AFC
:10F2F000009716A9FCF768FD002824DB3A002800D7
:10F3000020A91EAEFDF726FA00281CD1259A364BFF
:10F3100017001F401A4214D101212800FDF726FBD7
:10F32000059BB771B780AE62002B00D068E70E2353
:10F3300006AA9B181A88274B92021343039A069237
:10F3400071E7272040420400ACE7059B002B19D051
:10F35000E0222B6BD200190D114213D01C4A6863B6
:10F3600013402B63039BA86399021A4B0CAA0B430F
:10F370000C935060012339002800FFF7A1FA002800
:10F3800000D085E71E9BAB62A31CA7D0240D022CE6
:10F39000A4D1012128004942FDF7E8FA280016AA65
:10F3A00020A9FEF7ADFC041E00D07BE7280020AAB0
:10F3B00016A9FFF705FBC6E71424F2E62424F0E6BD
:10F3C000022A00D01CE78DE7FF03000063FC021057
:10F3D000FF0300800000F04F0000104000001010FC
:10F3E0000800002000FC0F70FFFF00FF70B58AB01E
:10F3F00001911600002301AA02A90500FDF7B6F944
:10F40000041E10DB2F21019816F07EFD002802D08B
:10F41000230D022B0AD1220333002800920D02A9EA
:10F42000FCF728FD040020000AB070BD14246442DB
:10F43000F9E7000070B58CB014001E0003910023A2
:10F4400003AA04A90500FDF791F9002823DB144B5A
:10F450000003800D984207D12A002800203204A919
:10F46000FDF778F9002816D1C023AA6F9B001099E8
:10F47000E3181B058A4200D90A00134380020343A4
:10F48000084A2800009604A9FCF79EFC002804DA2C
:10F49000831C00D13B380CB070BD8005800DFAE7AD
:10F4A000FF03000000FCFF7F37B5069C856FAC4270
:10F4B00003D80094FFF71EFB3EBD1C204042FBE733
:10F4C000F7B50400806A0D0016001F00FCF799FADA
:10F4D000002805D0074B084A0848094916F060FC87
:10F4E000084B32002900009320003B00FFF77AFB15
:10F4F000FEBDC046FE030310543303109AFC0210F5
:10F50000E71700004833031070B50400806A0D004F
:10F51000FCF777FA002805D1054B064A064807494B
:10F5200016F03EFC29002000FFF7C8FA70BDC04667
:10F53000FF030310363303109AFC02100B1800006F
:10F5400070B50400806A0D00FCF75BFA002805D155
:10F55000054B064A0648074916F022FC2900200000
:10F56000FFF74CFA70BDC046FF03031028330310A9
:10F570009AFC02101B180000F8B50500806A0C0008
:10F5800016001F00FCF73DFA002805D10E4B0F4A6C
:10F590000F48104916F004FC236BDA0704D40E4B15
:10F5A0000E4A0B480E49F5E79B0306D43B00320098
:10F5B00021002800FDF786FAF8BD21002800FEF79B
:10F5C000C5FA0028F2D0F7E7FF0303101A3303103F
:10F5D0009AFC02102D180000350403100B330310A1
:10F5E000E40D0000F8B50400806A0D0016001F004D
:10F5F000FCF707FA002805D1064B074A07480849D7
:10F6000016F0CEFB3B00320029002000FEF716FB6F
:10F61000F8BDC046FF030310FC3203109AFC021031
:10F620003F180000F8B50400806A0D0016001F00A6
:10F63000FCF7E7F9002805D1064B074A07480849B7
:10F6400016F0AEFB3B00320029002000FFF780FAE5
:10F65000F8BDC046FF030310DE3203109AFC02100F
:10F6600051180000F0B5050087B0806A0C00160044
:10F67000FCF7C7F9002805D1444B454A454846499F
:10F6800016F08EFB226B930704D4444B444A414846
:10F690004449F5E7002E00DA75E0676BE36A9203F0
:10F6A00002D5BB4200D23B009E4255D2EB6F9E4238
:10F6B00031D8002321001A002800FFF749FA00285A
:10F6C00027DB01235B422B60210033002800EA681E
:10F6D000FDF7F8F900281CDBA823216B5B030B4323
:10F6E0002363002302226364AB6E52429B6AA262D0
:10F6F0002264E06C3200E968E662A36415F052FC13
:10F7000000233A0021002800FFF722FA002800DD3C
:10F71000002007B0F0BD21002800FEF717FA0028EE
:10F72000F7D105A9A26AE36A02912100383101915B
:10F73000711E00912100059040312800FDF77DF9F0
:10F740000028E6D1A36B226BA362A023DB02134344
:10F750006663E6622363D3E79E42D1D90223002287
:10F7600021002800FFF7F4F90028D2DB636B9E42EA
:10F77000C6D96A460023210013752800013305AA63
:10F78000FEF75CFAF0E716204042C2E7FF030310E1
:10F79000CC3203109AFC02106218000022030310FE
:10F7A000B9320310AB0E000010B5806A0C00FCF7F4
:10F7B00028F9002805D1044B044A0548054916F0EC
:10F7C000EFFA606B10BDC046FF030310AB320310AD
:10F7D0009AFC02107218000010B5806A0C00FCF749
:10F7E00010F9002805D1074B074A0848084916F0C8
:10F7F000D7FA236BE06A9B0303D5636B984200D270
:10F80000180010BDFF0303109D3203109AFC021074
:10F810008F180000F0B5A9B005000391FFF75CF860
:10F82000041E12D1AB6A28001E9302AB023303AA56
:10F8300020A9FCF79BFF0400831C09D1039B18003F
:10F840000093FCF703FB002807D1200029B0F0BD8E
:10F850000028FADB11246442F7E73A49009818F0CF
:10F86000D1FE2B6F0190834269D3EB6E28002B668B
:10F8700006A9FDF779FF041EE7D10EAE2022300065
:10F8800020A915F08FFBF37D14AA002B50D12E4B2D
:10F89000059204932800012304AA06A9FFF710F893
:10F8A000041ED2D11EAFFB7F002B19D001212800EE
:10F8B000FDF75CF8244B3100169306AB1793280034
:10F8C0000123AF6216AABC71BC80FEF7F9FF1E9B34
:10F8D000041EAB62B9D1012128004942FDF746F868
:10F8E00002AB5B8819499B021943169100218020C5
:10F8F000179101998003194301431891009916AAA1
:10F90000D16013490B4306A9136151611EABDB7F24
:10F91000D161581E83410F485B4203400A4820A929
:10F920001B18936128000423FEF7CAFF04008CE72C
:10F9300031002800FCF70EFF041EA4D085E7242424
:10F9400089E7C04663FC021008FC0F60000010400D
:10F9500008000020F803F09FF0B5050087B0806A2A
:10F960000C001600FCF74DF8031E05D01F4B204A73
:10F970002048214916F014FA039626000836310073
:10F98000280003AAFCF7F2FE00282ADB030D022B55
:10F9900029D11A4B0003800D04AF984216D12B6A6F
:10F9A00004936B6A7B603A0031002800FCF7D2FEBA
:10F9B000002816D1A368A080E362E368A0622363F5
:10F9C0000223A371AB6A2360AC620AE00C4B800295
:10F9D0000343310028000B4A0097FCF7F5F9002893
:10F9E000E1DA07B0F0BD14204042FAE762040310E8
:10F9F000903203109AFC0210AE180000FF030000C2
:10FA00000800002000FC0F700300826A2833002ADF
:10FA100004D01A68914203D10A681A600020704726
:10FA200013001268F3E70000F8B5150084220C00FB
:10FA3000060000212800520015F0AEFAA36A002B40
:10FA40000BD1023318492B70280008301CF06CFAD7
:10FA50000120A36A0133A362F8BD0227012B02D162
:10FA600012492F70F0E7A288A38B93420DD1E07F5B
:10FA70000028F1D022002100300020320831FCF7AC
:10FA800069FE0028E8D10200A08021002B00300090
:10FA90000831FCF7EFF9831CBB43DDD1A3880133A8
:10FAA000A3800230DFD0D3E715FD021014FD021051
:10FAB0000A0010B52C320C000831FCF74BFE002870
:10FAC00001D1A080A06210BD10B5FEF70BF910BDEA
:10FAD00070B50F250A4C8A18914200D170BD0B7881
:10FAE000060958402840800000591B0946407340D1
:10FAF0002B409B001B59300958400131ECE7C046B0
:10FB00004034031080234A1E70B55B0105009A4201
:10FB100000D31900FF23FF31686899430C000028C7
:10FB200004D0AB688B4205D015F078FC200015F0AE
:10FB30008BFC68602968AC60220015F033FA002362
:10FB40002B7370BD03000020814206DB9A688A4255
:10FB500003D95B68181E00D0585C704710B50029A7
:10FB60000CDB83688B4209D94368002B06D05C18F4
:10FB70005B5C934202D001232270037310BD00002E
:10FB80008368F7B50400181E03D0237B002B01D136
:10FB90000120FEBD6368181EFBD0214D2B78002B81
:10FBA00001D111F081F91F4B01931B7A002B04D076
:10FBB0002F78002F21D000E000BFF02680212068A0
:10FBC0003606801949011FF0C3F92068A2686168F0
:10FBD00080191FF095F9019B1B7A002B1BD012484E
:10FBE0001FF06EF90022114B1A702B78934210D13E
:10FBF00011F038F900232373CAE70B481FF010FAFD
:10FC00000A4E0B48377015F0EDF93378002BFCD015
:10FC1000D3E700E000BF2B78002BEBD1E8E7C0462C
:10FC20006683012088690020946900206783012091
:10FC30002ED0DEC0034B044A1A6000225A609A603C
:10FC40001A7370479089002000F0FF10F0B585B05E
:10FC500017001E0005000C0012F0CAF900230A4A22
:10FC600080185941002902DA012008494042002346
:10FC70000290039100933A0033002100280012F013
:10FC80008AFD05B0F0BDC04650C30000FFFFFF7FF6
:10FC9000F0B585B017001E0005000C0012F0A8F9A1
:10FCA00000230A4A80185941002902DA0120084934
:10FCB000404200230290039100933A003300210058
:10FCC000280012F04FFD05B0F0BDC04650C3000043
:10FCD000FFFFFF7F73B56B46DE1D00230178337095
:10FCE0000400320040680133FFF7B0FF0500012037
:10FCF000002D0BDC237B002B07D0054818F012FDEC
:10FD00002900327803481CF055FB002076BDC04620
:10FD100098040310BC04031070B5040004A805ADDA
:10FD20002D780078638162602170657220720321F2
:10FD300011F0E2FA607A032111F0DEFA207A002253
:10FD4000012111F0FBFA0022607A012111F0F6FA8C
:10FD5000FA21638989005943606812F0BDFC3220A2
:10FD600012F082F92000FFF7B5FF70BD70B50C1CD2
:10FD700005000021201C14F027FF002800D0054CAE
:10FD80008B202C61211CC00514F0DBFE14F0A4FFB5
:10FD9000A88270BD33335340642310B543810023E0
:10FDA0000400037301338375FFF7E0FF200010BDEB
:10FDB00073B50B00050003291CD0052928D00129A3
:10FDC00030D101786A464068FFF740FF6E46040074
:10FDD0003078002C0DDC2B7B002B09D0124818F05A
:10FDE000A1FC210011481CF0E5FA642012F03CF956
:10FDF0000F4876BD6A4601784068FFF727FF6B46DB
:10FE000004005A7898780002104340BA80B2E0E7C4
:10FE10006A4601784068FFF719FF6B460400DA78FC
:10FE20001879F0E70024D6E7F20403101205031056
:10FE3000FFFF0000012110B5FFF7BAFF034A0300DE
:10FE40000020934201D01B06D80F10BDFFFF000019
:10FE500073B51500040020222800904340281FD0CD
:10FE6000002D01D0012076BD18010B0A01AA034321
:10FE700013705170022321786068FFF709FF051E97
:10FE8000F0DC237B002B09D01B4818F04BFC290029
:10FE90001A481CF08FFA642012F0E6F80020E2E71E
:10FEA00009015B0001AA89B22B4313700B0A53703E
:10FEB0009170032321786068FFF7EAFE061E08DCD4
:10FEC000237B002BEAD00E4818F02CFC31000B48A5
:10FED000DFE7602DC6D12000FFF7ACFF0028C1D1BD
:10FEE000193012F0C1F82000FFF7A4FF0028B9D1A3
:10FEF000193012F0B9F8B5E72B05031050050310BF
:10FF00006905031070B5847D002C07D080250C1C7A
:10FF10006D01A94201D303490C88A1B2FFF798FFF4
:10FF200070BDC04680340310F8B51F00837D040007
:10FF300016000D1C002B0BD0006914F053FE002896
:10FF400015D10021281C14F04DFE0021884208D153
:10FF5000A08A14F06DFE291C14F007FE14F0BCFEFC
:10FF600081B23B0032002000FFF772FFF8BD01496B
:10FF7000F7E7C046FF0F0000F0B587B00E00150090
:10FF80000021172268461F006C4615F005F8002076
:10FF9000162F02D9854202D1172007B0F0BD0E4BB3
:10FFA0000E4A2380FE235B42A3800633FF33637235
:10FFB0000B4B2282638103220A4BE274A38101234B
:10FFC00005322275694628000F32A670E373A375C7
:10FFD00014F0E8FFE0E7C046090400000705000050
:10FFE0000580FFFF030800007FB5FF230493039300
:10FFF00002930193E23B00931B221A21013B054827
:020000041001E9
:10000000FAF736FB0022044B1A71044A1A6007B053
:1000100000BDC046D4960020A4DB00208C34031021
:1000200010B50368014A1B6A984710BD130400000D
:1000300010B5094C112120000FF07AFD102120008D
:100040000FF0B4FDE12120004902FFF7E9FF012094
:1000500010F0BEFA10BDC046808A002070B50400C2
:10006000074D28000FF050FC012010F0B1FA2800D5
:100070002100FFF7D5FF012010F0AAFA70BDC0469D
:10008000808A0020344B10B518680B280BD801214A
:100090001EF09EFF064B4D4F51535557595B5D5F08
:1000A000062010F0AFFE062010F098FA002106207E
:1000B00010F0A8FE0021072010F0A4FE0021082067
:1000C00010F0A0FE0021092010F09CFE00210A2063
:1000D00010F098FE00210B2010F094FE00210C205F
:1000E00010F090FE00210D2010F08CFE0021142055
:1000F00010F088FE0021152010F084FE002116204B
:1001000010F080FE0021172010F07CFE042010F07B
:1001100065FA8021114B1A6B114B1A60114A126853
:1001200011631A68104B1A6010BD0720B9E7082048
:10013000B7E70920B5E70A20B3E70B20B1E70C20A9
:10014000AFE70D20ADE71420ABE71520A9E7162097
:10015000A7E71720A5E7C046A89800200000205078
:10016000A0DB00209C09002030302050F0B5802218
:1001700089B00720634911F0E5F90121072011F04A
:1001800091F9614C6149206812F0DCFB604B2568F5
:100190001C6803000933C2011B0313435D4A012796
:1001A000134005935C4B0E2207935C4B2100069392
:1001B00080235B030290049328000223009712F02F
:1001C000DBFB574B0E20EE18360D0636F6B231002B
:1001D00011F092F831000F2011F08EF823003A0050
:1001E0000833DBB29A404F4B1826EB181A603B00DD
:1001F000A34039002B630720039311F053F921002A
:100200007443029A04AB280012F006FC2C19464BEA
:10021000D8342360454B039A23602B68072113438E
:100220002B60062010F08EFD0721080010F08AFDDB
:100230000721082010F086FD0721092010F082FD1B
:1002400007210A2010F07EFD07210B2010F07AFD17
:1002500007210C2010F076FD07210D2010F072FD13
:100260000721142010F06EFD0721152010F06AFD03
:100270000721162010F066FD0721172010F062FDFF
:100280000021062010F0BEFD0021072010F0BAFD6D
:100290000021082010F0B6FD0021092010F0B2FD69
:1002A00000210A2010F0AEFD00210B2010F0AAFD65
:1002B00000210C2010F0A6FD00210D2010F0A2FD61
:1002C0000021142010F09EFD0021152010F09AFD51
:1002D0000021162010F096FD0021172010F092FD4D
:1002E0003000082110F02EFD3900300010F08AFD9A
:1002F000032010F06DF90021300010F083FD09B0EB
:10030000F0BDC046850001109C0900209034031008
:10031000EC7C0120FFFFFF9FCE3D10240000061063
:100320000000E0AF2C21000026E0000046E00000C5
:1003300010B50D4C52012060FF2049000240E13809
:1003400001400A43012B00D11A433220140610F059
:1003500045F9064B50201A68054B1B6804339B0077
:100360009C5010F03BF910BDA89800209C0900207B
:10037000EC7C0120F0B5002785B00090B94252D145
:1003800038233D004343294A9B185A1D15330392D5
:100390000293039B5B575A1C42D00026DBB20193A9
:1003A000029B019A9B57934237D1009A204C12012D
:1003B000204BD2195200D5541F499B1820005E7063
:1003C0000FF02DFE0A22009920000FF0B4FE1B4909
:1003D00020000FF024FE0A22290020000FF0ABFEBF
:1003E000174920000FF01BFE0A22310020000FF0F9
:1003F000A2FE144920000FF012FE0A2201992000EB
:100400000FF0B3FE104920000FF009FE0023320068
:10041000290000980137FFF78BFF0136082EBFD166
:100420000135102DB5D1380005B0F0BD3C110020CC
:10043000688A0020FCB40120351503108E050310D6
:100440009205031096050310C718031070B50E002F
:1004500000250F4CC0010419E068431C0FD00D4B60
:10046000626B1860531C02D0E1694B1C0CD10A4B23
:100470001B78002B03D0094909480FF0D0FD013546
:100480000434042DE8D170BD3300FFF751FFF6E7C7
:10049000ECE80020A89800208B8401209C05031024
:1004A000688A002008220E4B0E4910B55A500E499A
:1004B00000245A500B210D4AFE2099500C4A043159
:1004C0009C500C4A99500C4A0E399C50FFF7BEFFC5
:1004D000142010F07DF82100FE20FFF7B7FF10BDBB
:1004E000ECE800200C7F0000107F00001C7F000063
:1004F000347F0000207F0000387F0000F7B5002621
:10050000324B0093324B1B68B34200DCF7BD009BBB
:100510001D78002D54D101213000FFF797FF2D4B9E
:100520001B78002B4CD02C4C2C4920000FF077FD71
:100530000A22310020000FF0FEFD294920000FF0B3
:100540006EFD300008F09EFA200026490FF067FD8E
:10055000009F7A3FF86808F0EBFC1F4C224920000E
:100560000FF05DFD0A22290020000FF0E4FD1F4B73
:100570002000190001930FF052FD0A22F9692000B2
:100580000FF0D9FD1A4920000FF049FD0A22290079
:1005900020000FF0D0FD019920000FF040FD796B95
:1005A0000A2220000FF0C7FD0135200011490FF08D
:1005B00036FD0437042DCDD120000F490FF02FFD5B
:1005C000009B0136803300939CE7C04666E900201B
:1005D000DCE800208B840120688A00209E0503103F
:1005E000A4050310451D0310A7050310AC05031057
:1005F000AF0503101E0603100A0C0310044B10B5C0
:100600001868012112F062F9024B186010BDC04653
:100610009C090020EC7C012007B5C9004118082284
:10062000684614F0BFFC0098019903B000BD10B5F6
:1006300000220FF07DF810BD0A21435E0200181E53
:1006400001D01B01D01870474A6803008868103237
:10065000904203D2012300200B7470475A6810386F
:100660008860002A08D0811A09115181586000233E
:1006700043810372C360F0E71860F7E7F0B50378D1
:1006800089B0040001912B2B11D0002204922D2B54
:1006900002D101342C3B049323781A00303A092A02
:1006A00002D900202E2B70D1002600271EE0002347
:1006B0000134F0E7884B9F4220D802D1874B9E42FD
:1006C0001CD80023300039000A2214F043FC002318
:1006D000060003930F00EB4302954A1C01D1984298
:1006E0000CD8029A039BB6185F41013423781D0091
:1006F000303DEDB2092DDDD9002B2DD00023802512
:1007000005936D03AF424DD225002B780293303B09
:10071000092B54D9059B1B1BEB181BB20593029B9D
:100720002E2B07D16B7801351C00303CE4B20293CC
:10073000092C46D92023029A00249A43452A00D046
:100740008AE069782D2955D10122AB1C9A214900F4
:1007500000240A258C4676E0049B002B17D08023CA
:100760001B069F42CAD801D1002EC7D1019B019917
:100770001A7A7F239A43753B1343019A137200231D
:100780007242BB410A604B60012009B0F0BD019B81
:100790001A7A7F239A43773B1343019A1660576076
:1007A0001372F1E70023300039000A2212F0A4FB93
:1007B000059B060001331BB20F000593A2E701352C
:1007C000A3E7474B9F42ADD802D1464B9E42A9D8E2
:1007D0000023300039000A2214F0BCFB00230793E9
:1007E000059B0694013B1BB2069E079F0593361896
:1007F0004F4197E722006B1C2B29A7D1AB1CA5E723
:100800006C430C190599091961451BDD019B7F2477
:100810001B7A002A0ED0049A00200021002A01D061
:10082000802109060C22A3431343019A10605160F2
:100830001372A9E7049A0020002A01D02A49F1E79F
:100840002A49EFE70133197802913039C8B20928F3
:10085000D6D9002A00D064420020029B834200D0F7
:1008600093E7059B300039001C1912F055FE204B10
:1008700006000F000593002C01DD1E4B0593E317C6
:10088000E4185C40002C11D1049B002B03D0802184
:1008900009067B181F00019B1A7A7F239A43733B3A
:1008A0001343019A1660576013726DE701231C42CF
:1008B0000BD002990598FFF7AFFE02000B00300045
:1008C000390012F052FD06000F00029D6410013540
:1008D000EBB20293D6E7C0469999991999999999DB
:1008E00099990100989999990000F0FF0000F07F14
:1008F000B0340310F8340310002310B50400436033
:10090000FA208000A0600A482060086849682061D9
:100910006161994202D0486801304860A361E36197
:10092000236262620FF067FEE060200010BDC046E7
:10093000D8480310F0B56A4C85B02000F2F750FD9E
:10094000684B1B78002B08D0674D684928000FF0D2
:1009500093FB210028000FF09DFB654D20002A002D
:100960006449F3F729FE2A0020006349F3F724FEC7
:10097000624F20003A006249F3F71EFE614B2000EF
:100980001A0061490193F3F717FE604E2000320010
:100990005F49F3F711FE5F4D20002A005E49F3F72F
:1009A0000BFE320020005D49F3F706FE2A0020000E
:1009B0005B49F3F701FE5B4E200032005A49F3F722
:1009C000FBFD5A4D20002A005949F3F7F5FD32008E
:1009D00020005849F3F7F0FD2A0020005649F3F7AC
:1009E000EBFD320020005549F3F7E6FD2A00200018
:1009F0005349F3F7E1FD320020005249F3F7DCFDE3
:100A00002A0020005049F3F7D7FD20004F4A5049F3
:100A1000F3F7D2FD4F4D20002A004F49F3F7CCFDEC
:100A20004E4B20001A004E490293F3F7C5FD4D4B83
:100A300020001A004C490393F3F7BEFD4B4B2000F6
:100A40001E001A004A49F3F7B7FD2A002000494961
:100A5000F3F7B2FD2000029A4749F3F7ADFD2000FD
:100A6000039A4649F3F7A8FD320020004449F3F702
:100A7000A3FD3A0020004349F3F79EFD3A00200011
:100A80004149F3F799FD2000019A4049F3F794FD9D
:100A90002000019A3E49F3F78FFD3E4F20003A00B7
:100AA0003D49F3F789FD3D4E200032003C49F3F704
:100AB00083FD3C4D20002A003B49F3F77DFD3A00C1
:100AC00020003A49F3F778FD320020003849F3F767
:100AD00073FD2A0020003749F3F76EFD05B0F0BD25
:100AE000F47C012086840120688A002022060310FD
:100AF00057060310EF0503105B0603106206031090
:100B00006606031070060310740603107F060310B8
:100B1000830603108B0603108F060310970603103D
:100B20009C060310A1060310A5060310AB060310D4
:100B3000AF060310B5060310B9060310BD06031077
:100B4000D1060310E4060310F1060310FD0603109E
:100B5000010703100B0703100F07031017070310FB
:100B60001B07031023070310270703102F07031089
:100B7000330703103B07031040070310450703101A
:100B80004A0703104F07031050070310F30F031019
:100B9000F90F0310530703105707031061070310E1
:100BA0006507031070070310740703105A0703103A
:100BB000680703107707031073B5844D2B78002B5B
:100BC00003D0834983480FF057FA0A226946502020
:100BD00015F024F9804C6A4620008049F3F7ECFCBC
:100BE0000A226946512015F019F96A4620007C490D
:100BF000F3F7E2FC0A226946522015F00FF96A4623
:100C000020007849F3F7D8FC0A226946532015F0F2
:100C100005F96A4620007449F3F7CEFC0A226946BA
:100C2000462015F0FBF86A4620007049F3F7C4FC33
:100C30000A226946472015F0F1F86A4620006C49FF
:100C4000F3F7BAFC0A226946482015F0E7F86A462D
:100C500020006849F3F7B0FC0A226946492015F0E4
:100C6000DDF86A4620006449F3F7A6FC0A226946CB
:100C70004A2015F0D3F86A4620006049F3F79CFC3F
:100C80000A2269464B2015F0C9F86A4620005C49E3
:100C9000F3F792FC0A2269464C2015F0BFF86A4629
:100CA00020005849F3F788FC0A2269464D2015F0C8
:100CB000B5F86A4620005449F3F77EFC0A226946DB
:100CC0004E2015F0ABF86A4620005049F3F774FC4B
:100CD0000A2269464F2015F0A1F86A4620004C49C7
:100CE000F3F76AFC0A226946542015F097F86A4621
:100CF00020004849F3F760FC0A226946552015F0A8
:100D00008DF86A4620004449F3F756FC0A226946EA
:100D1000562015F083F86A4620004049F3F74CFC52
:100D20000A226946572015F079F86A4620003C49A6
:100D3000F3F742FC0A226946582015F06FF86A461C
:100D400020003849F3F738FC0A226946592015F08B
:100D500065F86A4620003449F3F72EFC0A226946FA
:100D60005A2015F05BF86A4620003049F3F724FC5E
:100D70000A2269465B2015F051F86A4620002C498A
:100D8000F3F71AFC0A2269465C2015F047F86A4618
:100D900020002849F3F710FC0A2269465D2015F06F
:100DA0003DF86A4620002449F3F706FC2B78002B17
:100DB0000BD0084E210030000FF06CF92B78002B7F
:100DC00003D030001D490FF057F973BD8684012010
:100DD00022060310688A0020F47C01206C100310A6
:100DE000751003107E10031087100310CC10031031
:100DF000D0100310D4100310D8100310DC1003100F
:100E0000E0100310E4100310E8100310EC100310BE
:100E1000F01003100710031012100310F810031045
:100E2000FC1003100011031004110310081103102B
:100E30000C11031010110310141103100A0C0310ED
:100E4000F0B59448A5B0F2F791FA0022431E06933C
:100E5000914B1A60914B1A600493914B1B7893420B
:100E600003D0904990480FF007F90024012527008E
:100E700007228E4909A814F095F88D4A0B218D4B55
:100E8000009202950BAA01940EA8F2F719FB8A4B67
:100E90000721009309AB1A000294019519A8F2F7F3
:100EA0000FFB0594059B069A93424CDC01230193AA
:100EB0000023784D3A0000930EA919AB2800F3F7F0
:100EC0005FF9764E7D4F31680790C901C9190EA8A8
:100ED000F2F7BDFA724B1B78002B0BD0724C78499D
:100EE00020000FF09CF833680A22DB012000D9595A
:100EF0000FF025F90123019300232800079A00939E
:100F00000EA919ABF3F73CF9644E6C4D316807003C
:100F1000C901043149190EA8F2F799FA604B1B7800
:100F2000002B0CD0604C674920000FF078F8336834
:100F30000A22DB01ED18200069680FF000F9584E15
:100F400032787B1C2AD10025544B554F1D603B78CD
:100F5000AB4200D087E05C48F2F786F90FF04BFB1C
:100F60005A4E5B4D3368C01A2B783060002B13D07B
:100F70004D4C584920000FF052F82B78002B0BD025
:100F80000A22200031680FF0E4F82B78002B03D000
:100F9000200051490FF070F825B0F0BD3E493F4D9B
:100FA0000B6801330B602B6801332B60002A31D0B2
:100FB0003D4C4A4920000FF032F80A223900200047
:100FC0000FF0BDF8464920000FF029F83148F2F73C
:100FD000CDF90A22010020000FF0CFF83378002B62
:100FE00018D00A22200029680FF0A5F83378002BCA
:100FF00010D020003B490FF012F83378002B09D0B5
:101000000C212A68384B4A439B1820000A22596851
:101010000FF095F8059B0133059343E7224C3349C4
:1010200020000EF0FCFF049B244E1B680A22DB010B
:10103000995920000FF07FF82A4920000EF0EFFFA9
:10104000049B0A221B682000DB01F61871680FF070
:1010500072F8200026490EF0E2FF049B049A1B68F8
:101060000135013313600C4C2368AB42D6DC3B786E
:10107000002B00D16FE70C4D1E4928000EF0CFFF6A
:101080003B78002B00D166E70A22280021680FF088
:1010900056F860E7F47C0120FCE70020F8E7002028
:1010A000868401207F070310688A00201808031037
:1010B000670F0310210B0310FAF60210ECE8002072
:1010C0009C070310A507031080E80020247D012061
:1010D00087840120F4070310FC070310AE070310F8
:1010E000BC070310DC20031004DC0020531B03109A
:1010F000DF070310E2070310F0B53A4D3A4C2B78A6
:1011000085B0002B19D0394E394930000EF0B4FFAC
:101110002B78002B11D0210030000EF0BBFF2B7874
:10112000002B0AD0300033490EF0A6FF2B78002B9D
:1011300003D0300030490EF09FFF00222F492000DD
:10114000F3F7E4F800222E4906002000F3F7DEF85A
:10115000002207002B492000F3F7D8F80123039061
:101160000193731C00D10196012302937B1C00D1D3
:101170000297039B013309D02000F2F7F7F8039A96
:101180000300210020000132F2F72AFE019B1648DD
:101190001D4C012B21D1029B012B1ED13B00721C47
:1011A0002100F2F71DFE2000F2F728F92B78002B22
:1011B0000BD00E4E210030000EF06CFF2B78002B70
:1011C00003D0300011490EF057FFFFF7B3FBFFF7D4
:1011D000F3FCFFF735FE05B0F0BD012300225B42B2
:1011E000DEE7C0468684012080E80020688A00206F
:1011F0001F08031032080310570803105908031082
:101200008B09031059F70210F47C01205B080310CE
:10121000F7B5754C2B212000FEF794FCFF2846D132
:1012200000222B212000FEF799FC00222021200023
:10123000FEF794FC002221212000FEF78FFC002203
:1012400022212000FEF78AFC002223212000FEF745
:1012500085FC002225212000FEF780FC00222621AB
:101260002000FEF77BFC002224212000FEF776FC04
:10127000202227212000FEF771FC1C2228212000BB
:10128000FEF76CFC232229212000FEF767FC0022D8
:101290002A212000FEF762FC00221F212000FEF719
:1012A0005DFC2000FEF76CFC05200FF091F9202179
:1012B0002000FEF747FC421E90414C4B2121187044
:1012C0002000FEF73FFC421E9041494B222118703E
:1012D0002000FEF737FC421E9041464B2321187038
:1012E0002000FEF72FFC421E9041434B2521187031
:1012F0002000FEF727FC421E9041404B262118702B
:101300002000FEF71FFC421E90413D4B2821187023
:101310002000FEF717FC3B4F272138702000FEF716
:1013200011FC394E292130702000FEF70BFC374BA1
:101330002421187020000193FEF704FC421E904106
:10134000334B1F2118702000FEF7FCFB314D2A2182
:1013500028602000FEF7F6FB2F4B1D2118602000AF
:10136000FEF7F0FB2D4B1860012804D900221D2147
:101370002000FEF7F3FB3B783B78C82B06D91C22F4
:1013800028212000FEF7EAFB1C233B7033783378DA
:10139000C82B06D9202227212000FEF7DFFB2023BF
:1013A0003370019B1B78019B1B78C82B07D9232224
:1013B00029212000FEF7D2FB2323019A13702B680A
:1013C000002B09D02B68012B06D000221F21200002
:1013D000FEF7C4FB00232B602000FEF7D1FB0520A5
:1013E0000FF0F6F8F7BDC0469089002086840120F2
:1013F00087840120898401208A8401208B84012034
:101400008C84012015830120148301201683012080
:1014100088840120D86C0120A06C0120785F002016
:1014200070B5744C0B2815D81DF0D2FD6F0625320F
:101430003F4C59D914A2C8D120212000FEF782FBCD
:101440006D4D002810D1012220212000FEF786FBDF
:1014500001232B7004200FF0BBF82000FEF790FB57
:1014600008200FF0B5F870BD002220212000FEF703
:1014700075FB0023EDE722212000FEF763FB5F4DA3
:10148000002802D101222221DFE700222221EDE7FC
:1014900025212000FEF756FB594D002802D10122DC
:1014A0002521D2E700222521E0E726212000FEF7B2
:1014B00049FB544D002802D101222621C5E7002214
:1014C0002621D3E724212000FEF73CFB4E4D0028C7
:1014D00002D101222421B8E700222421C6E72A21D3
:1014E0002000FEF72FFB494D002807D101222A21B9
:1014F0002000FEF733FB01232B60ABE700222A21FB
:101500002000FEF72BFB0023F6E70022202120001D
:10151000FEF724FB002221212000FEF71FFB002202
:1015200022212000FEF71AFB002223212000FEF7D3
:1015300015FB002225212000FEF710FB00222621AA
:101540002000FEF70BFB002224212000FEF706FB03
:101550000023294A13702E4A1370284A13702D4A0B
:101560001370274A1370274A1370274A137071E7C4
:10157000012220212000FEF7F1FA01222121200082
:10158000FEF7ECFA012222212000FEF7E7FA012201
:1015900023212000FEF7E2FA012225212000FEF798
:1015A000DDFA012226212000FEF7D8FA01222421AB
:1015B0002000FEF7D3FA01230F4ACBE700221F21B8
:1015C0002000FEF7CBFA0022134B1A6042E70122FB
:1015D0001F212000FEF7C2FA01220F4BF5E70F4D45
:1015E0002B68002B02D101221D2181E700221D2141
:1015F00086E7C046908900208684012089840120E6
:101600008B8401208C84012088840120A06C01201F
:10161000878401208A840120D86C0120785F002013
:1016200070B5124C050004212000FEF78BFA01284A
:101630001AD0012204212000FEF790FA2A0001218D
:101640002000FEF78BFA2000FEF79AFA01211820FD
:101650000FF0D8FB01200EF0BBFF002118200FF087
:10166000D1FB034B034A1A6070BDC046908900202D
:101670000CED00E00400FA0510B5034B0200012157
:101680001800FEF76BFA10BD9089002010B5040019
:10169000054B03602030F9F7E7FD20001430F9F71F
:1016A000E3FD200010BDC046D8480310F7B5002662
:1016B0000D0004004B684A6943608B688360CB6807
:1016C000C3600B694E610E61016903614369426148
:1016D00001A800910193F9F7C7FDAB692A6AA361DC
:1016E000EB692E62EE61E169E361236A01A822627F
:1016F00001930091F9F7B8FD6B6A6362F7BD0000D2
:1017000030B591B005000EF076FF304B30491860CF
:1017100003A80EF0BFFE0A22290068460EF0F8FE6C
:10172000694603A80EF039FF2A490EF043FF2A4B01
:1017300002002A4906A80EF0DDF8294C06A920006F
:10174000FFF7B4FF06A8FFF7A1FF68460EF054FEAE
:1017500003A80EF051FE20000EF025F8214B1B7857
:10176000002807D1002B03D01F4920480EF084FC2D
:1017700011B030BD002B1AD01D4906A80EF08AFE0C
:101780000A22290003A80EF0C3FE03A906A80EF042
:1017900004FF18490EF00EFF144B010018000EF064
:1017A00061FC03A80EF028FE06A80EF025FE124DDF
:1017B0002800F1F759FD21002800F3F72BFA20004B
:1017C0000EF017F8FFF798FCD2E7C046247D012001
:1017D0008E230310620B0310741F0310CC890020AA
:1017E00008E80020868401205F080310688A002032
:1017F00077080310A108031080E80020F0B5A14C81
:10180000A149A544050016A802920EF043FE0A2243
:10181000029910A80EF07CFE10A916A80EF0BDFECD
:101820009A490EF0C7FE9A4B02009A4920A80EF082
:1018300061F8994C20A92000FFF738FF20A8FFF796
:1018400025FF10A80EF0D8FD16A80EF0D5FD20003B
:101850000DF0A9FF914B1B78002808D1002B03D075
:101860008F4990480EF008FC8F4B9D44F0BD002B33
:1018700003D08E498B480EF0FFFB8D4E3000F1F700
:10188000F3FC21003000F3F7C5F920000DF0B1FFA3
:101890000A220BA9280014F0C1FA302120231B20B2
:1018A00004AA52181370013904AA1F3B8018891822
:1018B000C25C1C000133002A00D080E030202021CF
:1018C00004AD2D182955EA540027202601977848A1
:1018D0000199F1F7D3FF002822D0142370210124AD
:1018E0007B4304AA5218D654019B714D190028005D
:1018F0000093F1F7C3FF631C0393019B0133019332
:101900002C2861D114227A4320AB9B18621C1E55EF
:10191000985400221B199A700137642FD7D10027E1
:1019200020AD2C000026B74200D085E0604C20009E
:10193000F1F79AFC20005F49F3F7BBFA002300930C
:10194000009B9F4200D087E05B492000F3F7B1FA8B
:10195000514D28000DF04DFF4B4908A80EF09AFD9F
:101960000A22029905A80EF0D3FD05A908A80EF0D9
:1019700014FE46490EF01EFE504B0200454916A8C3
:101980000DF0B8FF16A92800FFF790FE16A8FFF784
:101990007DFE05A80EF030FD08A80EF02DFD2000FC
:1019A000F1F716FD041E06D019F09EFB210002007F
:1019B00028000DF082FE28000DF01BFF54E7CA54EA
:1019C000142B00D074E77FE728000099F1F756FF49
:1019D0002D280DD114237B4320AAD3181E55621C39
:1019E000023498541E550134132C00DC7CE793E735
:1019F00028000099F1F742FF0A2806D1300014238D
:101A00007B4320AAD3181855EDE728000099F1F779
:101A100035FF0D28F2D028000099F1F72FFF7B2821
:101A2000ECD028000099F1F729FF7D28E6D02800A6
:101A30000099F1F723FFE2E7200010A916F094F8CF
:101A4000002806D012222021200013F0A5FA00233E
:101A500023700136143466E72B78002B04D1009BE9
:101A60001435013300936BE70026A95D0029F6D0F9
:101A7000202902D02000F3F77DF80136142EF4D18E
:101A8000EDE7C046ACF7FFFF8E230310620B031097
:101A90008D080310CC89002008E8002086840120EE
:101AA0005F080310688A00205408000090080310A3
:101AB00080E80020590803104D0B0310C4080310E0
:101AC00010B5040090B0164903A80EF0E3FC0A22FA
:101AD000210068460EF01CFD694603A80EF05DFD6E
:101AE00010490EF067FD104B0200104906A80DF0DA
:101AF00001FF0F4C06A92000FFF7D8FD06A8FFF74D
:101B0000C5FD68460EF078FC03A80EF075FC094987
:101B100020000EF084FA20000DF06BFE10B010BD16
:101B20008E230310620B0310C4080310CC8900201D
:101B300008E800209C05031070B5040090B0A2498D
:101B400003A80EF0A7FC0A22210068460EF0E0FC74
:101B5000694603A80EF021FD9C490EF02BFD9C4B1D
:101B600002009C4906A80DF0C5FE9B4D06A9280061
:101B7000FFF79CFD06A8FFF789FD68460EF03CFCC8
:101B800003A80EF039FC28000DF00DFE002800D14E
:101B900018E1924C2000F1F767FB29002000F3F7D1
:101BA00039F828000DF025FE8D4B1B78002B00D056
:101BB000D1E020008B4A8C49F2F7FEFC20008B4AD2
:101BC0008B49F2F7F9FC20008A4A8B49F2F7F4FCC2
:101BD00020008A4A8A49F2F7EFFC2000894A8A49A4
:101BE000F2F7EAFC2000894A8949F2F7E5FC200077
:101BF000884A8949F2F7E0FC2000884A8849F2F7D0
:101C0000DBFC2000874A8849F2F7D6FC2000874A8F
:101C10008749F2F7D1FC2000864A8749F2F7CCFCCD
:101C20002000864A8649F2F7C7FC2000854A86498B
:101C3000F2F7C2FC2000854A8549F2F7BDFC20007E
:101C4000844A8549F2F7B8FC2000844A8449F2F7B7
:101C5000B3FC2000834A8449F2F7AEFC2000834A9B
:101C60008349F2F7A9FC2000824A8349F2F7A4FCD9
:101C70002000824A8249F2F79FFC2000814A824973
:101C8000F2F79AFC2000814A8149F2F795FC200086
:101C9000804A8149F2F790FC2000804A8049F2F79F
:101CA0008BFC20007F4A8049F2F786FC20007F4AA7
:101CB0007F49F2F781FC20007E4A7F49F2F77CFCE5
:101CC00020007E4A7E49F2F777FC20007D4A7E495B
:101CD000F2F772FC20007D4A7D49F2F76DFC20008E
:101CE0007C4A7D49F2F768FC20007C4A7C49F2F787
:101CF00063FC20007B4A7C49F2F75EFC20007B4AB3
:101D00007B49F2F759FC20007A4A7B49F2F754FCF0
:101D100020007A4A7A49F2F74FFC2000794A7A4942
:101D2000F2F74AFC2000794A7949F2F745FC200095
:101D3000784A7949F2F740FC2000784A7849F2F76E
:101D40003BFC2000774A7849F2F736FC2000774ABE
:101D50007749F2F731FC774D002229002000F2F795
:101D6000D5FA411C2000F1F741FD0A2809D02900CD
:101D70002000714AF2F720FC2000704A7049F2F707
:101D80001BFC704E002231002000F2F7BFFA050064
:101D9000431C10D0411C2000F1F728FD0A2804D074
:101DA00031002000684AF2F707FC01222000A91C3C
:101DB0005242F1F777FE210064480EF039F9200015
:101DC000F1F752FA10B070BD8E230310620B0310AE
:101DD000741F0310CC89002008E8002080E8002050
:101DE00086840120EF0503105706031050070310E7
:101DF00062060310F90F0310700603109706031014
:101E00007F0603109C0603108B060310B90603100F
:101E1000AB060310B5060310A10603103B07031021
:101E20000B070310400703101707031045070310A3
:101E3000230703104A0703102F0703105A07031044
:101E40005307031068070310610703107707031097
:101E500070070310D9140310C7080310E41403100B
:101E6000CB080310CF080310D4080310D8080310C0
:101E7000DD080310CC100310E1080310D01003108C
:101E8000E4080310D4100310E7080310D81003105F
:101E9000EA080310DC100310ED080310E010031033
:101EA000F0080310E4100310F3080310E810031007
:101EB000F6080310EC100310F9080310F0100310DB
:101EC000FC0803106C100310FF08031075100310BA
:101ED000020903107E100310050903108710031078
:101EE00008090310071003100B0903101210031048
:101EF0000E090310F810031011090310FC10031051
:101F00001409031000110310170903100411031022
:101F10001A090310081103101D0903100C110310F6
:101F200020090310101103102309031014110310CA
:101F300026090310370B0310290903102D0903107C
:101F4000590803108B0903104D0B0310688A0020F9
:101F5000F0B504000F0093B0431C00D076E00025DC
:101F6000514B05A8190000930EF094FA0A2229009B
:101F700002A80EF0CDFA02A905A80EF00EFB4B4EFA
:101F800031000EF017FB4A4902004A4B08A80191A4
:101F90000DF0B0FC484C08A92000FFF787FB08A80B
:101FA000FFF774FB02A80EF027FA05A80EF024FA3A
:101FB00020000021FEF73BFB20000DF0E2FB05288E
:101FC0003CD8009905A80EF065FA0A22290002A85B
:101FD0000EF09EFA02A905A80EF0DFFA31000EF00D
:101FE000E9FA364B0200019908A80DF083FC08A914
:101FF0002000FFF75BFB08A8FFF748FB02A80EF0E4
:10200000FBF905A80EF0F8F92D49002F13DD2D4935
:10201000AE0020000EF003F80A22711C20000EF022
:102020008AF8294920000DF0FAFFB11C0A2220008D
:102030000EF081F8254920000DF0F1FF1E48013512
:102040000DF0D7FB082D8BD113B0F0BD164905A8B4
:102050000EF020FA0A22210002A80EF059FA02A975
:1020600005A80EF09AFA11490EF0A4FA184B0200D6
:102070000F4908A80DF03EFC0F4C08A92000FFF7FF
:1020800015FB08A8FFF702FB02A80EF0B5F905A89A
:102090000EF0B2F9002F03DD20000E490DF0BFFF56
:1020A00020000DF0A6FBCFE78E230310620B031078
:1020B000CC8900208D08031008E80020C408031014
:1020C0008D09031054090310DC2003108A09031042
:1020D0009227031097090310437C002B06D1C36895
:1020E0005A1CC2601B78037401234374007C704740
:1020F00010B504002000FFF7EFFF031E0BD0093BD3
:10210000DBB2172B03D8074ADA40D20707D40123E2
:102110000020237202E0207A0130C0B210BD0023FB
:102120006374E7E71300800070B505000C002078A9
:10213000002800D170BD2800FFF7CEFF002806D090
:102140002378834205D1002301346B74EFE702202A
:10215000F0E70320EEE770B504000D00FFF7BCFFC9
:102160000023A84201D163740133180070BD73B518
:10217000C2B27F2804D80B68581C08601A7073BD5F
:102180006B46002480251C703F3422406D422A4358
:1021900080095A7082B2C0B21F2A0DD84022524222
:1021A00002439A700333013B1A78002AE7D008688B
:1021B000441C0C600270F6E7204028439609987092
:1021C000F0B20F2E05D8202252420243DA7001AB42
:1021D000E9E7204005431020120B40420243DD7026
:1021E0001A710533DFE70000F7B505000026FFF799
:1021F00073FF6E7401902800FFF76EFF0024019AB0
:1022000003006C74824257D0A04201D1022054E0F6
:102210005C284CD12800FFF75FFF0028F6D0274B41
:10222000752838D104276C742800FFF755FF002863
:10223000ECD0402818D83038C0B20F2833D800224C
:102240002401013F0443FFB223B26A74A4B297424F
:10225000EAD1A02280219201A21892B2C9008A423A
:1022600006D29B059E0DC6E7202398433738E3E747
:1022700090229201A21892B220008A4206D29B05B7
:102280009B0DB002184380235B02C0182900FFF7A2
:102290006EFFB0E702331A78002A04D09042F9D1D9
:1022A0005B78002B01D1032007E000226A742A68C2
